:100000000C94A2150C9450F00C9425F00C94FAEF7B
:100010000C94CFEF0C94A4EF0C9479EF0C944EEF6A
:100020000C9423EF0C94D3150C94D3150C94D31586
:100030000C94D3150C94D3150C94D3150D948D06F4
:100040000C94D3150C94D3150C94D3150C94D31590
:100050000C94D3150C94D3150C94D3150C948EEDED
:100060000C94D3150C9490F30C9466F30C94D31564
:100070000C94D3150C94D3150C94D3150C94D31560
:100080000C94D3150C94D3150C94D3150C94D31550
:100090000C94ECF40C9462F40C94A4F40D944E0BB8
:1000A0000C94D3150C94D3150C94D3150C94D31530
:1000B0000C94D3150C94D3150C94D3150C94D31520
:1000C0000C94D3150C94D3150C94D3150C9430F3D5
:1000D0000C9406F30C94D3150C94D3150C94D315EF
:1000E0000C94D31507634236B79BD8A71A396856C4
:1000F00018AEBAAB558C1D3CB7CC5763BD6DEDFD4A
:10010000753EF6177231BF000000803F0800000006
:10011000BE922449123EABAAAA2ABECDCCCC4C3EFC
:1001200000000080BEABAAAAAA3E00000000BF00EB
:100130000000803F0000000000084178D3BB4387E7
:10014000D1133D190E3CC3BD4282AD2B3E68EC82FB
:1001500076BED98FE1A93E4C80EFFFBE01C4FF7F80
:100160003F00000000000C940A980C9424A40C9406
:10017000DB750C9489340C9403170C9498220C941E
:1001800072160C949E980C94B4C10C9452FF0C946B
:10019000574D0C9432180C9432930C9451590C9482
:1001A000DD720C949A940C94DB7A0C946FC10C94CD
:1001B00028340C9495AA0C94FCE70C9459CE0C941A
:1001C0007EEA0C9413790C944EA60C94741F0C9434
:1001D0003A1C0C94AA7B0C94CE320C94166E0C94A0
:1001E0006F750C94C2330C94BEE70C94D6920C94A9
:1001F0009D800C942C1D0C944EEA0C941FE90C94D9
:100200003D1E0C94D8160C9486160C94E6F80C94AB
:100210005B770C9417EA0D9463130C9410E80C941C
:10022000ADE80D9459020C94BBA30C941F460C949A
:10023000CE170C949F7C0C94F8230C9476EA0C94C3
:100240006B4B0C949B340C94D55A0C94DC340C946A
:10025000B56D0C945F770C944AA70C94FB970C94A3
:100260006BA40C9430A50C94A4340C944ACF0C9439
:100270000E240C94F8240C945B320C9465C60C94F8
:1002800061CE0C9452EA0C9427CF0C94A5CF0C9419
:1002900042CE0D944E040C9476160C94E1250C94E9
:1002A000CC210C94B7330C9491200C940F1D0C941A
:1002B000334A0C94C0230C9464FB0C9416370C94B2
:1002C0005E320C94E51C0C947A7C0C9410860C9491
:1002D00046CE0C945DE90C9480A60C94CD920C94BF
:1002E000AA7C0C94F9340C94BFE70C9432250C943E
:1002F000D0720C941FCF0C94E8240C94F2EC0C9464
:10030000C7A00C94831F0C9495EA0C942CCF0C94EA
:10031000361E0C9485970C9413EB0C9465200C946A
:1003200092F70C94DB5A0C948D500C94AA860C9482
:1003300064320C94724A0C946ECF0C94077B0C942C
:10034000F0160C941E1D0C9447F70C9459770C94DE
:100350002C8F0C949BCF0C9475CE0C941BA00C94FA
:10036000B94B0C94BD330C94B9240C94CD4B0C9424
:1003700038590C94ADFB0C94199F0C945DC10C94EE
:100380001B260C9421740C94C51D0C9416ED0C9432
:10039000324B0C94246C0C94F1EA0D94E6010C940D
:1003A00069EA0C9457C60C94BAA30C94EC450C94CF
:1003B0001B1D0C94DD160C9482160C943ACE0C94F2
:1003C000E4F60C94CB720C947B200C9436CF0C94F6
:1003D000B4330C94AFFA0C94B8A30C94A2740C949C
:1003E0000A1E0C94C86D0C9496750C94DBF60C9454
:1003F00049220C94C8750C9487240C9496EB0C94A9
:1004000010E90C9490750C9471980C940FA10C94B5
:100410000D5A0C942EA00D9471040C942F1F0C9463
:1004200053CE0C949B740C9453250C94CFA90C942C
:10043000CC580C9412450C94A5650C94534D0C9417
:10044000579F0C9472730C948A200C94A7E90C9417
:10045000CC710C94F0EA0C946C750C94514D0C9486
:100460006BE90C945EC60C947E500C94BD4A0C94BF
:10047000807D0C948F280C9495A60C94812F0C945D
:10048000EF340C94B8930C9467CE0C94DA160C9459
:1004900088860C94854B0C94932F0C94F81C0C9428
:1004A00053770C943F750C942C770C9405350C9471
:1004B00079CE0C9402D50C9457770C940DED0C94D6
:1004C0002C300C948A160C946BCE0C94A3840C9450
:1004D00051770C9462EA0C94DB230C94F57B0C941A
:1004E0004FCE0C941AEB0C941C250C9403350C94F1
:1004F000347F0C94FC720C945D250C945DA70C94D5
:100500000A810C9487CF0C94A54B0C94D11C0C94AD
:1005100034CE0C94662F0C943CE90C944D210C9431
:100520006AA40C9426EA0C9442C60C94771C0C9492
:10053000E4250C941EE80C94732F0C9434980C94BE
:1005400091CF0C94B4250C943BC60C94C7320C94F8
:1005500093250C94CB590C94FB800C94C8240C94D8
:1005600056C10C9420870C947EC10C9474CE0C94CC
:1005700058730C9400EB0C947B1E0C9434C60C94B2
:10058000D5150C94EF840C944D870C9401FE0C94BB
:100590002D310C941BFE0C9411300C94AEEB0C948A
:1005A00049C60C944C8A0C94B01E0C9428F10C94FF
:1005B0001FA50C94B2450C94EFEA0C9476840C942D
:1005C0007C240C949C160C9485EC0C94F5230C94D0
:1005D000EDE70C9460E80C9478CF0C94381D0C94E3
:1005E00064CF0C9455770C9425930C945D770C9400
:1005F000514B0C9477210C9412770C9487190C941E
:10060000FC5A0C94D89D0C9408A00C946D1F0C946B
:10061000B02F0C9465210C9412F20C94FDFD0C94F7
:1006200080BA0C949C180C94E6D40C9421980C94E9
:10063000C6160C9499750C94E1800C94BD750C94BD
:10064000B9A30C94BB180C94C6240C94A4380C9435
:1006500077770C9459F70C945ACF0C9438EA0C9491
:1006600019170C949F250C94B9CF0C947FEA0C9425
:10067000D85A0C9493750C94E7750C943ECE0C9458
:10068000BC6D0C9468180C94A4250C9448980C9498
:100690003E1F0C94D37A0C94B5250C9429210C940C
:1006A00083FB0C9426170C9449CE0C9470200C9468
:1006B000D4160D9406060C947D5A0C947A1F0C9453
:1006C000C8840C94BA330C943CAA0C94B79C0C9438
:1006D00070920C94522F0C947D390C9443450C94D9
:1006E00052CF0C94CCEC0C94261F0C94CF220C947B
:1006F00085590C946F860C94D77A0C947A160C94C6
:1007000030750C94FBF60C94A7770C94AD1E0C94EA
:100710009D240C941C810C9448ED0C941AA50C9407
:10072000A1380C94C0E70C947F730C9459980C94E6
:10073000AFCF0C9495E90C9402590C94BDE70C943E
:10074000AEE90C947E160C94291D0C94D9970C9448
:10075000F84A0C94E5D40C9439220C94D1790C9479
:10076000B3220C945DCE0C946BEA0C943B260C9453
:10077000485A0C9405D50C947A870C9485250C94D2
:1007800047EB0C94461F0C9477250D94B7040C94FA
:1007900098740C944D1F0C949DC10C94921F0C9452
:1007A000C9340C9476EB0C9440CF0C94B2590C9451
:1007B00087500C94AF4B0C9461770C94BA750C94E1
:1007C000BC160C94A2FA0C94BD2F0C942F5A0D94C5
:1007D0004E130C94CAF60C94FAEB0C9492340C94CD
:1007E0009B8F0C946FCE0C94B6344E414E494E49BB
:1007F0005459494E46CDCCCC3D0AD7233C17B7D1EE
:100800003877CC2B329595E6241FB14F0A00002093
:10081000410000C84200401C4620BCBE4CCA1B0E12
:100820005AAEC59D746364696E6F70737578585B5A
:1008300000556E6B6E6F776E2073756666697820F3
:1008400000556E6B6E6F776E20636D642000636C75
:10085000724374723A2000454F46002F00496E3AA9
:1008600020003D00494E3A003D004C454741435968
:1008700020494E3A002500C2B04320483D002044A4
:100880004854323220747970652E20543D00494E10
:100890003A00204E6F20656D697420646174612197
:1008A0000020436F756E74657220747970652E2018
:1008B00076616C3D00494E3A0020436F756E746559
:1008C0007220747970652E20494E434F5252454331
:1008D0005420496E74657272757074206E756D6205
:1008E0006572212121004952513A002D3E0020001D
:1008F00023002D3E00200050656E6465643A20237D
:1009000000536574436D643A007375666669784395
:100910006F64653A0020666F7220286D73293A0073
:100920004354524C3A205363686564756C65206388
:100930006D642000206D73203A0041726D65642063
:10094000666F7220002044697361726D65640020D7
:1009500074696D653A004354524C3A205265733ABB
:10096000003D0050696E3A004354524C3A20436FA8
:100970006D6D616E6420626C6F636B65642062797B
:1009800020647269766572206F72206368616E6E92
:10099000656C2066726F7A656E004354524C3A2043
:1009A0004F4E3A416C726561647920416374697697
:1009B000650A004354524C3A2048414C543A416C29
:1009C000726561647920496E6163746976650A00B5
:1009D0004354524C3A20584F4E3A20446973616256
:1009E0006C65640A004354524C3A20584F4E3A41C9
:1009F0006C7265616479204163746976650A0043AD
:100A000054524C3A20584F464620736B69707065BB
:100A1000642E205072657620636D643A0043545210
:100A20004C3A205475726E6564206F66662066725B
:100A30006F6D3A004354524C3A20526573746F7292
:100A400065642066726F6D3A004354524C3A2049F7
:100A5000676E6F7265642C206368616E6E656C20D2
:100A6000636D643D0020457865633A004354524C01
:100A70003A204163746976653A004354524C3A20F7
:100A800048414C543A416C726561647920496E6109
:100A900063746976650A004354524C3A20584F4EAD
:100AA0003A2044697361626C65640A004354524C95
:100AB0003A20584F4E3A416C726561647920416327
:100AC000746976650A004354524C3A20584F4646A2
:100AD00020736B69707065642E2050726576206398
:100AE0006D643A004354524C3A205475726E6564FA
:100AF000206F66662066726F6D3A004354524C3A1E
:100B000020526573746F7265642066726F6D3A006F
:100B10004354524C3A204E6F7420656E6F7567686F
:100B2000206D656D6F727920666F722067726F75C8
:100B300070206F7065726174696F6E00496E7661C6
:100B40006C69642061726700496E76616C6964202B
:100B5000617267004354524C3A20556E6B6E6F774A
:100B60006E2073756666697800536B697070656492
:100B700020686F6D696520737475666600200020BB
:100B80005375623D00204974656D3D004354524CDD
:100B90003A2052414D3D004354524C3A204F757417
:100BA0004F664D656D6F72793A2000282D2920001F
:100BB000282B2920002076616C7565206973200040
:100BC00020756E6B6E6F776E0A005D3D005B0020D6
:100BD000696E76616C6964002000206F6B003A00DA
:100BE000206661696C6564003A00526574727969C7
:100BF0006E6720564354454D5020434D440A0052E1
:100C000065747279696E6720564320434D440A002B
:100C10005265747279696E67206D6F6462757320B6
:100C2000434D440A005265747279696E6720434DE2
:100C3000440A00206572726F723D004D423A207086
:100C40006F6C6C696E6720002056616C3A20004D15
:100C5000423A20004D423A204E6F742073757070F6
:100C60006F727465642072656720747970650A001C
:100C70004D423A20706F6C6C696E672064696D6DCF
:100C8000657220004D423A20496C6C6567616C20AA
:100C9000617267756D656E74730A00206572726F9C
:100CA000723D004D423A20706F6C6C696E67205047
:100CB0004920002D004D423A2050492056616C20B9
:100CC0003A004D423A20706F6C6C696E6720504953
:100CD00020004D423A20706F6C6C696E6720464D63
:100CE000206661756C742000206572726F723D0021
:100CF0004D423A20706F6C6C696E6720002D004D7C
:100D0000423A20464D2056616C203A004D423A202E
:100D1000706F6C6C696E6720464D20004354524CD6
:100D20002F706F6C6C3A204F75744F664D656D6F08
:100D300072793A2000207365632072656D61696E77
:100D4000696E6700537461747573206465666665C7
:100D50007265640A002D3E005075623A20002D3EF7
:100D6000005075623A20002D3E005075623A200016
:100D70000000000000636D6400007365740000767D
:100D8000616C000064656C000048535600005247D7
:100D900042000066616E00006D6F646500637472EE
:100DA0006C006875650000736174000074656D7097
:100DB0000072617700002D3E005075623A20002DD0
:100DC0003E005075623A2000556E6B6E6F776E2054
:100DD000636D64200A000000000000000000004F66
:100DE0004E000000000000004F46460000000000DA
:100DF00000524553540000000000544F47474C45F3
:100E000000000048414C540000000000584F4E00C4
:100E10000000000000584F46460000000000494E08
:100E200043524541534500444543524541534500D3
:100E3000454E41424C4500000044495341424C4517
:100E40000000554E465245455A4500465245455AC2
:100E5000450000004155544F000000000046414E3F
:100E60005F4F4E4C59004849474800000000004D74
:100E7000454449554D0000004C4F5700000000000C
:100E800000484541540000000000434F4F4C000013
:100E900000000044525900000000000053544F501D
:100EA00000000000005247420000000000004853CC
:100EB00056000000000000206661696C65643A001D
:100EC0004D6F64627573206F7020004D423A206F41
:100ED0006B003D004D423A205643230020636D6471
:100EE0003D003D004D423A2056435F6865617423E2
:100EF000004D423A204E6F7420737570706F72749B
:100F000065642072656720747970650A00205661F7
:100F10006C3A30780020543A00205265673A3078B5
:100F2000004D423A20416464723A00444D5800003A
:100F300000000000444D58524742570000444D58AD
:100F400052474200000050574D0000000000004D85
:100F500042555344494D0000544845524D4F0000FE
:100F60000052454C41590000000047524F55500077
:100F7000000000564354454D500000004D4255536B
:100F80005643000000414348414945520000535038
:100F9000494C45440000004D4F544F5200000000A2
:100FA0005049440000000000004D4255530000002D
:100FB000000055415254425244470052454C415959
:100FC00050574D00444D5852474257570056454ED2
:100FD000545300000000454C455641544F520043C5
:100FE0004F554E544552000048554D00000000003A
:100FF000004D455243555259000020002D3E0043FC
:101000006F6E76657274696E6720002D3E005772B0
:101010006F6E672041737369676E6D656E74200033
:10102000524742783A200020764C6576656C3A004B
:1010300020436F6E76563A0020436F6E76533A0027
:1010400020486F743A00436F6C643A0020436F6E1F
:1010500076657274656420563A00436F6E766572E9
:1010600074656420533A002D3E0057726F6E6720FE
:1010700041737369676E6D656E7420002D3E005775
:10108000726F6E672041737369676E6D656E742051
:101090000053617665643A00000000000000000023
:1010A000004F4E000000000000004F4646000000C8
:1010B000000000524553540000000000544F4747C1
:1010C0004C4500000048414C540000000000584FBF
:1010D0004E000000000000584F464600000000008F
:1010E000494E4352454153450044454352454153BF
:1010F0004500454E41424C450000004449534142A1
:101100004C450000554E465245455A45004652450D
:10111000455A450000004155544F0000000000466C
:10112000414E5F4F4E4C590048494748000000006F
:10113000004D454449554D0000004C4F57000000FC
:10114000000000484541540000000000434F4F4C50
:1011500000000000004452590000000000005354F9
:101160004F50000000000052474200000000000005
:1011700048535600000000000020537566663A0090
:101180002041543A00206973200044656C657469FD
:101190006E6720636F6E662E2052414D207761731B
:1011A0003A0053746F70706564006E6F7468696E96
:1011B0006720746F2073746F700053746F70706960
:1011C0006E67206368616E6E656C73202E2E2E0034
:1011D0004E6F7420756E6C6F636B656420696E2052
:1011E000313073202D20636F6E74696E7565202E0B
:1011F0002E2E00556E6C6F636B696E6720636F6E89
:10120000666967202E2E2E00436F6D706C657465C5
:101210002E2052656D6F766520746F7069632000B3
:1012200024636F6D6D616E6400536B697070696EDD
:10123000672E2E00436C65616E5570207265746177
:10124000696E656420746F7069632000220022005B
:101250004F75744F664D656D6F727921005D20008A
:101260003A5B000A005D00456D7074793A205B00BE
:101270000A003A004D41433A0055445020537973D7
:101280006C6F6720696E697469616C697A65642E38
:101290000A005379736C6F6720706172616D733AE5
:1012A000002E6C6F63616C00536572766963652014
:1012B0007265636F72643A20006D444E532072650C
:1012C00073706F6E64657220737461727465642EDE
:1012D000004572726F722073657474696E67207551
:1012E00070204D444E5320726573706F6E6465724A
:1012F0002100476F742049502061646472657373E4
:101300003A00276970205B69705B2C646E735B2CFC
:1013100067775B2C7375626E65745D5D5D5D27201C
:101320002D20736574207374617469632049500AB9
:10133000004661696C656420746F20636F6E666936
:10134000677572652045746865726E657420757383
:10135000696E6720444843502E20596F75206361A1
:101360006E20736574206970206D616E75616C6CA0
:10137000792100204D41534B3A002047573A002035
:10138000444E533A004C6F616465642066726F6D21
:1013900020666C6173682049503A000A7573657362
:1013A00020444843500A005374617274696E672088
:1013B0006C616E00546F6F206D616E79204D5154D9
:1013C0005420636F6E6E656374696F6E2065727210
:1013D0006F72732E2052657374617274204C414E8B
:1013E000002074727920616761696E20696E203512
:1013F000207365636F6E6473006661696C65642C4D
:101400002072633D004177616974696E6720666F81
:10141000722072657461696E656420746F706963AF
:101420007300636F6E6E6563746564206173200082
:10143000202E2E2E0020757365723A003A000A4164
:101440007474656D7074696E67204D5154542063D7
:101450006F6E6E656374696F6E20746F20006469CF
:1014600073636F6E6E6563746564005573696E6750
:10147000204D5154542070617373776F72642066ED
:10148000726F6D20636F6E666967002E6C6F6361AB
:101490006C006D444E53206E616D65207570646103
:1014A0007465643A2000446576696365204E616D19
:1014B000653A004174206C656173742064657669D7
:1014C0006365206E616D6520616E642062726F6B72
:1014D0006572204950206D75737420626520636FBA
:1014E0006E6669677572656400757074696D652CE8
:1014F00066726565686561700035323335626236E3
:101500005F323032332D31312D3137004C6967680D
:10151000744875622000246E616D650052656269D1
:101520006E6420737563636573732E204950206168
:101530006464726573733A004572726F723A207216
:101540006562696E64206661696C0052656E6577DC
:10155000656420737563636573732E204950206141
:101560006464726573733A004572726F723A2072E6
:10157000656E65776564206661696C000A4E6F2050
:101580006C696E6B0033307320454550524F4D20CF
:101590006973206E6F742072656C6F616465642E70
:1015A000205265626F6F7400416363657074696E89
:1015B0006720636F6D6D616E64732E2E2E0A004E70
:1015C0006F204D51545420636F6E66696775726564
:1015D00064004C6F6164696E6720636F6E66696753
:1015E0002066726F6D20706F7274616C2064697315
:1015F00061626C65642E2075736520676574204F89
:101600004E20746F20656E61626C6500436F6E667C
:1016100069672069732076616C696400436F6E743A
:10162000696E756520776974682070726576696F78
:1016300075736C79206C6F6164656420636F6E668E
:1016400069670043757272656E74204C414E206369
:101650006F6E6669672869702C646E732C67772CCF
:101660007375626E6574293A000A55736520746853
:1016700065736520636F6D6D616E64733A202768D2
:10168000656C7027202D20746869732074657874E8
:101690000A276D61632064653A61643A62653A6560
:1016A000663A66653A3030272073657420616E644F
:1016B0002073746F7265204D41432D6164647265BF
:1016C000737320696E20454550524F4D0A2769704B
:1016D000205B69705B2C646E735B2C67775B2C738B
:1016E00075626E65745D5D5D5D27202D2073657488
:1016F000207374617469632049500A2773617665A9
:1017000027202D20736176652063757272656E7473
:1017100020636F6E66696720696E204E5652414D98
:101720003B204F4E7C4F4646202D20656E61626CFB
:10173000652F64697361626C65206175746F736194
:1017400076650A2767657427205B636F6E66696735
:1017500020616464725D27202D2067657420636FAB
:101760006E6669672066726F6D207072652D636F9B
:101770006E666967757265642055524C20616E64AF
:101780002073746F726520616464722C204F4E7CEC
:101790004F4646202D20656E61626C652F6469732B
:1017A00061626C6520646F776E6C6F6164206F6E30
:1017B00020737461727475700A276C6F61642720DE
:1017C0002D206C6F616420636F6E6669672066729E
:1017D0006F6D204E5652414D0A2770776427202D99
:1017E00020646566696E6520616E642073746F7233
:1017F00065204D5154542070617373776F72640A81
:10180000276F746170776427202D20646566696E88
:101810006520616E642073746F7265204854545063
:10182000204150492070617373776F72640A276C8E
:101830006F67205B73657269616C5F6C6F676C6565
:1018400076656C5D205B7564705F6C6F676C657648
:10185000656C5D27202D20646566696E65206C6F60
:1018600067206C6576656C2028302E2E37290A2774
:101870006B696C6C27202D207465737420776174FC
:101880006368646F670A27636C65617227202D2087
:10189000636C65617220454550524F4D0A27736550
:1018A0006172636827202D2073656172636820313F
:1018B0002D77697265206465760A277265626F6F9D
:1018C0007427202D207265626F6F7420636F6E74B1
:1018D000726F6C6C657200536F6674207265626F14
:1018E0006F74696E672E2E2E00206E65770020695A
:1018F0007320003157543A003157543A20536561F0
:10190000726368696E67206465760052414D3D00E0
:101910000A5379736C6F6720000A312D77697265FD
:1019200020000A6D71747420000A6D6F6462757313
:10193000207632000A6D6F6462757320763120283C
:101940002B29000A696E7075747320000A6974652A
:101950006D7320000A436F6E666967757265643A3D
:10196000003157543A207365747570207265736F37
:101970006C7574696F6E20003157543A20445332AD
:101980003438322D313030206E6F742070726573B0
:10199000656E74003157543A204453323438322D36
:1019A0003130302049324320726573746F72656440
:1019B000003157543A204275732072657365742064
:1019C0006572726F72003157543A2042757320521B
:1019D0006573657420646F6E65003157543A204416
:1019E00053323438322D3130302070726573656E69
:1019F000742C207265736574004572726F722031A9
:101A00002D7720696E6974003157543A204453325F
:101A10003438325F3130305F4932435F544F5F3189
:101A2000575F42524944474520696E697400444DEE
:101A3000584F75742E20467265653A00444D5869BA
:101A40006E2042756666657220616C6C6F632065FE
:101A5000727200496E697420696E2063683A003BB7
:101A6000003D0050696E3A003B003D4C4F5700541A
:101A70006865726D6F3A004F6E65207769726520F8
:101A800052656164790A00467265653A00444D58B2
:101A9000206F757420737461727465642E204368BE
:101AA000616E6E656C733A2000444D5820696E205B
:101AB000737461727465642E204368616E6E656C28
:101AC000733A004170706C79696E6720636F6E665F
:101AD000696700436F6E666967206175746F736133
:101AE00076653A000A5379736C6F67206465627596
:101AF00067206C6576656C3A0053657269616C208D
:101B00006465627567206C6576656C3A0053617632
:101B100065640A005365742064796E616D696320A1
:101B200049500A00454550524F4D20636C65617223
:101B300065640A004D5154542050617373776F727D
:101B40006420757064617465640A004F54412050CC
:101B5000617373776F726420757064617465640A71
:101B600000636F756C64206E6F74207061727365B2
:101B70003A2000557064617465640A004E6F204914
:101B800050206164726573730052656C656173699E
:101B90006E6720736F636B657420616E642072657D
:101BA00074727900205361766564004C6F616469DA
:101BB0006E67204854545020636F6E666967206FCB
:101BC0006E20737461727475703A0000000000003A
:101BD000000000004F4E000000000000004F46468D
:101BE0000000000000005245535400000000005463
:101BF0004F47474C4500000048414C54000000004E
:101C000000584F4E000000000000584F46460000AC
:101C1000000000494E43524541534500444543525C
:101C20004541534500454E41424C45000000444962
:101C30005341424C450000554E465245455A4500D9
:101C4000465245455A450000004155544F0000009A
:101C5000000046414E5F4F4E4C59004849474800EE
:101C6000000000004D454449554D0000004C4F57C1
:101C700000000000000048454154000000000043FF
:101C80004F4F4C000000000044525900000000007B
:101C90000053544F50000000000052474200000023
:101CA0000000004853560000000000002B002D00EB
:101CB000455461673A200047657420455441473ACE
:101CC0002000485454502F312E310025733A2025DE
:101CD000730D0A0020485454502F312E310D0A48FC
:101CE0006F73743A2025730D0A4163636570743A0B
:101CF000202A2F2A0D0A436F6E6E656374696F6E1A
:101D00003A20636C6F73650D0A0025730020000D87
:101D10000A00474554006661696C656420746F2051
:101D2000636F6E6E6563740A004552524F523A20DB
:101D30005365727665722072657475726E65642083
:101D400000436F6E666967206E6F74206368616E12
:101D50006765640A00446F6E652E0A00436F6E6605
:101D600069672070617273696E67206661696C656E
:101D7000640A00676F7420436F6E6669670A0068C3
:101D800074747020726574636F6465200066726598
:101D9000652000436F6E666967205552493A206896
:101DA0007474703A2F2F002044656661756C74203E
:101DB000636F6E66696720736572766572207573EE
:101DC00065643A20006C617A79686F6D652E727572
:101DD000000A282B294D554C544956454E54000AAB
:101DE000282B2950574D5F52454C4159000A282B4A
:101DF000294D444E53000A282D2955415254425230
:101E000049444745000A282B295359534C4F470052
:101E10000A282B29504944000A282D294D435032C5
:101E200033303137000A282D294152544E45540091
:101E30000A282D294F5441000A282D2953504920A2
:101E40004C4544000A282B294D4F544F52204354EF
:101E500052000A282D294143204841494552000A91
:101E6000282D29434353383131202620484443311B
:101E7000303830000A282B29524553544152545FC0
:101E80004C414E5F4F4E5F4D5154545F4552524F3F
:101E90005253000A282D2948415244524553455473
:101EA0002C207573696E6720736F6674000A282B87
:101EB00029434F554E544552000A282B2944485473
:101EC000000A282B294453323438322D3130300067
:101ED0000A282B294F57495245000A282D294950D5
:101EE0004D4F44425553000A282B294D4F4442552B
:101EF0005320307830362061742053657269616CEC
:101F0000322073706565643A39363030000A282B08
:101F1000294144414652554954204C4544000A2821
:101F20002B29444D58000A282B2957697A4E65748D
:101F300035353030000A282B294672656552616DAF
:101F4000207072696E74696E67000A282B295741E8
:101F5000544348444F47006C617A79686F6D652E31
:101F60007275000A436F6E666967207365727665E5
:101F7000723A003230313130334C0020432B2B2069
:101F800076657273696F6E3A003532333562623648
:101F90005F323032332D31312D3137000A4C617AC6
:101FA00079686F6D652E7275204C69676874487525
:101FB0006220636F6E74726F6C6C65722000204FCC
:101FC000464600204F4E0020425950415353007264
:101FD0006561647900247374617465007570746957
:101FE0006D65006672656568656170002473746173
:101FF0007473002054696D65723A00204C6F636BF6
:10200000733A002000204C6F636B733A000A524110
:102010004D3D0020457870697265640A00202D747A
:102020006172676574207A6F6E652D0020416C6166
:10203000726D20457870697265640A0020636D6472
:102040003A00204375723A00205365743A00536198
:1020500076656420746F20454550524F4D005361A2
:1020600076696E6720636F6E66696720746F2045BE
:102070004550524F4D2E2E004C6F616465642045D3
:102080005441473A004E6F2073746F726564206349
:102090006F6E666967004C6F616465642066726F7D
:1020A0006D20454550524F4D006C6F616420666154
:1020B000696C6564004A534F4E20646574656374AF
:1020C0006564004C6F6164696E6720436F6E66697A
:1020D000672066726F6D20454550524F4D00556E1A
:1020E0006B6E6F776E207375666669782000556E2B
:1020F0006B6E6F776E20636D642000436F756E7436
:1021000065723A2000444D582D4F757420496E6910
:10211000743A2000444D582D4F75742073746F70BD
:102120003A200041737369676E65643A00444D5804
:10213000206374726C3A20006931360001693332D1
:1021400000027531360003753332000469386800C7
:102150000569386C0006753868000775386C00082A
:102160007831300009313030000A44656661756CA1
:10217000742073657269616C206D6F6465204E38E0
:1021800031207573656400384531002600384E31C2
:10219000000600384532002E00384E32000E00385E
:1021A0004F31003600384F32003E003745310024B1
:1021B00000374532002C00374F31003400374F32A2
:1021C000003C00374E31000400374E32000C004D09
:1021D0004255533A204D6F646275732074656D707B
:1021E0006C617465206E6F7420666F756E643A2042
:1021F000004D4255533A20496E76616C69642074F3
:10220000656D706C6174652E002C002C002C002C08
:10221000004D4255533A20636F6E666967206661D0
:10222000696C65643A004D4255533A20636F6E669F
:102230006967206572726F72004D4255533A206390
:102240006F6E666967206C6F6164656420004D4243
:1022500055533A204F7574206F66206D656D6F720F
:1022600079004D4255533A20506F6C6C696E67206F
:102270006572726F7220004D425553443A2049678F
:102280006E6F726564202D20657175616C207769B1
:102290007468207365747465642076616C004D42C7
:1022A00055533A204164642040533A20004D425532
:1022B00053443A204D61707065643A004D42555365
:1022C000443A204E65737465644D61707065643A7C
:1022D000004C6173744B6E6F776E2076616C756520
:1022E0003A2000536561726368696E6720726567A2
:1022F0003A200072656723206F7574206F66207224
:10230000616E676500536561726368696E6720720C
:10231000656723003A002066726F6D2074797065DE
:1023200020004D425553443A2020676F742000200E
:1023300076616C3A0020005265733A200020696E85
:102340007465726E616C2073656E64206572726F65
:1023500072202D206E6F207265672F636F696C008D
:1023600020696E7465726E616C2073656E642065A1
:1023700072726F72202D206E6F2074656D706C61AB
:1023800074650020696E7465726E616C2073656E91
:1023900064206572726F72202D206E6F2073746FCF
:1023A0007265004D425553443A20656E64506F6C1F
:1023B0006C20004D425553443A20506F6C6C200005
:1023C000206E6F7420666F756E64004D4255533AEF
:1023D0002020706172616D20002073656E6420653D
:1023E00072726F722E20004D4255533A20200041E8
:1023F00064642040563A20002056616C3A20004D1B
:10240000425553443A207375666669783A00206FE6
:10241000722073756666697820004D4255533A20E4
:102420004E6F2074656D706C61746520666F7220EC
:10243000004D6F746F723A2074696D656F7574002A
:10244000556E6B6E6F776E20636D64004D6F746FA9
:10245000723A20466F7263656420657865637574AF
:10246000696F6E004D756C746956656E7420636F8C
:102470006E666967206661696C6564004D756C7491
:102480006956656E7420696E6974004D756C746967
:1024900076656E742044652D496E697400204F7511
:1024A000743A00206D33002066726F6D2000204D5D
:1024B000617820726571756573743A002066616E8B
:1024C000253A002061637469766520563A00546F9E
:1024D00074616C20563A005049443A20616C726530
:1024E00061647920696E697469616C697A656400F8
:1024F0005049443A20496E76616C6964207061727B
:10250000616D2061727261792E002C002C002C000C
:102510002C005049443A20636F6E666967206661FB
:10252000696C65643A005049443A20636F6E66698D
:1025300067206572726F72005049443A20636F6E73
:10254000666967206C6F6164656420005049443A95
:10255000204F7574206F66206D656D6F7279005025
:1025600049443A2044652D496E69742000203C415D
:102570004C4D3E0020443A0020493A0020503A0099
:1025800020696E3A00207365743A005049443A203D
:10259000005049443A20496E76616C69642070614C
:1025A00072616D2061727261792E00536574206FC3
:1025B000757420746F20002050494420616C617252
:1025C0006D2E20002050494420616C61726D3A20CC
:1025D000636C6F736564005049443A20556E6B6EAE
:1025E0006F776E2073756666697820005049443AAB
:1025F00020556E6B6E6F776E20636D6420002053E4
:102600006574706F696E743A005049443A20002036
:10261000496E7075742076616C75653A0050494456
:102620003A200020696E697400200050574D2D4FEC
:1026300075742023002073746F7000200050574D74
:102640002D4F75742023003D0050696E3A002069BB
:102650006E69740052656C61792D4F75742023008A
:102660002073746F700052656C61792D4F75742002
:1026700023003D3E003A0070756220616374696F0B
:102680006E200069646C65006F6666006865617441
:10269000696E670066616E00647279696E670063D7
:1026A0006F6F6C696E670020697320004F7574202E
:1026B00000556E6B6E6F776E207375666669782055
:1026C00000556E6B6E6F776E20636D6420006163E2
:1026D00074696F6E0072656C61794374723A2000A0
:1026E0002072656164206572726F7220666F72205D
:1026F000003E2000203C003157543A003157543AF4
:10270000206E6F7420696E6974003157543A20420C
:102710005553592074696D656F7574003157543A7B
:10272000204453323438325F4552524F525F434F48
:102730004E464947003157543A20312D776972652A
:102740002073686F72746564005B305D3A2000200E
:102750002D202D202D20EFBBBF003E003E31202D2F
:10276000200000002100240027002A002D00300056
:10277000330001010000040107010A0100002200EA
:10278000250028002B002E0031003400020100003B
:10279000050108010B0105050505070508080808DE
:1027A000020202020A0A08080404040401010101E9
:1027B00001010101030303030303030304070707E4
:1027C0000C0C0C0C0C0C0C0C020202020606060689
:1027D000060606060B0B0B0B0B0B0B0B0102102056
:1027E0002008081020401020408002010201080447
:1027F00002010102040810204080804020100804DB
:102800000201800402018040201008040201080433
:102810000201010204081020408001020408102077
:10282000408000000A0B02090C0D0E08070304018A
:102830000000000000000000000000000000000098
:102840000000000000000000000000000000121165
:102850001000000000000000000000000000000068
:10286000000000000000000057726F6E672070616A
:10287000796C6164004354524C2F7478743A204F41
:1028800075744F664D656D6F72793A2000202D3E4C
:102890002041543A004368616E20747970653A00B3
:1028A0004E6F2073746F7265642076616C7565730A
:1028B000202D2064656661756C743A200053617642
:1028C000656420455441473A00536574204554419E
:1028D000473A20000000000000636D64000073654B
:1028E00074000076616C000064656C00004853560B
:1028F0000000524742000066616E00006D6F646523
:10290000006374726C006875650000736174000088
:1029100074656D7000726177000020002E00696E92
:1029200000735F6F7574006D79686F6D6500435457
:10293000524C2F657865633A204F75744F664D652C
:102940006D6F72793A2000202D3E2000456D69742C
:102950003A203C00202D3E20004974656D436D6493
:102960003A2000202D3E20004974656D3A20003148
:1029700057543A20427573207265736574206572EE
:10298000726F72003157543A20427573205265734A
:10299000657420646F6E65003157543A2044533299
:1029A0003438322070726573656E742C20726573D2
:1029B00065740049324320526573657400005EBC43
:1029C000E2613FDD83C29C7E20A3FD1F419DC321A8
:1029D0007FFCA2401E5F01E3BD3E6082DC237D9F41
:1029E000C1421CFEA0E1BF5D0380DE3C62BEE0028E
:1029F0005CDF81633D7C22C09E1D43A1FF4618FA27
:102A0000A427799BC584DA3866E5BB5907DB85675F
:102A100039BAE406581947A5FB7826C49A653BD90C
:102A200087045AB8E6A7F91B45C6987A24F8A64445
:102A30001A99C7257B3A6486D85B05E7B98CD230F2
:102A40006EEDB3510F4E10F2AC2F7193CD114FAD0F
:102A5000F3702ECC92D38D6F31B2EC0E50AFF113D8
:102A60004DCE90722C6D33D18F0C52B0EE326C8EF5
:102A7000D0530DEFB1F0AE4C1291CF2D73CA9476B6
:102A800028ABF517490856B4EA6937D58B5709EBD7
:102A9000B536688AD495CB2977F4AA4816E9B75594
:102AA0000B88D6346A2B7597C94A14F6A8742AC8BD
:102AB00096154BA9F7B6E80A54D7896B353E3E20E8
:102AC00000496E76616C696420636F6D6D616E6440
:102AD00000000020002300260029002C002F0032D7
:102AE00000000100000301060109013E3E3E004EC8
:102AF0006F204D414320636F6E6669677572656430
:102B00003A20736574206669726D77617265277308
:102B1000204D41430A00454550524F4D207369678F
:102B20006E6174757265206F6B00496E69746961BE
:102B30006C697A696E6720454550524F4D2E0000F2
:102B40000B01E70311241FBECFEFD1E2DEBFCDBFE3
:102B500000E00CBF18E0A0E0B2E0EAE5F5E502E035
:102B60000BBF02C007900D92A63CB107D9F72FE02A
:102B7000A6ECB8E001C01D92AE38B207E1F715E14E
:102B8000C1EAD5E100E006C021970109802FFE01CE
:102B90000F947122C03AD10780E00807A9F70F947B
:102BA00047160D949B2A0C940000FC0184819581AA
:102BB0000895FC01A481B581109721F118969C918C
:102BC00018979F708EEF890F823010F091111AC004
:102BD00019964D935D936D937C931C97A481B58159
:102BE00018969C911897907F926018969C930480F9
:102BF000F581E02D8085982F907F903619F48F70A5
:102C0000806A80870895FC01238130E090E080E0B5
:102C1000FC01EE0FFF1FEE5FF64FA081B181A217FE
:102C2000B30761F4880F991F880F991FFC01E251C7
:102C3000F74F40835183628373830895A081B181EC
:102C4000AB2B19F420813181EDCF019685309105B0
:102C5000F9F60895FC01238130E090E080E0FC016A
:102C6000EE0FFF1FEE5FF64F408151814217530771
:102C700061F4880F991F880F991FFC01E251F74FEB
:102C80006081718182819381089540815181452BBA
:102C900089F431832083880F991F880F991FFC01C5
:102CA000E251F74F108211821282138260E070E0CD
:102CB000CB01089501968530910589F6F7CF880FED
:102CC000991F880F991FFC01EA52F74F808191816B
:102CD000A281B3810196A11DB11D80839183A2833E
:102CE000B383089585E090E00C945F1684E090E053
:102CF0000C945F1683E090E00C945F1682E090E005
:102D00000C945F1681E090E00C945F1690E080E0F8
:102D10000C945F16CF93DF93EC01E881F981048472
:102D2000F585E02D199529893A892F5F3F4F3A8B18
:102D3000298BDF91CF910895CF93DF93EC018E859E
:102D400081110DC081E090E049895A892C853D852B
:102D50004217530708F080E0DF91CF910895E88192
:102D6000F9810484F585E02DCE0119958F3F9105F9
:102D700049F780E090E0F0CFFC01848595856817E5
:102D8000790708F4CB01928B818B0895DC011E96A4
:102D90002C911E97222339F0ED91FC910190F08146
:102DA000E02D6FEF19940895FC01878590890895AF
:102DB00081E0089590E080E00895DC011296ED91A5
:102DC000FC91309761F00190F081E02D309739F05F
:102DD000862F8295807F60856F70682B608708954D
:102DE000DC011296ED91FC91309751F00190F08149
:102DF000E02D309729F0808582958F7090E00895BE
:102E000090E080E008950F931F93CF93DF9300D05D
:102E100000D01F921F92CDB7DEB781E028960FB683
:102E2000F894DEBF0FBECDBFDF91CF911F910F9100
:102E3000089590E080E0089560EB7BE0811102C08E
:102E40006BEA7BE083E59DE00C94BAF2DC015596D9
:102E50002C915597273781F4ED91FC91008CF18DE1
:102E6000E02D199567E578E083E59DE00E94BAF2D0
:102E700083E59DE00C9404F10895009789F0FC012E
:102E800020852F70253061F40E9428C1009741F001
:102E9000FC0120852F70243019F4818592850895D6
:102EA00090E080E0089565E0FC01808191810E94BE
:102EB00028C1009749F0FC018085982F907F21F070
:102EC00082958F7090E0089590E080E00895EF92F1
:102ED000FF920F931F93CF93DF930097C1F0FC01F4
:102EE00020812223A1F08C0185E7E82E8DE0F82EC9
:102EF000C1E0D0E0B701C8010F94BB1A892B49F09B
:102F00002196F5E0EF0EF11CCE30D10599F7D0E017
:102F1000C0E0CE01DF91CF911F910F91FF90EF9014
:102F20000895CF92DF92EF92FF920F931F93CF936A
:102F3000DF93CDB7DEB7C154D1090FB6F894DEBF29
:102F40000FBECDBF6C01AB0130E020E060E4CE01EC
:102F500001967C010F94910DF70101900020E9F793
:102F600031978F010E191F09A801B701C6010F94EF
:102F7000FE26892B11F010E000E0C801CF5BDF4F87
:102F80000FB6F894DEBF0FBECDBFDF91CF911F917A
:102F90000F91FF90EF90DF90CF900895CF92DF9246
:102FA000EF92FF920F931F93CF93DF93CDB7DEB7CE
:102FB000C054D1090FB6F894DEBF0FBECDBF8091CB
:102FC000820E9091830E059709F449C06115710531
:102FD00009F445C069017A018B0140E450E0CE015B
:102FE00001960F940C276FE270E0CE0101960F94CA
:102FF000D326892B41F4980143E050E060E4CE01F0
:1030000001960F94910D4FE350E0B601CE01019669
:103010000F94EE260E94CEC0882309F18091820E83
:103020009091830E0697D9F48091690E811117C093
:10303000B701CE0101960E94F4D181E090E0C05C1E
:10304000DF4F0FB6F894DEBF0FBECDBFDF91CF913B
:103050001F910F91FF90EF90DF90CF90089590E037
:1030600080E0EDCFCF92DF92EF92FF920F931F930C
:10307000CF93DF93CDB7DEB760970FB6F894DEBF7E
:103080000FBECDBF7C016B01CA01B9012AE0AE01C0
:103090004F5F5F4F0F945F1BD701ED91FC9102884A
:1030A000F389E02D9801AE014F5F5F4FB601C70174
:1030B000199560960FB6F894DEBF0FBECDBFDF91B5
:1030C000CF911F910F91FF90EF90DF90CF900895D7
:1030D000CF92DF92EF92FF920F931F93CF93DF93E4
:1030E000CDB7DEB760970FB6F894DEBF0FBECDBF89
:1030F0007C016B01BA01A901CE0101960F94810EEA
:10310000D701ED91FC910288F389E02D9801AE0181
:103110004F5F5F4FB601C701199560960FB6F894DF
:10312000DEBF0FBECDBFDF91CF911F910F91FF90FA
:10313000EF90DF90CF9008951F93CF93DF93FC0122
:10314000162FC389D489818992899C012F5F3F4FB3
:10315000328B218BC80FD91FCE010F94D4211817A1
:1031600021F0612FCE010F94DC2181E090E0DF910E
:10317000CF911F910895FC0181899289248535851D
:103180008217930740F423893489820F931F0F9489
:10319000D42190E008958FEF9FEF08958F929F9232
:1031A000AF92BF92CF92DF92EF92FF920F931F9355
:1031B000CF93DF93E091840EF091850E309709F460
:1031C00067C0812EF02E932EC22EA52ED42EB72EA0
:1031D000E62EBC01CF010E94B0C0EC01892B19F48E
:1031E00081E090E057C088858F708530C9F760E036
:1031F000CE010E9428C18C0161E0CE010E9428C14D
:10320000FC01C185D285D80119962D913C912130C0
:10321000310561F13CF46F2DCE01232B09F70F949A
:103220007607DECF2230310531F127303105C1F686
:10323000892BB1F280858F70853091F6C681D78158
:10324000209771F288858F70843061F40F2D182DCE
:103250002C2D392D4D2D5A2D6E2D7B2D89859A853E
:103260000E94CE180A80DB81C02DEACF6F2DCE01DF
:1032700003960F9476076E2DCE010F9476076D2D71
:10328000CE0101960F9476076C2DCE010296C7CF22
:1032900090E080E0DF91CF911F910F91FF90EF9030
:1032A000DF90CF90BF90AF909F908F900895CF9276
:1032B000DF92EF92FF920F931F93CF93DF93E091F2
:1032C0001709F09118093097C9F090859F709530D3
:1032D000A9F469017A01EB01682FCF010E9428C18E
:1032E000FC0190859F70943049F481859285009708
:1032F00029F09601A701BE010E94CE18DF91CF915F
:103300001F910F91FF90EF90DF90CF9008958F92D3
:103310009F92AF92BF92CF92DF92EF92FF920F9364
:103320001F93CF93DF938091150990911609892BF4
:1033300009F48BC021E030E0D0E0C0E0CC24C3949D
:10334000D12C46010C2E02C0880C991C0A94E2F77D
:10335000092C000CAA08BB08790184E0E80EF11CD6
:10336000C90150E040E060911C0270911D02FC0117
:103370006817790720F4E0911C02F0911D0260911A
:103380007C0E70917D0EE60FF71FA081E09115096C
:10339000F0911609BC0161507109E60FF71F6081B9
:1033A0006A17F1F06091CB087091CC086330710519
:1033B000B4F04091D1085091D2086091D308709137
:1033C000D408482959296A297B294093D108509368
:1033D000D2086093D3087093D408A08351E041E0F1
:1033E0000196E816F90609F0BECF4423D9F1809181
:1033F000CB089091CC0801969093CC088093CB0891
:103400005523E9F0E0911509F0911609E20FF31F39
:10341000028110E0218130E0408150E031976081ED
:1034200070E0CE010E94571980E00F94730D6093F5
:10343000CD087093CE088093CF089093D008219642
:103440009701C430D10509F07CCFDF91CF911F9156
:103450000F91FF90EF90DF90CF90BF90AF909F9033
:103460008F9008951092CC081092CB08C9CFCF92BC
:10347000DF92EF92FF920F931F93CF93DF9300D0D1
:1034800000D0CDB7DEB7809126098111A4C080910C
:10349000820E9091830E02970CF49DC080911F09BB
:1034A00090912009009709F496C064EF74E00E949F
:1034B000B0C08C01009709F48EC00E94BAC1E82EFA
:1034C000F12CE114F10409F486C070E060E0C80159
:1034D0000E943D176C01EA94EF2809F48BC061E06B
:1034E000C8010E9428C1FC010185128585EC94E089
:1034F0009A8389831B821C821D821E82CE010396C1
:103500000F946D06CE0101960E9418CB62E972E11C
:1035100082EA9CE00E94BAF2B60182EA9CE00E9434
:1035200054F267E477E082EA9CE00E9454F24AE0B9
:1035300050E0B80182EA9CE00E940BF267E477E079
:1035400082EA9CE00E9454F260EA79E082EA9CE020
:103550000E9454F282EA9CE00E9404F162E072E070
:1035600081E79DE00E9452FFD092670DC092660DE8
:103570001093690D0093680D80EA99E0892BE9F5B5
:1035800082EF94E090936B0D80936A0D80911909FE
:1035900090911A09009741F070E060E00E943D1799
:1035A0009093660E8093650E8091650E9091660EE5
:1035B000009731F190936D0D80936C0D10926F0D0B
:1035C00010926E0D81E08093260969E772E182EA2C
:1035D0009CE00E94BAF226960FB6F894DEBF0FBEAA
:1035E000CDBFDF91CF911F910F91FF90EF90DF90B2
:1035F000CF90089502E012E079CF80EA99E0C2CF3F
:103600008BEC93E0D7CFCF93DF9300D000D01F9205
:103610001F92CDB7DEB7FC01862F8F706181607F6E
:10362000682B618388E0DE01119601900D928A95E6
:10363000E1F729813A814B815C816D817E818F81A7
:10364000988528960FB6F894DEBF0FBECDBFDF91E8
:10365000CF910895CF93DF9300D000D01F921F9297
:10366000CDB7DEB7FC01608398E0DE0111960190D2
:103670000D929A95E1F729813A814B815C816D81A8
:103680007E818F81988528960FB6F894DEBF0FBE95
:10369000CDBFDF91CF9108956F927F928F929F92CD
:1036A000AF92BF92CF92DF92EF92FF920F931F9350
:1036B000CF93DF93CDB7DEB7A0970FB6F894DEBFF8
:1036C0000FBECDBF8C01862E7A01DC018D919C91BD
:1036D0001197892B09F466C01496ED91FC913097EF
:1036E00009F460C080818071BFEF6B135DC0B1F4DD
:1036F00081E0A0960FB6F894DEBF0FBECDBFDF917C
:10370000CF911F910F91FF90EF90DF90CF90BF90DE
:10371000AF909F908F907F906F90089543305105A8
:1037200039F3818082942FE0822267EF78E083E58D
:103730009DE00E94BAF24AE050E0D80113966C91E5
:1037400083E59DE00E9421F165EF78E083E59DE04F
:103750000E94BAF2D8011496ED91FC9161816F70CC
:103760004AE050E083E59DE00E9421F162EF78E0BD
:1037700083E59DE00E94BAF24AE050E0682D83E5BF
:103780009DE00E9421F183E59DE00E9404F1D801B3
:103790001496ED91FC9181818F70881207C0808111
:1037A0008F7E808380E0A5CF8111FCCF198E1A8E89
:1037B0001B8E1C8E1D8E1E8E1F8E18A28A8D8F70E2
:1037C0008A8FD8011496ED91FC9181818F708815B4
:1037D000A9F1B3E0EB16F10489F160EF78E083E53D
:1037E0009DE00E94BAF24AE050E0F801638183E56F
:1037F0009DE00E9421F16EEE78E083E59DE00E945D
:10380000BAF2D8011496ED91FC9161816F704AE093
:1038100050E083E59DE00E9421F16BEE78E083E5C6
:103820009DE00E94BAF24AE050E0682D83E59DE0F9
:103830000E9421F183E59DE00E9404F1F8012081BE
:103840003181FCE0F81508F416C1E82DF0E0882776
:10385000E35DF34E8F4F0D9471223A1C771CF81CD8
:103860000F1D1B1DF81CD11CF81C1E1D291DE51C5D
:103870002C1D381DD8011496CD90DC90F601818165
:103880008F70853009F4F7C050F48230C1F069E0E0
:1038900075E0C9010E94B0C03C01912C4BC087303B
:1038A000D1F08A30A1F762E075E0C9010E94B0C092
:1038B0003C01D6019C9092FA992490F83BC06CEFA1
:1038C00074E0C9010E94B0C03C01D6019C9090FAFE
:1038D000992490F82FC06BEF74E0C9010E94B0C02A
:1038E0003C01F601908091FA992490F823C06EE093
:1038F00075E0C9010E94B0C03C01D8011496ED9159
:10390000FC91808180FB992490F8982F9E7F80FF06
:10391000916090836114710469F461E0CE0149966D
:103920000E942A1B298B3A8B4B8B5C8B6D8B7E8B79
:103930008F8B988FF801A080B18064E475E0C50199
:103940000E94B0C06C0169E475E0C5010E94B0C07E
:103950005C01892B81F4C114D10469F460E0CE01CB
:1039600049960E942A1B29833A834B835C836D838B
:103970007E838F839887D8011496ED91FC91611412
:10398000710409F07CC0898D811179C0B82DBF7098
:103990008B2E8181807F882A818280818F7E8083A7
:1039A000A7CE63E175E0C9010E94B0C03C01D80117
:1039B0001496ED91FC91808181FB992490F8982FC9
:1039C0009D7F81FF92609083B5CF69E175E0C90169
:1039D0000E94B0C03C01D8011496ED91FC91808109
:1039E00082FB992490F8982F9B7F82FF9460EBCF05
:1039F00069E075E0C9010E94B0C03C01892B09F063
:103A00004CCF62E0CE0149960E942A1B29873A8753
:103A10004B875C876D877E878F87988B3ECF6FE162
:103A200075E0C9010E94B0C03C01D8011496ED9127
:103A3000FC9190804CCF64E275E0F3CF6AE275E0D0
:103A4000C9010E94B0C03C01D8011496ED91FC91CF
:103A500049CF60E375E0F4CF67E375E0C9010E94E8
:103A6000B0C03C01D8011496ED91FC91908023CF19
:103A70006DE375E0F3CF912C712C612C5BCF83E06B
:103A8000E816F104B9F0982D9F70892E8181807F0E
:103A9000882A818280818F7E8083E98CFA8C0B8DCD
:103AA0001C8D2D8D3E8D4F8D58A1692DC3010F9416
:103AB00096101ECE81818F70881509F419CE8294DC
:103AC00090EF8922882A81828081806168CFCF939C
:103AD000DF9300D000D01F921F92CDB7DEB7FC015C
:103AE00091819F70906B9183448355836683778324
:103AF00088E0DE01119601900D928A95E1F7298107
:103B00003A814B815C816D817E818F819885289679
:103B10000FB6F894DEBF0FBECDBFDF91CF910895F1
:103B2000CF93DF9300D000D01F921F92CDB7DEB7A6
:103B3000FC016F3F710519F014F06FEF70E077FD35
:103B400060E09181892F82958F7081508230C8F416
:103B5000648388E0DE01119601900D928A95E1F769
:103B600029813A814B815C816D817E818F8198852D
:103B700028960FB6F894DEBF0FBECDBFDF91CF9170
:103B800008959F7090619183E3CFCF93DF93CDB77A
:103B9000DEB760970FB6F894DEBF0FBECDBF1982B7
:103BA0001A821B821C821D821E821F8218868A81B5
:103BB0008F708A836FEF70E0CE0101960E94901D96
:103BC00060960FB6F894DEBF0FBECDBFDF91CF91E8
:103BD0000895CF92DF92EF92FF92DC01362F11967B
:103BE000EC911197E295EF70EC3008F0B6C0F0E080
:103BF0008827E250F24E8F4F0D947122B01E361E70
:103C0000361EAD1EAD1EAD1E7B1E3D1EAD1EAD1E75
:103C10000A1E0A1E14968D919D910D90BC91A02DA7
:103C2000662399F0B7FD9FC08F3F9105A105B105AF
:103C300029F024F08FEF90E0A0E0B0E02FEF30E02B
:103C4000A901481B590BCA010CC0B7FD89C08F3FA1
:103C50009105A105B10529F024F08FEF90E0A0E0D7
:103C6000B0E0FF90EF90DF90CF90089514962C91E4
:103C7000822F90E06623A9F3E1CF1496CD90DD90DA
:103C8000ED90FC901797662301F120E030E0A90148
:103C9000C701B6010F94B02087FD65C020E030E079
:103CA0004FE753E4C701B6010F94B82318160CF47C
:103CB00057C0A701960160E070E08FE793E40F948E
:103CC000A3220F948223CB01CCCF20E030E0A901C6
:103CD000C701B6010F94B02087FD42C020E030E05C
:103CE0004FE753E4C701B6010F94B8231816DCF16F
:103CF000C701B601E6CF14966D917D918D919C918F
:103D000017973323B1F06D395FEF75078507950776
:103D100054F1611524E67207810591050CF52CE933
:103D20003FEF4FEF5FEF0F941C22C90181509F4F6F
:103D300098CF6D394FEF7407840794078CF06115A5
:103D400054E675078105910574F424E630E040E0FF
:103D500050E00F941C22C90184CF8FEF9FEF81CFD9
:103D600090E080E07ECF8FEF90E07BCFCF93DF932A
:103D7000EC01DB01898182958F708630E1F128F4B6
:103D800081508230C8F080E014C0873009F18A5039
:103D90008230C8F72FEF30E00F94882224E630E01D
:103DA00040E050E00F941C222C833D834E835F83C0
:103DB00081E0DF91CF9108952FEF30E00F948822BA
:103DC00024E630E040E050E00F941C222C83F0CF3A
:103DD0002FEF30E00F94882224E630E040E050E0FE
:103DE0000F941C22CA01B9010F94B7206C837D8304
:103DF0008E839F83DDCF2CE933E60F94882224E65F
:103E000030E040E050E00F941C222C833D834E8331
:103E10005F83B9CFDC011196EC911197E295EF70B9
:103E2000E150EB3008F039C0F0E08827E55EF04E55
:103E30008F4F0D9471223E1F3E1F4D1F261F261FC0
:103E40002F1F461F461F461F261F261F14966D91C3
:103E50007D918D919C9117970F94B720089514969A
:103E60006D917D918D919C91179724E630E040E013
:103E700050E00F941C22CA01B901EECF14966C9148
:103E800070E090E080E00F94B520089514966D9155
:103E90007D918D919C911797089560E070E0CB0122
:103EA0000895DC011196EC911197E295EF70E150C5
:103EB000EB3008F037C0F0E08827EE59F04E8F4F16
:103EC0000D947122741F741F921F6D1F6D1F831F2D
:103ED0007A1F7A1F7A1F6D1F6D1F14966D917D9149
:103EE0008D919C911797089514966C9170E090E0D5
:103EF00080E0089514966D917D918D919C91179716
:103F00000F948223089514966D917D918D919C91CB
:103F1000179724E630E040E050E00F941C22CA01DD
:103F2000B901089560E070E0CB0108958F929F92EF
:103F3000AF92BF92CF92DF92EF920F931F93CF93E6
:103F4000DF9300D000D01F921F92CDB7DEB7FC01E7
:103F500009831A832B833C834D835E836F83788729
:103F6000808191810097A1F490E080E028960FB6BF
:103F7000F894DEBF0FBECDBFDF91CF911F910F919F
:103F8000EF90DF90CF90BF90AF909F908F9008956B
:103F90008F010E94BAC1C82ED12C86E0C816D10468
:103FA00064F40E943DC7BC01F801808191810E94A8
:103FB000BCC5FFEFCF1ADF0AF0CF65E0F8018081C2
:103FC00091810E9428C18C01892B71F289818031F5
:103FD00058F6CE0101960E94511F161617061806B4
:103FE000190644F4F8018085982F9D70A1F08F7018
:103FF000873089F0F80180858F70808765E479E0EB
:1040000083E59DE00E94BAF283E59DE00E9404F101
:1040100081E090E0ABCF0E9426D14B015C01CE0144
:1040200001960E94511F860E971EA81EB91EF80108
:1040300081869286A386B48682E0E11087E099812A
:104040009295907F892BF80180876AE379E083E578
:104050009DE00E94BAF2CE0101960E94511FAB0171
:10406000BC012AE030E083E59DE00E94C3F164E3F7
:1040700079E083E59DE00E94BAF2F801418552851E
:10408000638574852AE030E083E59DE00E94C3F1FA
:10409000BBCFDC011196EC911197E295EF70E150E6
:1040A000EB3008F03EC0F0E08827E65AFF4D8F4F16
:1040B0000D947122702070209120652065208A2047
:1040C0007B207B207B206520652014962D913D91DF
:1040D0004D915C911797A4E6B0E00F943B220895B0
:1040E00014966C9184E6689FB0011124072E000C91
:1040F000880B990B089520E030E048EC52E41496C8
:104100006D917D918D919C9117970F9416210F942D
:104110008223089514966D917D918D919C911797AE
:10412000089560E070E0CB010895FC01A7812A2F7B
:104130002E7FD1F0818182958F7081508330A0F4E1
:10414000A695A150BB0B2BE531E00F94882224E605
:1041500030E040E050E00F941C22DA01C90187569C
:104160009F4FAF4FBF4F08958FEF9FEF08952F924E
:104170003F924F925F926F927F928F929F92AF92F7
:10418000BF92CF92DF92EF92FF920F93CF93DF9384
:1041900000D01F92CDB7DEB77C017A8369835C8340
:1041A0004B83DB011C92FC016081662309F44EC045
:1041B00030FF4CC0F9E06F9FB001112468567F4E6C
:1041C000CD010F94F21AD70111968C91807F41F0A6
:1041D0004B815C8160E077E089819A810F94EE26C3
:1041E000E981FA8101900020E9F7319729813A812C
:1041F000E21BF30B19012E0E3F1E4B815C814E1BFF
:104200005F0B415051095C834B83D7011196EC91B0
:1042100011978E2F807F09F4F7C0E295EF70E1507F
:10422000EC3008F0F1C0F0E08827E65EFE4D8F4FDD
:104230000D9471222921CC2139229822B322772191
:1042400049224922492265214D21CF2229803A80E5
:10425000DCCFF7018481282F30E050E040E00023DC
:1042600059F030E0A4E6B0E00F944E222FEF30E09A
:1042700040E050E00F941C225F934F933F932F93A5
:104280008EE495E09F938F93FC81FF932B812F9376
:104290003F922F920F942627B2C017968C911797B2
:1042A0008F9316968C9116978F9315968C911597E0
:1042B0008F9314968C918F9381E595E09F938F93C4
:1042C000BC81BF93EB81EF93E3CF17968C91179747
:1042D0008F9316968C9116978F9315968C911597B0
:1042E0008F9314968C918F9385E595E0E7CF149684
:1042F000CD90DD90ED90FC901797F7FE34C084E6EA
:10430000882E912CA12CB12CC701B601A5019401D6
:104310000F941C229B01AC0188279927DC01821B8A
:10432000930BA40BB50BBF93AF939F938F9366270B
:104330007727CB016C197D098E099F09A50194018E
:104340000F941C225F934F933F932F9389E595E041
:104350009F938F933C813F934B814F933F922F923A
:104360000F9426274CC0C701B60124E630E040E098
:1043700050E00F941C229F938F937F936F935F93D2
:104380004F933F932F938AE595E09F938F939C8162
:104390009F93AB81AF93E2CFC7010E949520BC01F0
:1043A000D7011696CC9016971796DC901797D0FAEF
:1043B000DD24D0F814969C9114971596FC90EB8010
:1043C000BC80292F30E050E040E077FD35C001117E
:1043D00035C07F936F931F921F921F929F931F92DE
:1043E000FF92DF92CF9283E695E09F938F93FC81BB
:1043F000FF932B812F933F922F920F9426270FB676
:10440000F894DEBF0FBECDBF89819A810F900F90C7
:104410000F900F90DF91CF910F91FF90EF90DF9071
:10442000CF90BF90AF909F908F907F906F905F9054
:104430004F903F902F900895002361F0292F30E096
:10444000A4E6B0E00F944E222FEF30E040E050E0C1
:104450000F941C225F934F933F932F931F92FF92D1
:10446000DF92CF9286E695E09F938F93BF92EF9273
:1044700075CF15968C9115971F928F9316969C91D8
:10448000169717968C9181708F939F9389E695E08C
:1044900015CF14968D909D90AD90BC90179720E00D
:1044A00030E0A901C501B4010F94B0202401350109
:1044B00087FF04C077FA709477F87094C301B20153
:1044C0000F9482236B01072E000C880B990B0F941D
:1044D000B7209B01AC01C301B2010F94A32220E0DD
:1044E00030E04AE754E40F9416210F940D240F9402
:1044F0008223062F772E20E030E0A901C501B40108
:104500000F94B02087FF07C07F920F93DF92CF9266
:104510008FE695E0D3CE7F920F93DF92CF9280E724
:1045200095E09F938F933C813F934B814F93B0CE07
:1045300014968C9114971F928F9315968C911597C2
:104540001F928F9316968C911F928F9386E695E01B
:104550009F938F93BC81BF93EB81EF933F922F92F8
:104560000F9426274CCF17968C9117971F928F93F5
:1045700014968C9114971F928F9315968C91159782
:104580001F928F9316968C911F928F9383E695E0DE
:104590009F938F93BC81BF93EB81EF93DFCE1496F3
:1045A0006D917C914B815C81C1010F940C272CCFC4
:1045B000EF92FF920F93CF93DF93CDB7DEB7A09723
:1045C0000FB6F894DEBF0FBECDBF7C0100E020E047
:1045D00033E040E250E0BE016F5F7F4F0E94B720A2
:1045E000BE016F5F7F4F83E59DE00E9454F260E85B
:1045F00071E183E59DE00E94BAF2F7016181629565
:104600006F704AE050E083E59DE00E9421F169E788
:1046100071E183E59DE00E94BAF2F70161816F705C
:104620004AE050E083E59DE00E9421F183E59DE0B2
:104630000E9404F1A0960FB6F894DEBF0FBECDBF66
:10464000DF91CF910F91FF90EF900895CF93DF937B
:10465000EC016115710539F48F8181708F8381E0E0
:10466000DF91CF9108958981982F92959F7029F1BC
:1046700080E09430A8F79B01770F440B550B295924
:10468000310941095109A4E6B0E00F943B222BE522
:1046900031E040E050E00F941C2237FF02C030E0D0
:1046A00020E02536310514F024E630E02F5F220F9C
:1046B0008F818170282B2F83D2CF8F708062898366
:1046C000DACF2F923F924F925F926F927F928F92AA
:1046D0009F92AF92BF92CF92DF92EF92FF920F9391
:1046E0001F93CF93DF93CDB7DEB768970FB6F894DB
:1046F000DEBF0FBECDBF1C0109871A872B873C8701
:104700004D875E876F87788B22E1E216F10408F00F
:1047100035C0F701EA5FFB4F3081398BCE01099636
:104720000E94952097FD04C0BC01C1010E94262370
:104730009A85892F8F70D1011196EC911197E07FA6
:10474000E82B1196EC93119789858C93E295EF7085
:10475000EC3008F063C0F0E08827EE54FC4D8F4F3A
:104760000D947122B525DB23DB235325C023E125DE
:104770001C255D255D255D251C251C25198ACECFB0
:10478000B12C92959F709D3008F0C9C4E92FF0E0DC
:104790008827E253FC4D8F4F0D9471220E241B2667
:1047A0003B261B26E425E4251B261B268F288F2865
:1047B0001B261B26E82492959F709D3008F018C197
:1047C000E92FF0E08827E851FC4D8F4F0D947122BE
:1047D0000E24C624B9247C24F823F5239D24C82460
:1047E000F824F82487248724E8248889F101878322
:1047F0008F85D10116968C9316978E8515968C937E
:1048000015978D8514968C9314979295907F119699
:104810008C9111978F70982B11969C93B989BB231B
:1048200009F467C0F101818182958F702B2F30E0F0
:104830008217130609F45DC06FEF7FE083E59DE00A
:104840000E94BAF2D10111966C9162956F704AE0A4
:1048500050E083E59DE00E9421F16CEF7FE083E56D
:104860009DE00E94BAF24AE050E0698983E59DE04C
:104870000E9421F16AEF7FE083E59DE00E94BAF299
:10488000F101008119821A821B821C821D821E8204
:104890001F82188689898295807F9A819F70892BD3
:1048A0008A830983EE24EA94FE2C118122813381CC
:1048B0004481558166817781CE0101960E946123F2
:1048C000D1012C9311963C93119712964C93129709
:1048D00013965C93139714966C93149715967C9388
:1048E000159716968C93169717969C93C1010E9464
:1048F000D82288E0F10178C18F859889F1018683FB
:10490000878190FB80F987838E85858387CF8D850E
:104910009E85AF85B889B7FD0EC08F3F9105A10573
:10492000B10529F024F08FEF90E0A0E0B0E0D101D4
:1049300014968C9373CF80E0FACF6D857E858F853A
:10494000988920E06D39BFEF7B078B079B076CF0E0
:104950002FEF6115E4E67E078105910534F424E626
:1049600030E040E050E00F941C22D10114962C93CB
:1049700055CF8F859889F1018683878190FB80F9D7
:1049800087838E8585838D85848348CF8D85CFCF22
:10499000CD84DE84EF84F88820E030E0A901C701EF
:1049A000B6010F94B02060E087FD0FC020E030E03A
:1049B0004FE753E4C701B6010F94B8236FEF181601
:1049C00024F0C701B6010F948923F101648326CF37
:1049D000D10111968C9111978F70806C11968C93E8
:1049E00011978D859E8515969C938E93149716CF5F
:1049F0006FE770E183E59DE00E94BAF26A856295F7
:104A00006F704AE050E083E59DE00E9421F16CE781
:104A100070E183E59DE00E94BAF2F1016181629547
:104A20006F704AE050E083E59DE00E9421F183E54C
:104A30009DE00E9404F1F2CE92959F70933091F028
:104A40009C3031F24D855E856F857889F101448314
:104A50005583668377839295907F81818F70982BA1
:104A60009183DCCE60E0C1010E94E91DD101149662
:104A70008C9314978F85988916968C931697179612
:104A80008C91179790FB80F917968C9317978E85CA
:104A900015968C93159711968C9111978F70806253
:104AA00011968C93BBCE60E0CE0109960E94E91D61
:104AB000D10114968C931497EECF92959F709D30F0
:104AC00008F066C0E92FF0E08827E659FA4D8F4FCD
:104AD0000D9471220E248525B4253225B425B425E4
:104AE0007725A425A425A42593259F25E8248D8535
:104AF0009E85AF85B889F10184839583A683B783AA
:104B000081818F708066818389CE6D8570E090E0B1
:104B100080E00F94B520D10114966D937D938D9311
:104B20009C9317977BCE6D857E858F8598890F9492
:104B3000B720F10164837583868397836FCE6D857B
:104B40007E858F859889E5CF9295907FF10181814F
:104B50008F70982B91838D859E85AF85B8898483CE
:104B60009583A683B7835ACE9295907FD1011196F3
:104B70008C9111978F70982B11969C938D859E85A3
:104B8000AF85B889F10184839583A683B78346CE28
:104B90006AE670E183E59DE00E94BAF26A8562955B
:104BA0006F704AE050E083E59DE00E9421F167E6E6
:104BB00070E183E59DE00E94BAF2D10111966C91FB
:104BC0002ECFBB24B394DDCD4D855E856F8578896E
:104BD000F10144835583668377839295907F818129
:104BE0008F70982B918388E0DE01119601900D92D1
:104BF0008A95E1F729813A814B815C816D817E81C3
:104C00008F81988568960FB6F894DEBF0FBECDBF32
:104C1000DF91CF911F910F91FF90EF90DF90CF9098
:104C2000BF90AF909F908F907F906F905F904F90CC
:104C30003F902F900895963009F43EC148F46D8559
:104C4000913071F06FEF70E0933051F060E008C088
:104C5000973009F43DC19A506D857E859230B0F74A
:104C600084E68F8788898E7F888B1E868A858F70E1
:104C700080628A876D872E8530E0AFEFB0E00F94B9
:104C80004E22C12CD12C7601CA946115F4E67F071F
:104C90008105910544F424E630E040E050E00F94B3
:104CA0001C2269017A0186012D852A8B622E712CC6
:104CB000BB2009F475C088898695A82FA150BB0B2D
:104CC0002D01BFEF4B165B0609F023C1003811051B
:104CD0000CF005C18FE790E08C199D09869DD001ED
:104CE000879DB00D969DB00D11242FEF30E00F94ED
:104CF000882221E83EE740E050E00F941C22F101B9
:104D00002783ABE9B0E0A70196010F943B22EFE7C0
:104D10008E2E912CA12CB12CA50194010F941C2254
:104D200089019A010C591F4F2F4F3F4FAEEFB1E051
:104D3000A70196010F943B22A50194010F941C2218
:104D4000D3010F943B222FEF30E040E050E00F946E
:104D50001C2239012FEF6216710421F01CF0662429
:104D60006A94712C6AE570E183E59DE00E94BAF2D5
:104D70004AE050E0B80183E59DE00E940BF26CE44C
:104D800070E183E59DE00E94BAF24AE050E0B30191
:104D900083E59DE00E940BF283E59DE00E9404F113
:104DA000E6E9F7E2E491F0E0EE0FFF1FE458F84D7A
:104DB00085919491ECEDF7E2E4912F85388931707B
:104DC000AFEFBFEF0F944E222DE631E040E050E010
:104DD0000F941C2244275527AAEFB5E00F943B22DD
:104DE000DC01CB019058AF4FBF4FCD01BB2797FDE2
:104DF000B095AB2F8E3FE1E09E0708F069C1382FD8
:104E00008F3F910508F486C14EEF481B50E03FEFFD
:104E10007301FFEFEF1AFF0AF801FF2731960095A3
:104E200010E03E9FC0013F9F900D1124292F332792
:104E3000200F311FD7010F9488224B015C01882479
:104E4000AA24BB245E9F90015F9F300D1124232F65
:104E50003327200F311F0F948822BB27A92F982FAB
:104E6000872F882A992AAA2A4E9F90014F9F300D9A
:104E70001124232F3327200F311FD7010F948822AD
:104E8000B82FA72F962F882788279927BB278829EF
:104E90009929AA29F101A6839583848360E270E1B0
:104EA00083E59DE00E94BAF2C1010E94D82260E031
:104EB00080E00E94ABCEB2CC6D857E858F859889CF
:104EC00024E630E040E050E00F941C22B901C8CE47
:104ED0006D857E858F8598890F948223C1CEA70129
:104EE00096012058310941095109ABE9B0E00F940E
:104EF0003B222FE730E040E050E00F941C22890174
:104F00009A010C591F4F2F4F3F4FD10117961C92FA
:104F100029CF9201AAEBBFEF0F94802244E6842EA2
:104F2000912CA12CB12CA50194010F941C22DA0123
:104F3000C9018C599F4FAF4FBF4F8B8B9C8BAD8B53
:104F4000BE8B26E430E0D2010F948822A5019401A3
:104F50000F941C2249015A019EE1890E911CA11C4B
:104F6000B11C003811050CF099C08FE790E08C1946
:104F70009D09869DD001879DB00D969DB00D112491
:104F8000A50194010F9446229B01AC01AFEFB0E064
:104F90000F943B2224E63AE640E050E00F941C22B6
:104FA000D10117962C932B893C894D895E892C0D54
:104FB0003D1D4E1D5F1DAEEFB1E00F943B2223EE71
:104FC00030E040E050E00F941C2229013A01388F74
:104FD0002F8BAFEFB0E0A70196010F943B222FE794
:104FE00030E040E050E00F941C228901EA89AE2FA6
:104FF000B0E0A30192010F943B222FEF30E040E09C
:1050000050E00F941C2239012F3F310521F01CF094
:1050100066246A94712C66E470E183E59DE00E9449
:10502000BAF22AE030E04B895C896D897E8983E59C
:105030009DE00E94C3F160E470E183E59DE00E9481
:10504000BAF22AE030E0B501A40183E59DE00E94B8
:10505000C3F168E370E183E59DE00E94BAF24AE0A3
:1050600050E0B80183E59DE00E940BF260E370E13F
:1050700083E59DE00E94BAF24AE050E0B30183E587
:105080009DE00E940BF267E270E183E59DE00E94E3
:10509000BAF24AE050E06F89788D7ACEA701960186
:1050A0002058310941095109ABE9B0E00F943B2286
:1050B0002FE730E040E050E00F941C2289019A0174
:1050C0000C591F4F2F4F3F4FD10117961C92A3CF62
:1050D0008C3FF3E09F0768F48D3F22E0920728F4AD
:1050E00052E0580F3FEF40E093CE3CEF381B5FEFAC
:1050F000FACF8A3F35E0930781F08B3FE4E09E07CB
:1051000028F444E0480F5FEF30E082CE5AEF581B9E
:1051100030E001C050E04FEF7BCE50E0F9CF6EE0C1
:1051200070E183E59DE00E94BAF26A8562956F7036
:105130004AE050E083E59DE00E9421F16BE070E1E0
:1051400038CDFC019181892F82958F7021F08230BA
:1051500029F080E008959F70906291839B0177FF12
:1051600002C030E020E02E3681E0380714F02DE652
:1051700031E02683878130FB80F9878381E00895C1
:10518000EF92FF920F931F93CF93DF93FC01892B34
:1051900069F19081992351F19D3291F180ED890F50
:1051A0008A3070F1C8E0D0E0953211F1CEEFDFEF38
:1051B0009B37F1F0C7E1D0E09332D1F08F0181EA63
:1051C000E82E80E1F82EC1E0D0E0C7010F94CB1AA1
:1051D000AC01B701C8010F94E41A892B49F021965C
:1051E00089E0E80EF11CC931D10579F7CFEFDFEF87
:1051F000CE01DF91CF911F910F91FF90EF90089515
:10520000D0E0C0E0F5CFEF92FF920F931F93CF93C2
:10521000DF93EC01892B51F188858F70843009F57B
:10522000E984FA84C7010E94C0288C011816190667
:10523000ECF4C7010E9431F6C801012E000CAA0B44
:10524000BB0B89879A87AB87BC878885807F826004
:105250008887C801DF91CF911F910F91FF90EF9048
:105260000895823019F409851A85F3CF10E000E023
:10527000F0CF2F923F924F925F926F927F928F92D8
:105280009F92AF92BF92CF92DF92EF92FF920F93D5
:105290001F93CF93DF93CDB7DEB76C970FB6F8941B
:1052A000DEBF0FBECDBF6115710549F528E0FC01D9
:1052B000DE01119601900D922A95E1F729813A813C
:1052C0004B815C816D817E818F8198856C960FB654
:1052D000F894DEBF0FBECDBFDF91CF911F910F912C
:1052E000FF90EF90DF90CF90BF90AF909F908F9006
:1052F0007F906F905F904F903F902F9008956B013B
:105300008C0164EB78E0C6010E94B0C0FC01892BDF
:1053100009F40EC180858F70843009F452C0853045
:1053200009F006C1E680F780E114F10409F400C138
:10533000F70180858F70823011F4E280F380E114F0
:10534000F10409F4F5C0F70180858F70853011F004
:10535000F701F3CFC7010E94BAC18230C9F760E0FC
:10536000C7010E9428C15C010E94032961E0C701B6
:105370000E9428C14C01FC0180858F70823041F76A
:10538000C8010E94511FF4014184528463847484D3
:105390006415750586059705D9F6A114B10409F4BD
:1053A000C7C019821A821B821C821D821E821F8224
:1053B00018868A818F708A83F5016185CE010196F6
:1053C0004EC068E775E0818592850F94DE26892BB3
:1053D00009F0AEC0C8010E94511F61157105810519
:1053E000910509F48BC0660F771F881F991F2FEF57
:1053F00030E040E050E00F941C2257FD15C02330F0
:105400003105410551050CF05FC0DA01C901019673
:10541000A11DB11D82309105A105B105D9F10397F8
:10542000A105B10509F450C019821A821B821C82A1
:105430001D821E821F8218868A818F708A8367E090
:10544000CE0101960E94031B29873A874B875C8710
:105450006D877E878F87988B62E1CE0109960E94C7
:105460002A1B298B3A8B4B8B5C8B6D8B7E8B8F8BA6
:10547000988F49895A896B897C898D899E89AF89E2
:10548000B88D49835A836B837C838D839E83AF83DE
:10549000B88714CF19821A821B821C821D821E8239
:1054A0001F8218868A818F708A8367E0CE010196F9
:1054B0000E94031B29873A874B875C876D877E870D
:1054C0008F87988B61E1C9CF19821A821B821C8257
:1054D0001D821E821F8218868A818F708A8367E0F0
:1054E000CE0101960E94031B29873A874B875C8770
:1054F0006D877E878F87988B60E1AFCF19821A8284
:105500001B821C821D821E821F8218868A818F70D8
:105510008A8367E0CE0101960E94031B29873A87A0
:105520004B875C876D877E878F87988B62E095CFEE
:105530006CE775E0C6010E94B0C05C01009709F4F9
:10554000C5C0FC0180858F70853009F0AEC0C501F3
:105550000E94BAC1843009F0B9C060E0C5010E9460
:1055600028C14C0161E0C5010E9428C13C0162E0F4
:10557000C5010E9428C1FC01C184D284E384F48463
:1055800063E0C5010E9428C15C01C8010E94511F4F
:105590006C157D058E059F059CF419821A821B826D
:1055A0001C821D821E821F8218868A818F708A83C8
:1055B00040E050E0BA01CE0101960E94671D51CF34
:1055C000F4010184F285E02DFA8FE98FF301218443
:1055D0003284F5010184F285E02DFC8FEB8F198276
:1055E0001A821B821C821D821E821F8218868A815B
:1055F0008F708A83298D3A8D4901330FAA08BB0821
:1056000026010D2C000C66087708C8010E94511F66
:105610009B01AC012419350946095709B101032C36
:10562000000C880B990B681979098A099B090F945A
:10563000EA21EB8DFC8D9F01FF0F440B550B2419C4
:105640003509460957090F941C22820E931EA41E89
:10565000B51EC101298D3A8D821B930B6B8D7C8DFC
:105660006C197D090F945D2277FF02C06F5F7F4F39
:1056700075956795CB01770FAA0BBB0B880E991E0A
:10568000AA1EBB1EB7FC0CC0A401B5013FEF8316D8
:105690009104A104B10409F00CF48DCF4FEF01C0C7
:1056A00040E050E060E070E086CF81110FC01982C9
:1056B0001A821B821C828A818F708A8349815A8157
:1056C0006B817C8180E090E0DC01DBCEF8014081E1
:1056D00051816281738184819581A681B781D1CE08
:1056E0004F925F926F927F928F929F92AF92BF92F2
:1056F000CF92DF92EF92FF920F931F93CF93DF939E
:10570000CDB7DEB760970FB6F894DEBF0FBECDBF42
:105710006115710539F528E0FC01DE011196019053
:105720000D922A95E1F729813A814B815C816D8147
:105730007E818F81988560960FB6F894DEBF0FBE8C
:10574000CDBFDF91CF911F910F91FF90EF90DF9030
:10575000CF90BF90AF909F908F907F906F905F9011
:105760004F9008956B018C0164EB78E0C6010E94B4
:10577000B0C05C01F801F080FF2009F44EC0009732
:1057800009F44BC0FC0180858F70843009F4BFC0E0
:10579000853009F042C060E875E083E59DE00E9435
:1057A00054F283E59DE00E9404F1F501E680F78064
:1057B000E114F10491F1F70180858F705701823077
:1057C00061F0B12CA12CE114F10409F41DC1F70121
:1057D00080858F70853021F0F701E280F380F3CF70
:1057E000C7010E94BAC18230B9F760E0C7010E94C8
:1057F00028C10E9403294C0161E0C7010E9428C111
:10580000F80120812815190439F7FC0120852F7033
:10581000223011F7009709F001C16CE775E0C6016D
:105820000E94B0C07C01F8018181807F09F407C12A
:10583000E114F10409F47DC0F70180858F70853093
:1058400009F001C1C7010E94BAC1843009F0FBC050
:10585000C8010E94511F4B015C0160E0C7010E941A
:1058600028C1FC0181859285A385B48519821A829D
:105870001B821C821D821E821F8218868816990632
:10588000AA06BB060CF499C08A818F708A8363E0F4
:10589000C7010E9428C15C0162E0C7010E9428C1C3
:1058A000FC01418452846384748461E0C7010E94D6
:1058B00028C14C0160E0C7010E9428C1FC01C184DD
:1058C000D284E384F484C8010E94511FF50121852C
:1058D00032854385548524193509460957096C19C1
:1058E0007D098E099F090F94EA21F40121853285F3
:1058F000438554852C193D094E095F090F941C22DC
:10590000BA01A901440D551D661D771D31C068E718
:1059100075E0818592850F94DE26892B09F07DCF75
:10592000F0E1FF1609F460C0FF1568F082E0F81698
:10593000E1F1F80140815181628173818481958117
:10594000A681B78129C0E1E1FE16F1F1F2E1FF1273
:10595000F0CF19821A821B821C821D821E821F8236
:1059600018868A818F708A8344E150E060E070E09D
:10597000CE0101960E94671D29873A874B875C8775
:105980006D877E878F87988B49855A856B857C8547
:105990008D859E85AF85B88949835A836B837C83C7
:1059A0008D839E83AF83B887BECE19821A821B82F5
:1059B0001C821D821E821F8218868A818F708A83B4
:1059C00040E050E0BA01D4CF19821A821B821C82B7
:1059D0001D821E821F8218868A818F708A8340E80A
:1059E00050E060E070E0C4CF19821A821B821C82F2
:1059F0001D821E821F8218868A818F708A834FEFD4
:105A000050E060E070E0B4CFA114B10409F405CF18
:105A1000F50180858F7009F400CFC50119821A82C3
:105A20001B821C821D821E821F8218862A812F7073
:105A30002A83FC01418552856385748599CFE114E1
:105A4000F10409F476CFF70180858F7009F071CFEA
:105A500019821A821B821C828A818F708A834981F3
:105A60005A816B817C8180E090E0DC0195CF0F93BF
:105A70001F93CF93DF938C01FC01C081D1816FE232
:105A800070E0CE010F941B270097E9F0FC01119202
:105A9000CF010E946717EC0169E079E083E59DE0A2
:105AA0000E94BAF24AE050E0BE0183E59DE00E9408
:105AB0000BF283E59DE00E9404F1CE01DF91CF91CE
:105AC0001F910F910895CE010E946717EC01892B59
:105AD000A1F3F80111821082F0CFDC01ED91FC916D
:105AE000309729F090859F7081E0953009F080E033
:105AF0000895EF92FF920F931F93CF93DF93EC01E2
:105B00007B018E819F81892BA9F4888199810E94D4
:105B1000BAC1082F10E00530110564F40E943DC79A
:105B20009F838E83BC01888199810E94BCC50F5FD1
:105B30001F4FF1CFEE81FF813097D9F08085982FEC
:105B40009F70A9F4807F82608087EE81FF8111863B
:105B5000128613861486EE81FF81F782E682C701E2
:105B6000DF91CF911F910F91FF90EF9008959230A8
:105B700061F3F12CE12CF3CFCF92DF92EF92FF9201
:105B80000F931F93CF93DF93EC016A017B018E810A
:105B90009F81892BA9F4888199810E94BAC1082F1D
:105BA00010E00530110564F40E943DC79F838E8389
:105BB000BC01888199810E94BCC50F5F1F4FF1CF46
:105BC000EE81FF81309781F08085982F9F7051F48E
:105BD000807F82608087EE81FF81C186D286E386E6
:105BE000F48602C09230B9F3DF91CF911F910F91EB
:105BF000FF90EF90DF90CF900895FC018681978110
:105C0000009799F0FC0120852F70223029F46185DE
:105C10007285838594850895253039F460E00E946B
:105C200028C1009711F0FC01F2CF60E070E0CB01D9
:105C300008950F931F93CF93DF93FC01C281D3810B
:105C40002097C9F18B0188858F70853021F5CE01B1
:105C50000E94BAC18017110671F16CF1602FCE015C
:105C60000E9428C1FC01892B31F180858F70823020
:105C700039F461857285838594850F94B72006C0B9
:105C80008330C9F46185728583859485DF91CF91D6
:105C90001F910F910895672B71F4823029F4698563
:105CA0007A858B859C85E9CF833029F469857A854F
:105CB0008B859C85EBCF60E070E0CB01E7CF0F9345
:105CC0001F93CF93DF93FC01C281D3812097F9F01A
:105CD00088858F70823049F4672BC9F489859A854D
:105CE000DF91CF911F910F910895853081F48B0141
:105CF000CE010E94BAC18017110649F044F0602F0E
:105D0000CE010E9428C1FC0181859285E9CF90E0F7
:105D100080E0E6CF0F931F93CF93DF93EC018B01CD
:105D20007B836A8381E892E09983888370E060E0F6
:105D3000C8010E945F2E97FD19C09D838C83D801F6
:105D40001296ED91FC913097C1F090859F70923042
:105D500089F0953091F4CF010E94BAC190E09F8301
:105D60008E83DF91CF911F910F9108959195819529
:105D70009109E3CF81E090E0F2CF90E080E0EFCFB7
:105D80008F929F92AF92BF92CF92DF92EF92FF924B
:105D90000F931F93CF93DF93EC01888199810E9429
:105DA000BAC1082F10E00430110554F40E943DC719
:105DB000BC01888199810E94BCC50F5F1F4FF3CF42
:105DC00060E0888199810E9428C17C01009769F177
:105DD000DC0118968C9118978F70843041F51996D4
:105DE000CD90DC90C114D10401F1F60180818823AB
:105DF000E1F08BE2882E8FE0982EB12CA12C1A2D89
:105E0000C4010F94CB1AAC01B401C6010F94E41A7B
:105E1000892B09F42FC1FFEFAF1ABF0A89E0880E62
:105E2000911CA7E1AA16B10451F71FEF04C08230FC
:105E3000E1F7F70111851887E880F98061E0C70173
:105E40000E9428C16C019B838A8362E0C7010E9483
:105E500028C19D838C8364E0C7010E9428C17C0116
:105E60009F838E83153108F031C0E12FF0E0882741
:105E7000E35CF04D8F4F0D947122732F732F732FAE
:105E8000522F662F662F662F662F662F662F662F7E
:105E9000662F812FB02F932F662FBD2F732F1130B8
:105EA000662F2C308AE090E00F9482188C01BE019E
:105EB0000E948A2E83E293E0D80111969C938E93E0
:105EC00019961C921E9218971A870987DF91CF9115
:105ED0001F910F91FF90EF90DF90CF90BF90AF9008
:105EE0009F908F90089588E090E00F9482188C0125
:105EF000BE010E948A2E8FEF92E0F8019183808389
:105F0000E3CF8EE090E00F9482188C01DC011396B1
:105F1000DC93CE9312978DEA93E08D939C93C80106
:105F20000E94BCA3D1CF86E090E00F948218FC01C0
:105F3000D383C2838DED92E091838083E114F104D9
:105F4000C9F0D70118968C9118978F70823091F410
:105F500016968D919C9195838483FA87E987B6CFB5
:105F600086E090E00F948218FC01D383C2838BEB10
:105F700092E0E2CF90E080E0EECF8BE090E00F94F3
:105F800082188C01FC01D383C2838BE893E0918358
:105F90008083168270E060E0CE010E945F2E97FD44
:105FA0002DC0D80115969C938E931497D801149602
:105FB0008D919C91009719F0863491052CF080E228
:105FC00090E0F8019583848361E070E0CE010E9447
:105FD000192E20E030E04AE754E40F9416210F9484
:105FE0008923611571058105910589F0D8011796FE
:105FF0006D937D938D939C931A9766CF9195819520
:106000009109F8019583848381E08683CFCF88E866
:1060100093E1A0E0B0E0F80187839087A187B28781
:1060200053CF86E090E00F948218FC01D383C283A3
:1060300089E693E09183808315821482C114D10490
:1060400009F48BCFD60118968C918F70863009F0A9
:1060500084CFD582C48281CF84E090E00F948218EF
:10606000FC01D383C28327E433E0318320839A8702
:1060700089872CCFC6010E9431F68A2D90E0B0E0CE
:10608000A0E0F70181879287A387B4878085807F0E
:1060900082608087D0CECF92DF92EF92FF926A012A
:1060A0007B0163E0FC01808191810E9428C1FC0199
:1060B000892BA9F080858D7091F4C094D094E094E0
:1060C000F094CC24CA9481859285A385B4858C21D3
:1060D0009D21AE21BF2181879287A387B487FF903E
:1060E000EF90DF90CF900895CF92DF92EF92FF92E2
:1060F0006A017B0163E0FC01808191810E9428C1DB
:10610000FC01892BA9F09085892F8D7089F4907FEF
:1061100092609087CC24FF244185528563857485E5
:106120004C295D296E297F294187528763877487AF
:10613000FF90EF90DF90CF900895CF92DF92EF9293
:10614000FF926A017B0163E0FC01808191810E94E2
:1061500028C1009791F0FC0120852F70223069F44E
:1061600061857285838594856C217D218E219F2197
:10617000FF90EF90DF90CF90089560E070E0CB014A
:10618000F7CFAF92BF92CF92DF92EF92FF920F9331
:106190001F93CF93DF93CDB7DEB7CD56D1090FB69E
:1061A000F894DEBF0FBECDBF5C01A7960FAFA797D7
:1061B000A8961FAFA897A9962FAFA997AA963FAF09
:1061C000AA97AB964FAFAB97AC965FAFAC97AD9637
:1061D0006FAFAD97AE967FAFAE9723961FAE1EAE54
:1061E0002397FE01ED5BFF4F82E1DF011D928A954F
:1061F000E9F772961192119287E0DF011D928A955C
:10620000E9F7CE018A599F4F0E94D822F0FE2CC098
:10621000A796EFADA797E83108F050C1F0E08827C6
:10622000EB5EFE4C8F4F0D94712264322D315B3248
:106230005E325E325B322D315E325E325E325E3213
:106240005E325E325E322D312D315E325E325E3232
:106250002D312D312D315E3264326FED7DE0CE0176
:106260008B5A9F4F0F94C41A0E94CEC0882309F402
:1062700007C18091690E811103C1C114D10409F0D5
:106280005EC030E020E043E050E060E4CE010196E3
:106290000F94910DD501ED91FC91608171814FE3D7
:1062A00050E0CE0101960F94EE26F1FE10C1A796A4
:1062B0008FADA797823009F40AC1853009F407C170
:1062C000A8968FADA89782958F709FE0980F9F70CA
:1062D000923018F0883009F0FAC001E020E032E096
:1062E00044E150E0BE016F5B7F4FCE018A599F4F62
:1062F0000E94B720BE016F5B7F4FCE0101960E94C6
:10630000F4D162EC7DE083E59DE00E94BAF2BE012B
:106310006F5F7F4F83E59DE00E9454F26FEB7DE05D
:1063200083E59DE00E94BAF2BE016F5B7F4F83E57B
:106330009DE00E9454F283E59DE00E9404F1A8963E
:106340008FADA897807F870100271072882311F0F6
:10635000F1FC04C00115110509F4F5C030E020E09E
:1063600043E050E060E4CE0101960F94910DD50119
:10637000ED91FC91608171814FE350E0CE01019677
:106380000F94EE26C114D10469F06EE875E0CE01D9
:1063900001960F94C8264FE350E0B601CE01019656
:1063A0000F94EE266EE875E0CE0101960F94C82694
:1063B0004FE350E064E87DE00115110511F46AE750
:1063C0007DE0CE0101960F94D41AA8968FADA897C0
:1063D00082958F708450823008F09FC067E1CE01B3
:1063E0008A599F4F0E942A1B6F962FAF6F97A096D6
:1063F0003FAFA097A1964FAFA197A2965FAFA2978C
:10640000A3966FAFA397A4967FAFA497A5968FAFDF
:10641000A597A6969FAFA69700E020E033E044E161
:1064200050E0BE016F5B7F4FCE018A599F4F0E94A3
:10643000B7206AE67DE083E59DE00E94BAF2BE01E6
:106440006F5F7F4F83E59DE00E9454F267E67DE039
:1064500083E59DE00E94BAF2BE016F5B7F4F83E54A
:106460009DE00E9454F283E59DE00E9404F10E94A9
:10647000CEC0882329F08091690E882309F455C085
:10648000A701FF0C660B770BC5010E94743090E0EA
:1064900080E0C359DF4F0FB6F894DEBF0FBECDBF0B
:1064A000DF91CF911F910F91FF90EF90DF90CF90F0
:1064B000BF90AF90089568EE7DE0D1CE68EC7DE0AE
:1064C00083E59DE00E94BAF2E894F0F8CDCEF0FEAC
:1064D00036CF66968FAD6697882309F430CFBE011C
:1064E0006B5A7F4FCE0101960E94F4D169EB7DE09B
:1064F00083E59DE00E94BAF2BE016F5F7F4F83E5A6
:106500009DE00E9454F266EB7DE083E59DE00E94F1
:10651000BAF2BE016B5A7F4F0ACF20E032E0012B66
:1065200011F020E033E000E07ACFBE016F5B7F4FD7
:10653000CE0101960E94F4D140E052E060E070E0AC
:10654000C5010E944B30F0FE90C0A796EFADA79713
:10655000E150E53118F5F0E08827EE54FD4C8F4FFF
:106560000D947122BD33CE32CE32CE32CE32BD3317
:10657000CE32CE32CE32CE32CE32CE32CE32C23326
:10658000BA33CE32CE32CE32C732B433B73361E80B
:106590007EE0CE018B5A9F4F0F94C41A30E020E06A
:1065A00043E050E060E4CE0101960F94910DD501D7
:1065B000ED91FC91608171814FE350E0CE01019635
:1065C0000F94EE26C114D10469F06EE875E0CE0197
:1065D00001960F94C8264FE350E0B601CE01019614
:1065E0000F94EE266EE875E0CE0101960F94C82652
:1065F0004FE350E065E77DE0CE0101960F94D41A99
:1066000061E67DE083E59DE00E94BAF2BE016F5F26
:106610007F4F83E59DE00E9454F26EE57DE083E5C7
:106620009DE00E94BAF2BE016B5A7F4F83E59DE068
:106630000E9454F283E59DE00E9404F10E94CEC0C6
:10664000882309F41DCF8091690E811119CFBE01F5
:106650006B5A7F4FCE0101960E94F4D140E051E089
:1066600060E070E0C5010E944B30F2FE7AC040E06D
:1066700050E061E070E0C5010E949D30672B682BFF
:10668000692B09F482C069E37EE0CE018B5A9F4FEB
:106690000F94C41A30E020E043E050E060E4CE0103
:1066A00001960F94910DD501ED91FC91608171815E
:1066B0004FE350E0CE0101960F94EE26C114D104B1
:1066C00069F06EE875E0CE0101960F94C8264FE39D
:1066D00050E0B601CE0101960F94EE266EE875E00B
:1066E000CE0101960F94C8264FE350E06DE97DE09E
:1066F000CE0101960F94D41A68E57DE083E59DE014
:106700000E94BAF2BE016F5F7F4F83E59DE00E9459
:1067100054F265E57DE083E59DE00E94BAF2BE019A
:106720006B5A7F4F83E59DE00E9454F283E59DE024
:106730000E9404F10E94CEC0882309F4A1CE80916A
:10674000690E81119DCEBE016B5A7F4FCE0101961D
:106750000E94F4D140E054E060E070E0C5010E9486
:106760004B3081E090E095CE6AE87EE012CF63E99D
:106770007EE00FCF6DE57EE00CCFF50180858530A2
:1067800009F00CCF64E57EE004CF40E050E062E029
:1067900070E0C5010E949D30672B682B692B19F0B2
:1067A0006BE47EE072CF60E37EE06FCFAF92BF928A
:1067B000CF92EF920F931F93CF93DF93CDB7DEB7B6
:1067C000C856D1090FB6F894DEBF0FBECDBF5C012D
:1067D000A2960FAFA297A3961FAFA397A4962FAF31
:1067E000A497A5963FAFA597A6964FAFA697A79655
:1067F0005FAFA797A8966FAFA897A9967FAFA99705
:106800009E2D28E0FE01EF59FF4FDE01A75ABF4F32
:1068100001900D922A95E1F7A296EFADA297E15073
:10682000ED3008F0F2C0EC2CF0E08827E55EFB4C80
:106830008F4F0D94712292349B34F9340335EF3429
:106840002834893405350535A434B634DC34C934EC
:10685000992331F0C5010E945317009709F449C0EC
:1068600067E0CE01875A9F4F0E942A1B60E279E0C1
:1068700083E59DE00E94BAF24AE050E06A966FAD6F
:106880006A9783E59DE00E9421F165E179E083E567
:106890009DE00E94BAF2CE01875A9F4F0E94511F7D
:1068A000AB01BC012AE030E083E59DE00E94C3F12A
:1068B00083E59DE00E9404F16A960FAD6A976B969E
:1068C0001FAD6B976C962FAD6C976D963FAD6D9726
:1068D0006E964FAD6E976F965FAD6F97A0966FAD4A
:1068E000A097A1967FADA197C5010E94961F81E058
:1068F00090E0C859DF4F0FB6F894DEBF0FBECDBF92
:10690000DF91CF911F910F91EF90CF90BF90AF90FB
:106910000895911105C0C5010E945317009749F3CE
:1069200066E09FCF992329F0C5010E945317009775
:1069300001F362E096CF911105C0C5010E94531783
:106940000097B9F261E08DCF40E050E061E070E087
:10695000C5010E949D30672B682B692B29F4C50166
:106960000E945317009729F26BE07BCF40E050E084
:1069700061E070E0C5010E949D30672B682B692B98
:1069800031F0C5010E945317009709F4B2CF6AE0B5
:1069900068CF40E050E062E070E0C5010E949D30A9
:1069A000672B682B692B31F0C5010E9453170097A4
:1069B00009F49FCF6CE055CF40E050E062E070E01A
:1069C000C5010E949D30672B682B692B31F4C501EE
:1069D0000E945317009709F48CCF6DE042CF9111BC
:1069E00006C0C5010E945317009709F482CF63E0E7
:1069F00038CF992331F0C5010E945317009709F44D
:106A000078CF65E02ECF64E02CCF90E080E071CFAE
:106A1000CF93C62F63E0FC01808191810E9428C141
:106A2000FC01892B21F19085892F8D7001F5907FD4
:106A30009260908781859285A385B4858827BB273E
:106A40008C2B81879287A387B48761E079E083E507
:106A50009DE00E94BAF24AE050E06C2F83E59DE091
:106A60000E9421F183E59DE0CF910C9404F1CF9138
:106A70000895CF92DF92FF920F931F93CF93DF93EE
:106A8000F12C6115710509F499C06A01EB018C01C3
:106A9000CB010E946D2DF82E882309F48FC0D2FE01
:106AA00009C0D8018C918B3009F44BC0E8F58A30CD
:106AB00009F44CC0D0FE09C0F801608186EF860F52
:106AC000843018F0CE010E940835D1FE6EC0D80186
:106AD00014964D915D916D917C91179711968C91C3
:106AE00082958F70873038F0893008F43EC08A5024
:106AF000823008F46CC0CE010E94D915EC81FD8172
:106B0000309709F452C080858F709EEF980F9230B5
:106B100010F081114AC0D80111969C91907F808518
:106B20008F70892B808741C08C30B9F040E050E0F5
:106B300062E070E08D3009F0BDCFCE010E9474306C
:106B4000B9CF40E050E061E070E0F7CF40E050E0C6
:106B500061E070E0CE010E944B3040E050E062E026
:106B600070E0CE010E944B30A5CFEC81FD813097C3
:106B7000E1F080858F709EEF980F923010F08111B8
:106B800014C04187528763877487EC81FD818085BB
:106B9000807F83608087EC81FD818085982F907F46
:106BA0008F708067903609F4BDCF61E970E183E5AD
:106BB0009DE00E94BAF2C8010E94D8228F2DDF9179
:106BC000CF911F910F91FF90DF90CF900895CE014C
:106BD0000E94D915EACF63E0FC01808191810E9477
:106BE00028C1009719F0FC01818508958FEF089561
:106BF000CF92DF92EF92FF920F931F93CF93DF9389
:106C00006115710509F458C06A017B018C01CB0143
:106C10000E946D2DD82F882371F1D70114968D9184
:106C20009C910097E9F1FC01C0852C2F2F703EEF5D
:106C3000320F323010F0211128C0C295CF70D0FE33
:106C400059C0C7010E94EB35F8018083CC2351F174
:106C5000C295C07F81818F70C82BC183D7011496E4
:106C6000ED91FC9181859285A385B485F80184839B
:106C70009583A683B7838D2FDF91CF911F910F91BD
:106C8000FF90EF90DF90CF900895253049F460E0B9
:106C90000E9428C1009721F0DC011896CC91CDCF3D
:106CA000C0E0CDCFD7011496ED91FC9180858F7017
:106CB000823021F0833081F0D0E0DDCF41855285F4
:106CC00063857485F80181818F70806A8183448334
:106CD000558366837783CFCF4185528563857485DD
:106CE000F80181818F708067818344835583668337
:106CF0007783C1CFCC23B1F2C295C07FF801AACF70
:106D0000AF92BF92CF92DF92EF92FF920F931F93B9
:106D1000CF93DF9300D000D01F921F92CDB7DEB784
:106D20005C017B0160FF03C0E894E0F8F4F8F4FC38
:106D30000DC00F94DA0E663971058105910530F0AA
:106D40008091820E9091830E059719F5A701442733
:106D50005770052E000C660B770BC5010E9474302E
:106D600064E47DE083E59DE00E94BAF28FEF9FEF3F
:106D700028960FB6F894DEBF0FBECDBFDF91CF913E
:106D80001F910F91FF90EF90DF90CF90BF90AF9049
:106D9000089519821A821B821C821D821E821F8204
:106DA00018868A818F708A8340E053E0B501CE0156
:106DB00001960E94F83540E057E060E070E0C501C0
:106DC0000E949D30E62AF72AD12CC12C09811A8114
:106DD0002B813C814D815E816F817885C5010E9448
:106DE000C130C6CFCF93DF93EC0140E053E060E0C9
:106DF00070E00E949D30611571058105910599F043
:106E00002091820E3091830E2630310561F4CE013F
:106E10000E94803640E053E060E070E0CE01DF91F8
:106E2000CF910C944B30DF91CF9108958F929F9228
:106E3000AF92CF92EF92FF920F931F93CF93DF9376
:106E400000D000D01F921F92CDB7DEB74C0109834E
:106E50001A832B833C834D835E836F8378876EE434
:106E600078E083E59DE00E94BAF2CE0101960E948F
:106E7000D8228981811130C00A810F70013089F1D7
:106E800040F1023019F010E00530F1F5D401ED9138
:106E9000FC91068CF78DE02D09811A812B813C81B4
:106EA0004D815E816F817885C401199581E090E004
:106EB00028960FB6F894DEBF0FBECDBFDF91CF91FD
:106EC0001F910F91FF90EF90CF90AF909F908F9078
:106ED0000895CC24C394DACF813071F1823009F463
:106EE00051C061E478E083E59DE00E94BAF24AE097
:106EF00050E0698183E59DE00E9421F183E59DE0FA
:106F00000E9404F101E010E061E378E083E59DE098
:106F10000E94BAF24AE050E0B80183E59DE00E9489
:106F20000BF283E59DE00E9404F1CE0101960E94E0
:106F3000D82290E080E0BCCFCE0101960E9437C1FC
:106F40004497B8F46EE170E0CE0101960E94B61E3F
:106F5000F4016281738140E052E0CE0101960E940B
:106F6000393560E072E1D40112968D919C910E94B6
:106F70008036D401ED91FC91068CF78DE02DCC2468
:106F8000C3948ACF1D821E821F821886D401ED9180
:106F9000FC91068CF78DE02DCC24C39402E01A817D
:106FA0002B813C8140E07DCF8F929F92AF92BF9228
:106FB000CF92DF92EF92FF920F931F93CF93DF93C5
:106FC000CDB7DEB760970FB6F894DEBF0FBECDBF6A
:106FD0008C017B0140E058E060E070E00E949D3051
:106FE000672B682B692B09F0A9C062E070E0C8012B
:106FF0000E945F2E6C0119861A861B861C861D86D0
:107000001E861F86188A8A858F708A87D7FC96C04D
:1070100040E052E0B801CE0109960E94F83563E0E5
:1070200070E0C8010E945F2EAC011816190614F01A
:107030004FE350E081E0C816D10429F4EF2CFF0C97
:10704000FF08FF2404C082E0C816D104D4F32FEF58
:1070500030E0D7010F9488229A01550F440B550B4D
:107060000F941C2249016901C8010E94EB35E82EEA
:10707000F12C60E0CE0109960E94E91D8816990660
:10708000F9F4CD2841F082E0E816F10419F185E029
:10709000E816F104F9F081E090E060960FB6F894FC
:1070A000DEBF0FBECDBFDF91CF911F910F91FF903B
:1070B000EF90DF90CF90BF90AF909F908F9008950A
:1070C000CD2859F186E0E816F10441F081E0E81698
:1070D000F10421F061E0C8010E940835B401CE013D
:1070E00009960E94901D40E052E0B801CE01099639
:1070F0000E94393582E0E816F10421F085E0E816B7
:10710000F10429F460E071E0C8010E94803660E07B
:1071100072E0C8010E948036BECF85E0E816F10417
:1071200009F4B9CF82E0E816F10409F4B4CF62E0C3
:10713000C8010E94083560E071E0EBCF90E080E08C
:10714000ACCF81E090E008950F931F93CF93DF932E
:1071500000D000D01F921F92CDB7DEB719821A82DD
:107160001B821C821D821E821F8218862A812F701C
:107170002A83FC0102811381C8010E94EB35813012
:1071800041F020F0823011F0853081F490E080E011
:1071900002C081E090E028960FB6F894DEBF0FBEE3
:1071A000CDBFDF91CF911F910F91089540E052E044
:1071B000B801CE0101960E94F83560E0CE0101963B
:1071C0000E94E91DE8CF8F929F92AF92BF92CF921B
:1071D000DF92EF92FF920F931F93CF93DF93CDB780
:1071E000DEB767970FB6F894DEBF0FBECDBF8C0138
:1071F0007B014C018BE0880E911C9F8A8E8AF801DE
:10720000128611861386148E138E672B09F463C0C1
:10721000A090840EB090850EA114B10409F45BC057
:107220006FE270E0C7010F94D3266C01892B09F43B
:107230004AC0F701DE01119690E080E0BD01219186
:10724000222341F02F3231F08431910519F02D9332
:107250000196F5CF860F971FFC011082C5010E9491
:10726000B0C0F80191838083B6016F5F7F4F4FE01C
:1072700050E0C4010F940C27CE0146960E94372D92
:10728000F801948F838F8E899F89892B09F4138647
:10729000C8010E946D2D882319F0C8010E94C02EDC
:1072A00067960FB6F894DEBF0FBECDBFDF91CF91CA
:1072B0001F910F91FF90EF90DF90CF90BF90AF9014
:1072C0009F908F900895B701C5010E94B0C0F8014A
:1072D00091838083DDCFF80111821082D9CFDC0148
:1072E00019968D919C91009739F0DC01ED91FC91FC
:1072F0000280F381E02D199408958F929F92AF92AE
:10730000BF92CF92DF92EF92FF920F931F93CF9392
:10731000DF93CDB7DEB7CD55D1090FB6F894DEBFF8
:107320000FBECDBF8C016B016115710519F04115C0
:107330005105D1F460E772E183E59DE00E94BAF265
:1073400067E672E183E59DE00E94BAF2B80183E549
:107350009DE00E9454F265E672E183E59DE00E94A3
:10736000BAF283E59DE032C0460F571FDA011C9246
:107370000F94DA0E4B0163E672E183E59DE00E9413
:10738000BAF24AE050E0B40183E59DE00E940BF2BE
:1073900060E672E183E59DE00E94BAF2B80183E500
:1073A0009DE00E9454F26DE572E183E59DE00E944C
:1073B000BAF2BAE38B16B1E09B06F4F460E572E131
:1073C0008CEA9CE00E94BAF28CEA9CE00E9404F1F4
:1073D000C35ADF4F0FB6F894DEBF0FBECDBFDF91AB
:1073E000CF911F910F91FF90EF90DF90CF90BF90C2
:1073F000AF909F908F9008956EE472E183E59DE0D9
:107400000E94BAF2B60183E59DE00E9454F26CE45A
:1074100072E183E59DE00E94BAF283E59DE00E945F
:1074200004F11A821982FE0133968EE3DF011D9268
:107430008A95E9F78091820E9091830E059791F5D8
:1074400063E070E0C8010E9491177C01892BE9F587
:10745000E091D20AF091D30A808180FFB9CF61E038
:1074600070E0C8010E949117892B09F4B1CF64E242
:1074700070E0C8010F941B27892B09F0A9CF64E3A2
:1074800072E183E59DE00E94BAF2B80183E59DE0D8
:107490000E9454F283E59DE00E9404F1C8010E941D
:1074A000CDCD96CF61E070E0C8010E9491177C01BC
:1074B000892B49F562E070E0C8010E9491177C01B8
:1074C00069E272E1892B09F448CFE00EF11E60E217
:1074D00072E1C7010F94BB1A892BE9F4F601019000
:1074E0000020E9F73197EC19FD093297A0F0C801A7
:1074F0000E94CDCDF6018081882309F469CFC601B1
:107500000E947AF565CF4FE350E0B801CE010196B5
:107510000F940C27DACF64E270E0C8010F941B27A8
:10752000892B09F055CFB701CE018F5B9F4F0E9489
:10753000E338CE018F5B9F4F0E946D2D882339F178
:10754000B601CE018F5B9F4F0E94E1C71816190646
:10755000F4F489818823D9F08091820E9091830E72
:107560000597A9F068E072E183E59DE00E94BAF218
:10757000BE016F5F7F4F83E59DE00E9454F283E57B
:107580009DE00E9404F1CE0101960E94CDCDCE0176
:107590008F5B9F4F0E946F391BCFCF93DF93EC011E
:1075A000798368831A8619861B861C8E1B8E0E941F
:1075B0006D2D882329F0CE01DF91CF910C94C02E40
:1075C000DF91CF910895CF93DF93EC01FB012481EC
:1075D000358140815181628173810E94C3F1CE0166
:1075E000DF91CF910895CF92DF92EF92FF921F9398
:1075F000CF93DF9300D000D0CDB7DEB764E772E160
:1076000082EA9CE00E94BAF286E8E82E8CE0F82E2E
:1076100010E090E1C92ED12CF70181917F018031DA
:1076200030F460E975E082EA9CE00E9454F2153083
:1076300041F1F7013197808190E0B0E0A0E08983CB
:107640009A83AB83BC83DE82CD82BE016F5F7F4FA6
:1076500082EA9CE00E94E33A62E772E10E94BAF299
:107660001F5F1630C9F626960FB6F894DEBF0FBE20
:10767000CDBFDF91CF911F91FF90EF90DF90CF9022
:10768000089580918B0C90E0B0E0A0E089839A830C
:10769000AB83BC83DE82CD82BE016F5F7F4F82EA07
:1076A0009CE00E94E33A0E9404F1DACFEF92FF924D
:1076B0000F931F93CF93DF9300D000D0CDB7DEB7E9
:1076C0007C018B0160EC7EE083E59DE00E94BAF2D4
:1076D000D701ED91FC916081718183E59DE00E946D
:1076E00054F267EB7EE083E59DE00E94BAF2012E42
:1076F000000C220B330B09831A832B833C8380E11C
:1077000090E09E838D83BE016F5F7F4F83E59DE098
:107710000E94E33A0E9404F140E058E060E070E02B
:10772000C7010E94743026960FB6F894DEBF0FBED4
:10773000CDBFDF91CF911F910F91FF90EF900895F2
:107740003F924F925F926F927F928F929F92AF92F1
:10775000BF92CF92DF92EF92FF920F931F93CF933E
:10776000DF93CDB7DEB72C970FB6F894DEBF0FBE10
:10777000CDBF5C01362E972E3A01690161E27FE0B0
:1077800083E59DE00E94BAF24AE050E0632D792D36
:1077900083E59DE00E940BF269E17FE083E59DE0D7
:1077A0000E94BAF2C301B0E0A0E08F839887A98756
:1077B000BA8730E1432E512C5C864B86BE01695F4F
:1077C0007F4F83E59DE00E94E33A4C0165E17FE055
:1077D0000E94BAF24AE050E0B601C4010E940BF2E6
:1077E0006DE07FE0C4010E94BAF2C701B0E0A0E002
:1077F00089839A83AB83BC835E824D82BE016F5FB7
:107800007F4FC4010E94E33A0E9404F18091240951
:107810009091250970E060E0892B09F047C081E074
:1078200090E0909325098093240926E040E855E2F2
:1078300060E070E087E09AE00E94C6F33092F70AB9
:1078400087E09AE09093F60A8093F50A1092020C72
:107850001092040C1092030C0130110509F44EC073
:107860000CF041C0012B09F44EC0C114D10409F43D
:1078700057C082E0C816D10409F062C070927D0B37
:1078800060927C0B10927F0B10927E0BF092810B1A
:10789000E092800B86E00E9481D31092250910921D
:1078A0002409882309F456C0682F70E0C5010E949E
:1078B000563B90E080E02C960FB6F894DEBF0FBEEA
:1078C000CDBFDF91CF911F910F91FF90EF90DF908F
:1078D000CF90BF90AF909F908F907F906F905F9070
:1078E0004F903F9008950330110581F00430110549
:1078F00009F0BBCFFE24EF24FE24B7CFFE2CEE24EC
:10790000EE24EA94B2CFFF24FA94AFCFEF2821F40B
:1079100092E0E92EF12CEECFEE24E394F12CEACFA5
:1079200070927D0B60927C0B90E080E0EE2011F075
:1079300080E09FEF90937F0B80937E0B85E0ABCF31
:1079400061EF7EE083E59DE00E94BAF21092250986
:107950001092240981E090E0AECF2F923F924F9297
:107960005F926F927F928F929F92AF92BF92CF92CF
:10797000DF92EF92FF920F931F93CF93DF93CDB7D8
:10798000DEB72C970FB6F894DEBF0FBECDBF5C01FB
:1079900009831A832B833C834D835E836F837887AF
:1079A000CE0101960E9437C11C01023011F0053052
:1079B00011F4312C212CF50102811381F80180850D
:1079C0008F70853009F07FC0C8010E94BAC1E82ECF
:1079D000F12CF2E0EF16F1040CF475C060E0C80180
:1079E0000E9428C1FC01818592859C878B8761E07C
:1079F000C8010E9428C1FC014184528463847484BC
:107A000088248A94982CF2E0EF16F10459F062E091
:107A1000C8010E9428C1FC0181849284F3E0EF1622
:107A2000F104A1F48FE390E09A87898792E0C92E50
:107A3000D12C29853A85D1010F94802224E630E0AB
:107A400040E050E00F941C2279011CC063E0C801A3
:107A50000E9428C1FC01818592859A87898782E0EE
:107A6000C82ED12CF4E0EF16F10439F064E0C8011F
:107A70000E9428C1FC01C184D28489859A85710144
:107A8000892BB9F684019601A2016B857C85C5011D
:107A90000E94A03B2C960FB6F894DEBF0FBECDBF60
:107AA000DF91CF911F910F91FF90EF90DF90CF90DA
:107AB000BF90AF909F908F907F906F905F904F900E
:107AC0003F902F90089590E080E0E4CF8F929F92B6
:107AD000AF92BF92DF92EF92FF920F931F93CF93DB
:107AE000DF93CDB7DEB7A5970FB6F894DEBF0FBE14
:107AF000CDBF7C010E8F1F8F28A339A34AA35BA3A0
:107B00006CA37DA3CE014E960E940A1F4B015C011F
:107B1000D7011296ED91FC9180858F70843009F029
:107B2000E9C0102F61857285CE0101960E94E3386D
:107B3000CE0101960E946D2D882309F44AC08985E3
:107B4000893009F046C070E060E0CE0101960E94E5
:107B50005F2E082FD92E64EE7EE083E59DE00E9423
:107B6000BAF24AE050E0602F7D2D83E59DE00E944F
:107B70000BF262EE7EE083E59DE00E94BAF2B50171
:107B8000A40183E59DE00E946CC66CED7EE083E578
:107B90009DE00E94BAF2612F70E04AE050E083E578
:107BA0009DE00E940BF283E59DE00E9404F180912C
:107BB000240990912509892B29F140E053E0B70170
:107BC000CE014E960E94393570E060E0C7010E94F8
:107BD000563B10E000E0CE0101960E946F39C801CB
:107BE000A5960FB6F894DEBF0FBECDBFDF91CF9143
:107BF0001F910F91FF90EF90DF90BF90AF909F90FB
:107C00008F90089581E090E0909325098093240956
:107C100026E040E855E260E070E087E09AE00E94EC
:107C2000C6F30093F70A87E09AE09093F60A8093F0
:107C3000F50A1092020C1092040C1092030CE981C8
:107C4000FA81153021F01F3011F0123011F58085C6
:107C50008F70808770E060E083ED97E090937D0BFC
:107C600080937C0B10927F0B10927E0B7093810B94
:107C70006093800B86E00E9481D3109225091092B8
:107C8000240901E010E0882309F4A5CF682F70E0F3
:107C90009DCF80858F708061808722E538EB42E13F
:107CA00052E4C501B4010F94A42220E030E040E288
:107CB00051E40F9416212DEE3EE94CE35EE30F9460
:107CC00010234B015C0120E030E0A9010F94B823A0
:107CD00020E030E040E05FE387FD07C0C501B4016C
:107CE0000F94A4220F948223B7CFC501B4010F943F
:107CF000A322F8CF10E000E072CFCF92DF92EF9294
:107D0000FF920F931F93CF93DF9300D000D01F9269
:107D10001F92CDB7DEB77C0109831A832B833C8386
:107D20004D835E836F837887CE0101960E9437C1B1
:107D30008C018981882359F09A819F70923008F0D4
:107D4000BAC0823011F0853011F410E000E070E02C
:107D500060E0C7010E945F2ED82EC92E64ED7EE040
:107D600083E59DE00E94BAF24AE050E06D2D7C2D43
:107D700083E59DE00E940BF262ED7EE083E59DE0ED
:107D80000E94BAF24AE050E0B80183E59DE00E940B
:107D90000BF283E59DE00E9404F18091240990910B
:107DA0002509892BE9F040E053E0B701CE010196A7
:107DB0000E94393570E060E0C7010E94563B90E0B8
:107DC00080E028960FB6F894DEBF0FBECDBFDF91DE
:107DD000CF911F910F91FF90EF90DF90CF9008957A
:107DE00081E090E0909325098093240926E040E803
:107DF00055E260E070E087E09AE00E94C6F3D0921E
:107E0000F70A87E09AE09093F60A8093F50A1092B9
:107E1000020C1092040C1092030C80ED97E09093EA
:107E20007D0B80937C0B10927F0B10927E0B0115C3
:107E30001105E1F185E090E09093810B8093800B38
:107E400086E00E9481D3D82E64E670E080E090E066
:107E50000E94F3D0D1100AC06BEC7EE083E59DE078
:107E60000E94BAF283E59DE00E9404F182ED97E062
:107E700090937D0B80937C0B10927F0B10927E0B66
:107E800024E6209FC001219F900D11249093810B27
:107E90008093800B86E00E9481D310922509109276
:107EA0002409882359F0682F70E086CF1092810B47
:107EB0001092800BC5CF8FEF9FEF83CF81E090E0D2
:107EC00080CF2F923F924F925F926F927F928F92CC
:107ED0009F92AF92BF92CF92DF92EF92FF920F9359
:107EE0001F93CF93DF93CDB7DEB7C75CD1090FB631
:107EF000F894DEBF0FBECDBF1C01CF54DF4F088307
:107F0000C15BD040CE54DF4F1883C25BD040CD540C
:107F1000DF4F2883C35BD040CC54DF4F3883C45B32
:107F2000D040CB54DF4F4883C55BD040CA54DF4FAD
:107F30005883C65BD040C954DF4F6883C75BD040CD
:107F4000C854DF4F7883C85BD040C754DF4FF982F5
:107F5000E882C95BD040C254DF4FC882CE5BD040BC
:107F6000C154DF4FA882CF5BD0400F94DA0E6B0173
:107F7000C054DF4F79836883C05CD040683C710592
:107F8000B4F467E97BE08CEA9CE00E94BAF24AE034
:107F900050E0B6018CEA9CE00E940BF28CEA9CE077
:107FA0000E9404F1AA24AA94BA2C0C9482490E943B
:107FB00026D1CC53DF4F688379838A839B83C45C4B
:107FC000D040CE54DF4F8881C25BD0408F70282FC5
:107FD00030E0C454DF4F39832883CC5BD04080919C
:107FE000820E9091830ECE53DF4F99838883C25CBB
:107FF000D040C754DF4FE881F981C95BD04030974A
:1080000021F0808181110C947E4ED1011B968C91C0
:10801000882341F0C1010B96C754DF4F99838883B1
:10802000C95BD040C454DF4FE881F981CC5BD040BC
:10803000EF2B11F00C94DA4EC754DF4FE881F98131
:10804000C95BD040309711F00C94874ED1015B96FC
:108050000D90BC91A02DC454DF4FB983A883CC5B95
:10806000D040AB2B11F40C94DA4ECE54DF4F888104
:10807000C25BD0408F7011F00C94DA4EC454DF4FC5
:108080006881CC5BD040CE018F549F4F0E94031B70
:10809000C756DF4F2883C959D040C656DF4F3883B3
:1080A000CA59D040C556DF4F4883CB59D040C4563B
:1080B000DF4F5883CC59D040C356DF4F6883CD592A
:1080C000D040C256DF4F7883CE59D040C156DF4FE3
:1080D0008883CF59D040C056DF4F9883C05AD040D4
:1080E0000C94DA4ED1012D913C91232B09F45ACFF7
:1080F000C454DF4FE881F981CC5BD040349799F5C7
:10810000C154DF4FE880CF5BD040CF54DF4F0881B0
:10811000C15BD040CE54DF4F1881C25BD040CD54FC
:10812000DF4F2881C35BD040CC54DF4F3881C45B24
:10813000D040CB54DF4F4881C55BD040CA54DF4F9D
:108140005881C65BD040C954DF4F6881C75BD040BF
:10815000C854DF4F7881C85BD040C1010E94961F90
:108160005C010C94824928E0FE01EF54FF4FDE01D0
:10817000A755BF4F01900D922A95E1F7CF54DF4FDD
:108180001881C15BD040143009F412C348F41123A4
:1081900009F469C0912C812CAA24AA94BA2C8CC30E
:1081A00088EF810F8230B0F788E0FE01EF54FF4F77
:1081B000DE01119601900D928A95E1F7CE54DF4FC2
:1081C0008881C25BD040807F09F485C3CE018F5483
:1081D0009F4F0E9449204B015C0181149104A1042E
:1081E000B10409F478C3193041F4B094A094909488
:1081F0008094811C911CA11CB11CB101CE018F5433
:108200009F4F0E944AC760E0CE018F549F4F0E944B
:108210002A1B6A962FAF6A976B963FAF6B976C9647
:108220004FAF6C976D965FAF6D976E966FAF6E9711
:108230006F967FAF6F97A0968FAFA097A1969FAFD5
:10824000A197C454DF4FA881B981CC5BD040A23044
:10825000B10509F49AC30CF044C3AB2B09F4D3C3A2
:10826000912C812C58C519821A821B821C821D8276
:108270001E821F8218862A812F702A83CE54DF4FD8
:108280002881C25BD040207F09F484CFC454DF4FE3
:1082900008811981CC5BD0400A30110509F440C235
:1082A00054F40115110571F10230110509F4E1C012
:1082B000912C812C2CC2C454DF4F28813981CC5B96
:1082C000D0402B30310509F4D3C12C30310581F772
:1082D000B101CE0101960E944AC7CE018F549F4F33
:1082E0000E949520BC01CE0101960E94262388E0C1
:1082F000FE013196DE01AF54BF4F01900D928A9579
:10830000E1F702C2892B59F064E57BE083E59DE04B
:108310000E94BAF283E59DE00E9404F1C9CFC10139
:108320000E94F74F8C0161E070E01816190614F0F6
:1083300070E060E04AE050E083E59DE00E940BF2CF
:1083400060E077E083E59DE00E9454F2CE018F5417
:108350009F4F0E94511FAB01BC012AE030E083E532
:108360009DE00E94C3F183E59DE00E9404F1CE01EF
:108370008F549F4F1016110614F00C946C4E0E94EF
:10838000511F672B682B692B09F069C162E0CE0190
:108390008F549F4F0E942A1BCF56DF4F2883C1590D
:1083A000D040CE56DF4F3883C259D040CD56DF4F34
:1083B0004883C359D040CC56DF4F5883C459D0406E
:1083C000CB56DF4F6883C559D040CA56DF4F7883FC
:1083D000C659D040C956DF4F8883C759D040C856C8
:1083E000DF4F9883C859D04088248394982C31E07B
:1083F000C554DF4F3883CB5BD0405524539442C0E3
:1084000061E0CE018F549F4F0E942A1BC757DF4F58
:108410002883C958D040C657DF4F3883CA58D04048
:10842000C557DF4F4883CB58D040C457DF4F5883E0
:10843000CC58D040C357DF4F6883CD58D040C25787
:10844000DF4F7883CE58D040C157DF4F8883CF5855
:10845000D040C057DF4F9883C059D04088248394C0
:10846000982C81E0C554DF4F8883CB5BD040512CE2
:1084700009C0912C812CC554DF4F1882CB5BD040B2
:1084800055245A94B101CE0101960E944AC78A81AF
:10849000982F92959F70945F9F70923060F4CE54A5
:1084A000DF4F9881C25BD04092959F70923019F453
:1084B0008F7080628A83D10118969C91973071F4F5
:1084C000CE54DF4F8881C25BD040807E803211F075
:1084D000803421F48A818F7080628A83F101A185C2
:1084E000B285892F90E0109741F0ED91FC911197A2
:1084F000048CF58DE02DCD0119957C01CF54DF4F13
:108500000881C15BD040CE54DF4F1881C25BD040A0
:10851000CD54DF4F2881C35BD040CC54DF4F38812E
:10852000C45BD040CB54DF4F4881C55BD040CA54B8
:10853000DF4F5881C65BD040C954DF4F6881C75BAD
:10854000D040C854DF4F7881C85BD040CE0101963F
:108550000E946123CF57DF4F2883C158D040CE57A8
:10856000DF4F3883C258D040CD57DF4F4883C358C0
:10857000D040CC57DF4F5883C458D040CB57DF4F43
:108580006883C558D040CA57DF4F7883C658D0405B
:10859000C957DF4F8883C758D040C857DF4F9883EB
:1085A000C858D040CE0101960E94D822C554DF4F52
:1085B000F881CB5BD040FF2351F1CE54DF4F88814F
:1085C000C25BD04082958F709FE0980F9F70923071
:1085D00020F08A5F8F708230D0F48A8182958F700C
:1085E00081508230A0F42D8130E0AFEFB0E00F94E5
:1085F0004E222FEF611504E670078105910534F4D2
:1086000024E630E040E050E00F941C222D8388E007
:10861000FE013196DE01AF54BF4F01900D928A9555
:10862000E1F712E1912AF12CAA24AA94BA2CD101E3
:1086300018968C911897873009F08DC5C054DF4F7C
:10864000E881F981C05CD040EE35F1400CF090C378
:1086500060E17BE08CEA9CE00E94BAF29FCC912C16
:10866000812C91E0C554DF4F9883CB5BD040C5CEC1
:10867000B101CE0101960E944AC7CA54DF4F8881DA
:10868000C65BD0409A8192959F7039F0923049F044
:10869000912C812CFF24F3943BC09A819F709062AF
:1086A0009A8390E08536910514F084E690E08E83FD
:1086B00088E0FE013196DE01AF54BF4F01900D926C
:1086C0008A95E1F762E0CE018F549F4F0E94031B11
:1086D000EA962FAFEA97EB963FAFEB97EC964FAF4A
:1086E000EC97ED965FAFED97EE966FAFEE97EF9646
:1086F0007FAFEF97C158DF4F8883CF57D040C05826
:10870000DF4F9883C058D040812CF2E19F2EF12C8E
:10871000C554DF4F1882CB5BD04055245A9484CF88
:10872000B101CE0101960E944AC7C954DF4F68814A
:10873000C75BD040C854DF4F7881C85BD0407170B0
:10874000CE0101960E94A128C554DF4F8883CB5BE0
:10875000D040912C812CFF24F3948823F1F288E0FF
:10876000FE013196DE01AF54BF4F01900D928A9504
:10877000E1F762E0CE018F549F4F0E94031BE29607
:108780002FAFE297E3963FAFE397E4964FAFE497BE
:10879000E5965FAFE597E6966FAFE697E7967FAF12
:1087A000E797E8968FAFE897E9969FAFE997ACCF48
:1087B000C454DF4F28813981CC5BD040293031054A
:1087C00009F461C0C1010E94F74F1816190674F52B
:1087D00062E0CE018F549F4F0E942A1BAA962FAFB2
:1087E000AA97AB963FAFAB97AC964FAFAC97AD9611
:1087F0005FAFAD97AE966FAFAE97AF967FAFAF97C7
:10880000E0968FAFE097E1969FAFE197882483943D
:10881000982CAA24AA94BA2CF12C31E0C554DF4F2D
:108820003883CB5BD0405524539401CF61E0CE0117
:108830008F549F4F0E942A1BA2962FAFA297A396F8
:108840003FAFA397A4964FAFA497A5965FAFA59708
:10885000A6966FAFA697A7967FAFA797A8968FAF5C
:10886000A897A9969FAFA99788248394982CAA24A7
:10887000AA94BA2CF12C81E0C554DF4F8883CB5BDE
:10888000D040512CD4CE40E050E061E070E0C10116
:108890000E949D30672B682B692BA9F040E050E0C7
:1088A00061E070E0C1010E944B308824839424E091
:1088B000922EAA24A394B12CF12CC554DF4F188218
:1088C000CB5BD040DDC040E050E061E070E0C10132
:1088D0000E947430EACF95E0892E912CA12CB12C06
:1088E00082CCC454DF4FE881F981CC5BD040EA30C0
:1088F000F10509F4B3C13B9709F0B2CCCE54DF4F78
:108900008881C25BD04082958F70823009F023C28B
:10891000C501B40124E630E040E050E00F941C2291
:10892000CA54DF4F8881C65BD04090E0280F391FC2
:1089300037FF02C030E020E02536310514F024E690
:1089400030E0CA54DF4F2883C65BD04062E0CE01DE
:108950008F549F4F0E94031B2A962FAF2A972B9666
:108960003FAF2B972C964FAF2C972D965FAF2D973F
:108970002E966FAF2E972F967FAF2F9760968FAF63
:10898000609761969FAF6197C3C1C554DF4F18824E
:10899000CB5BD040D10119968D919C911A9700978D
:1089A00009F038C018968C9190E000E5402E512CCB
:1089B000612C712C8530910549F0412C512C3201EC
:1089C000449721F0412C512C32014A94CE54DF4F70
:1089D000E881C25BD040E295EF70E150EB3008F0E7
:1089E0002EC1F0E08827E850FB4B8F4F0D94712289
:1089F000124512451F461F461F46EC45B245B2457B
:108A0000B24543454345F1E0C554DF4FF883CB5BA6
:108A1000D040C0CFDC01ED91FC91048CF58DE02DB0
:108A20001995C3CFCB54DF4F1881C55BD040C5012A
:108A3000B40124E630E040E050E00F941C22DA015B
:108A4000C901810F911DA11DB11DB7FF03C080E0B9
:108A500090E0DC018F3F9105A105B10529F024F0DC
:108A60008FEF90E0A0E0B0E0CB54DF4F8883C55B90
:108A7000D040812C12E1912EF12CAA24AA94BA2C78
:108A800055245A94D4CDCB54DF4FC880D980EA8086
:108A9000FB80C55BD040B4E68B169104A104B10401
:108AA000DCF5A4E6B0E0A70196010F943B22860E08
:108AB000971EA81EB91E4114510461047104B9F037
:108AC000A30192010F943B22362F272FB501A40159
:108AD00077FF03C040E050E0BA01832E922E5C0184
:108AE000481559056A057B0514F44A015B01CB540E
:108AF000DF4F88829982AA82BB82C55BD040CE5468
:108B0000DF4F8881C25BD0408F708066CE54DF4FCC
:108B10008883C25BD040ADCFC501B40124E630E00C
:108B200040E050E00F941C22C20ED31EE41EF51E3E
:108B3000411451046104710461F0F7FE03C0C12CBB
:108B4000D12C76014C145D046E047F0414F473017F
:108B50006201CB54DF4FC882D982EA82FB82C55BB7
:108B6000D04087CFCB54DF4F688179818A819B8148
:108B7000C55BD0400F9482236B017C01C501B40119
:108B800024E630E040E050E00F941C22CA01B90115
:108B90006C0D7D1D8E1D9F1D4114510461047104D7
:108BA00081F06B017C01F7FE03C0C12CD12C760152
:108BB000C701B601461657066806790614F4C301C4
:108BC000B2010F94B720CB54DF4F688379838A8337
:108BD0009B83C55BD0404DCFCB54DF4F88819981BB
:108BE000AA81BB81C55BD040880E991EAA1EBB1E00
:108BF0004114510461047104C9F0A4E6B0E0A3017A
:108C000092010F943B22362F272FB501A40177FF45
:108C100003C040E050E0BA01832E922E5C0148155B
:108C200059056A057B0514F44A015B01CB54DF4FFB
:108C300088829982AA82BB82C55BD0401ACF88E025
:108C4000FE013196DE01AF54BF4F01900D928A951F
:108C5000E1F7912C812CFF24F3940FCFCE54DF4FFA
:108C60008881C25BD04082958F70823009F055C0F8
:108C7000C501B40124E630E040E050E00F941C222E
:108C8000C954DF4F8881C75BD040C854DF4F68812B
:108C9000C85BD040962F9170280F391F2E36E1E027
:108CA0003E072CF437FF05C02DE631E002C030E06E
:108CB00020E0C954DF4F2883C75BD040C854DF4F42
:108CC0008881C85BD04030FB80F9C854DF4F88836F
:108CD000C85BD04062E0CE018F549F4F0E94031BBF
:108CE00062962FAF629763963FAF639764964FAFDC
:108CF000649765965FAF659766966FAF6697679660
:108D00007FAF679768968FAF689769969FAF6997AF
:108D1000812CB2E19B2EF12C18C088E0FE01319627
:108D2000DE01AF54BF4F01900D928A95E1F768E4E0
:108D30007BE08CEA9CE00E94BAF28CEA9CE00E9404
:108D400004F1912C812CFF24F394C554DF4F188239
:108D5000CB5BD04092CE88E0FE013196DE01AF546D
:108D6000BF4F01900D928A95E1F76CE37BE0E1CF74
:108D7000C254DF4F1881CE5BD040112309F46FC07D
:108D80001296ED91FC9180858F70853009F074C04A
:108D9000CE53DF4FE881F981C25CD040359709F4AA
:108DA0006BC0C1010E94F74F21E0181619060CF0A4
:108DB00020E0522EC754DF4F48815981C95BD04013
:108DC000C154DF4F2881CF5BD040BE016F547F4F2D
:108DD000D10112968D919C910E94304FC454DF4F67
:108DE000E881F981CC5BD040319709F045C0CE5481
:108DF000DF4F8881C25BD040807FF1F1C154DF4FEB
:108E0000C880CF5BD040E52CC755DF4F0881C95AD9
:108E1000D040C655DF4F1881CA5AD040C555DF4FE4
:108E20002881CB5AD040C455DF4F3881CC5AD0402E
:108E3000C355DF4F4881CD5AD040C255DF4F5881CE
:108E4000CE5AD040C155DF4F6881CF5AD040C0556F
:108E5000DF4F7881C05BD040C1010E94D633CF5430
:108E6000DF4F8881C15BD040853009F445C150F4A3
:108E70008330B9F1D12CC3C0C254DF4F1882CE5B0E
:108E8000D040EDCF863009F482C0873099F7C10118
:108E90000E94EB35182F863009F066C064EE7AE048
:108EA00083E59DE00E94BAF24AE050E066E070E09F
:108EB00083E59DE00E940BF283E59DE00E9404F1B2
:108EC00062E0CE018F549F4F0E942A1B29AF3AAF18
:108ED0004BAF5CAF6DAF7EAF8FAF21969FAF219749
:108EE0003FC0C1010E94EB35853021F093E0A92EEF
:108EF000B12C08C26BEF7AE083E59DE00E94BAF2E4
:108F00004AE050E065E070E083E59DE00E940BF2EE
:108F100083E59DE00E9404F1B101CE018F549F4F83
:108F20000E944AC761E0CE018F549F4F0E942A1BC6
:108F300022962FAF229723963FAF239724964FAFC9
:108F4000249725965FAF259726966FAF269727968D
:108F50007FAF279728968FAF289729969FAF29979D
:108F6000689480F890F886CF66EC7AE083E59DE01F
:108F70000E94BAF2612F70E04AE050E083E59DE084
:108F80000E940BF283E59DE00E9404F1AFCF40E028
:108F900050E061E070E0C1010E949D30672B682BBA
:108FA000692B09F0A6C0FFEF5F120EC0C1010E943D
:108FB000F74F512C181619064CF46CEA7AE083E549
:108FC0009DE00E94BAF292CF5110F7CFB101CE01CD
:108FD0008F549F4F0E944AC761E0CE018F549F4F2C
:108FE0000E942A1B29AB3AAB4BAB5CAB6DAB7EABA3
:108FF0008FAB98AF689480F890F8E6E0DE2E84019D
:109000000160CE54DF4F8881C25BD040982F9F70A3
:10901000923050F4CF54DF4F9881C15BD0409923F8
:1090200019F0840101601160807F09F489C0126029
:10903000C254DF4F2881CE5BD04021111D7FA80193
:10904000B101CE018F549F4F0E9439354801AA24A7
:10905000A394B12CF110FFC6D10119968D919C916A
:10906000009709F0A7C340E050E062E070E0C10162
:109070000E949D30672B682B692B09F4CDC368E6ED
:1090800079E08CEA9CE00E94BAF28CEA9CE00E94B3
:1090900004F192FC0CC666E579E083E59DE00E9450
:1090A000BAF24AE050E0B50183E59DE00E940BF280
:1090B0006FE479E083E59DE00E94BAF20E9426D138
:1090C000AB01BC01CC53DF4F088119812A813B8160
:1090D000C45CD040401B510B620B730B2AE030E0A4
:1090E00083E59DE00E941FF183E59DE00E9404F16D
:1090F00009C167E97AE063CF0FEF50120BC0C101DD
:109100000E94F74F55245394181619062CF06AE75D
:109110007AE055CF5520D9F362E0CE018F549F4FAE
:109120000E942A1B29A73AA74BA75CA76DA77EA779
:109130008FA798AB689480F890F875E0D72E5FCF32
:1091400040E052E0B101CE018F549F4F0E94F835AC
:1091500081116DCF6DCF3FEF53129DC0C1010E94B1
:10916000F74F55245394181619060CF497C0512C38
:109170006CE67AE083E59DE00E94BAF2052D052CAD
:10918000000C110BC054DF4F19830883C05CD04022
:109190004AE050E0B80183E59DE00E940BF265E6ED
:1091A0007AE083E59DE00E94BAF2C554DF4F188152
:1091B000CB5BD040612F70E04AE050E083E59DE05A
:1091C0000E940BF283E59DE00E9404F1C754DF4F3B
:1091D00008811981C95BD0400115110509F4B7C098
:1091E0006FED7DE0C8010F94BB1ACC24C394D12C41
:1091F000892B09F45DC068EE7DE0C8010F94BB1AAD
:1092000042E0C42ED12C892B09F452C063E07EE0E9
:10921000C8010F94BB1A35E0C32ED12C892B09F459
:1092200047C06CE07EE0C8010F94BB1A26E0C22E56
:10923000D12C892BE9F161E87EE0C8010F94BB1ABB
:10924000892B99F16AE87EE0C8010F94BB1A892B3B
:1092500009F473C064E57EE0C8010F94BB1ABEE058
:10926000CB2ED12C892B21F16DE57EE0C8010F9426
:10927000BB1AAFE0CA2ED12C892BD1F063E97EE076
:10928000C8010F94BB1AD12CC12C892B89F4F5E1AC
:10929000CF2ED12C0DC0552009F46ACF81E0C554E2
:1092A000DF4F8883CB5BD04063CF93E1C92ED12CB5
:1092B000C1010E94EB35682E712C6114710431F4E8
:1092C000C054DF4F68807980C05CD040C114D104A5
:1092D00009F486C06C147D04A1F169E47AE083E5A9
:1092E0009DE00E94BAF24AE050E0B30183E59DE0C0
:1092F0000E940BF283E59DE00E9404F1EDEFAE2E9B
:10930000BB24BA94C501C953DF4F0FB6F894DEBF32
:109310000FBECDBFDF91CF911F910F91FF90EF90C6
:10932000DF90CF90BF90AF909F908F907F906F9085
:109330005F904F903F902F90089584E1C82ED12CDC
:10934000B7CFC754DF4F19821882C95BD040C454CD
:10935000DF4FE881F981CC5BD0403197A9F4C2544A
:10936000DF4FF881CE5BD040FF2399F0CE54DF4F22
:109370008881C25BD040807F01E0C254DF4F088308
:10938000CE5BD040811105C0C254DF4F1882CE5B46
:10939000D040CF54DF4FD880C15BD04015E11D15C0
:1093A00008F4E7C1ED2DF0E08827E652F64B8F4F29
:1093B0000D947122334A6B4B514B724A334A324BF4
:1093C000F84ABD4A334A334AA54BAF4BCD4BCD4B40
:1093D000854B854BB94BB94BB94B854B854B854B71
:1093E000D10119968D919C91009709F4B0CFDC01C1
:1093F000ED91FC910488F589E02DC154DF4FA880E0
:10940000CF5BD040C554DF4FC880CB5BD0407801E4
:10941000CF54DF4F0881C15BD040CE54DF4F18815D
:10942000C25BD040CD54DF4F2881C35BD040CC54C9
:10943000DF4F3881C45BD040CB54DF4F4881C55BE0
:10944000D040CA54DF4F5881C65BD040C954DF4F6B
:109450006881C75BD040C854DF4F7881C85BD0407B
:1094600019950C94B040D12CC254DF4F8881CE5B4B
:10947000D040882309F4EECDC154DF4FC880CF5BC4
:10948000D040952D9170E92EC755DF4F0881C95AFC
:10949000D040C655DF4F1881CA5AD040C555DF4F5E
:1094A0002881CB5AD040C455DF4F3881CC5AD040A8
:1094B000C355DF4F4881CD5AD040C255DF4F588148
:1094C000CE5AD040C155DF4F6881CF5AD040C055E9
:1094D000DF4F7881C05BD040C1010E94D633E89451
:1094E00091F8B8CDC1010E94EB35853009F0FECC72
:1094F00064E37AE083E59DE00E94BAF24AE050E03E
:1095000065E070E083E59DE00E940BF283E59DE05D
:109510000E9404F1B101CE018F549F4F0E944AC7AF
:10952000D10118968C918530C9F46EE0CE018F542C
:109530009F4F0E942A1B29A33AA34BA35CA36DA3B0
:109540007EA38FA398A7689480F890F8D12CB1E0FF
:10955000C554DF4FB883CB5BD04086CF61E0CE01EE
:109560008F549F4F0E942A1B298F3A8F4B8F5C8FFD
:109570006D8F7E8F8F8F98A3E6CFC1010E94EB3550
:10958000182F863091F56DE17AE083E59DE00E9429
:10959000BAF24AE050E066E070E083E59DE00E94A8
:1095A0000BF283E59DE00E9404F162E0CE018F544E
:1095B0009F4F0E942A1B298B3A8B4B8B5C8B6D8BA8
:1095C0007E8B8F8B988F40E050E068E070E0C101A7
:1095D0000E944B30689480F890F8D12CE1E0C5549B
:1095E000DF4FE883CB5BD0403FCF6FEF79E0BECC5D
:1095F00040E050E061E070E0C1010E949D30672BC7
:10960000682B692B61F5511027C0B101CE018F5431
:109610009F4F0E944AC761E0CE018F549F4F0E9426
:109620002A1B29873A874B875C876D877E878F87C0
:10963000988B40E050E068E070E0C1010E94743017
:10964000689480F890F876E0D72EF1E0C554DF4FAB
:10965000F883CB5BD04008CF65EE79E0B0CC60ED0D
:1096600079E0ADCC5520D1F062E0CE018F549F4F10
:109670000E942A1B29833A834B835C836D837E83FC
:109680008F839887689480F890F865E0D62E01E083
:10969000C554DF4F0883CB5BD040E6CE63EB79E067
:1096A0008ECCCE54DF4F8881C25BD0408F70D12CDE
:1096B000823068F7C1010E94EB35689480F890F819
:1096C000853009F413CCD12C11E0C554DF4F188339
:1096D000CB5BD040C9CECE54DF4F8881C25BD04037
:1096E0008F70823080F7552081F06AE979E083E558
:1096F0009DE00E94BAF261E0C1010E94083560E07D
:1097000071E1C1010E948036F1CBCE54DF4F8881D8
:10971000C25BD040982F9F70923008F043C0DD208C
:1097200069F0807F31F4B101CE018F549F4F0E94C8
:109730004AC7689480F823E0922AD12C31E0C554BE
:10974000DF4F3883CB5BD0408FCE689492F8D12C1A
:1097500081E0C554DF4F8883CB5BD04085CE6894D1
:1097600092F8D12C91E0C554DF4F9883CB5BD04069
:109770007BCECE54DF4F8881C25BD040807F51F4D6
:10978000689490F8D12CA1E0C554DF4FA883CB5B3F
:10979000D0406ACEB3E09B2A20CFD12C812C54E05C
:1097A000952E53CFD12C21E0C554DF4F2883CB5BBE
:1097B000D0405ACEDC01ED91FC91008CF18DE02D72
:1097C000CF54DF4F0881C15BD040CE54DF4F1881AA
:1097D000C25BD040CD54DF4F2881C35BD040CC5416
:1097E000DF4F3881C45BD040CB54DF4F4881C55B2D
:1097F000D040CA54DF4F5881C65BD040C954DF4FB8
:109800006881C75BD040C854DF4F7881C85BD040C7
:109810001995811128CC33CCF10181859285892B52
:1098200009F473C08114910439F0A401B101CE018F
:109830008F549F4F0E943935D10119968D919C917B
:10984000C754DF4FE880F980C95BD040DC01ED915F
:10985000FC910488F589E02DC154DF4FA880CF5BCF
:10986000D040C554DF4FC880CB5BD040CF54DF4FD2
:109870000881C15BD040CE54DF4F1881C25BD0401D
:10988000CD54DF4F2881C35BD040CC54DF4F3881AB
:10989000C45BD040CB54DF4F4881C55BD040CA5435
:1098A000DF4F5881C65BD040C954DF4F6881C75B2A
:1098B000D040C854DF4F7881C85BD04019955C0117
:1098C000F10181859285DC01ED91FC91048CF58D8F
:1098D000E02D1995059711F4689480F892FC2CC13D
:1098E000DD2021F06D2DC1010E940835CE53DF4FE0
:1098F00008811981C25CD040B4010530110509F41A
:10990000CACBC1010E948036C6CB8085863009F45F
:1099100077C008F5843009F417C1853009F7811440
:10992000910439F0A401B101CE018F549F4F0E94E0
:109930003935C454DF4F08811981CC5BD0400230E7
:10994000110509F4FDC00330110509F4D2C001303E
:10995000110531F6CAC0883009F45AC1893009F0BE
:10996000BFCF8114910439F0A401B101CE018F540D
:109970009F4F0E943935C554DF4FE881CB5BD04003
:10998000EE2309F4ADCF552079F0CF54DF4F888115
:10999000C15BD040813041F4CE54DF4F8881C25B3F
:1099A000D040807F09F49CCFCF54DF4F0881C15B4A
:1099B000D040CE54DF4F1881C25BD040CD54DF4F32
:1099C0002881C35BD040CC54DF4F3881C45BD0408A
:1099D000CB54DF4F4881C55BD040CA54DF4F58811C
:1099E000C65BD040C954DF4F6881C75BD040C854C4
:1099F000DF4F7881C85BD040C1010E947D3EF2C03C
:109A0000CF54DF4FF880C15BD040FF2009F487CFEF
:109A100070E060E0C1010E945F2E8C01811491040E
:109A200039F0A401B101CE018F549F4F0E94393506
:109A30000115110509F454CF712C612C17FF06C0D4
:109A400011950195110966246394712CC801019741
:109A50008634910508F044CFE02E61E0802F0E940B
:109A6000ABCEEFEFEF0DE53110F5F0E08827E45CC9
:109A7000F24B8F4F0D947122514D534D574D574D11
:109A8000534D514D534D574D574D574D574D574DC4
:109A9000574D514D514D574D574D574D574D514DB8
:109AA000514DF1E06F26662D8E2D0E947DCE63E62E
:109AB00079E083E59DE00E94BAF24AE050E0B80107
:109AC00083E59DE00E940BF261E679E083E59DE08D
:109AD0000E94BAF24AE050E0B30183E59DE00E94A3
:109AE0000BF283E59DE00E9404F1689480F890F801
:109AF00023C0C1010E94FD2D892B49F4D101ED91B4
:109B0000FC916081718182E995E00E940FD2CE01C3
:109B10008F549F4F0E940A1F20E030E048EC52E42F
:109B20000F9416210F9482232B0188E00F94730D5C
:109B3000A201C1010E94BC2DAA24A394B12CD0CEB5
:109B4000689480F891F8F8CF8114910439F0A40159
:109B5000B101CE018F549F4F0E943935C554DF4F5C
:109B6000B881CB5BD040BB2309F4BACECF54DF4FD2
:109B70008881C15BD0405520B9F1813041F4CE5489
:109B8000DF4F8881C25BD040807F09F4A9CECF54DB
:109B9000DF4F0881C15BD040CE54DF4F1881C25BDC
:109BA000D040CD54DF4F2881C35BD040CC54DF4F31
:109BB0003881C45BD040CB54DF4F4881C55BD04077
:109BC000CA54DF4F5881C65BD040C954DF4F68810B
:109BD000C75BD040C854DF4F7881C85BD040C1011B
:109BE0000E94AD3C5C017CCE813089F6CE018F5461
:109BF0009F4F0E9437C1449750F66EE170E0CE014E
:109C00008F549F4F0E94B61E689480F891F8BFCF82
:109C10008114910439F0A401B101CE018F549F4FFA
:109C20000E943935C554DF4FF881CB5BD040FF230C
:109C300009F456CE552079F0CF54DF4F8881C15BAF
:109C4000D040813041F4CE54DF4F8881C25BD04098
:109C5000807F09F445CECF54DF4F0881C15BD040EF
:109C6000CE54DF4F1881C25BD040CD54DF4F2881E6
:109C7000C35BD040CC54DF4F3881C45BD040CB5461
:109C8000DF4F4881C55BD040CA54DF4F5881C65B67
:109C9000D040C954DF4F6881C75BD040C854DF4F04
:109CA0007881C85BD040C1010E94663D9BCFCE53F6
:109CB000DF4F28813981C25CD0402530310509F45D
:109CC000EAC940E054E0B101CE018F549F4F0E9499
:109CD000393560E074E015CE0E94511F672B682B68
:109CE000692B11F00C940042912C812C11E0C55489
:109CF000DF4F1883CB5BD0400C943742C454DF4F06
:109D000028813981CC5BD040232B09F053C080815E
:109D1000882311F40C942640CE0187549F4F0E9453
:109D2000372DC454DF4F99838883CC5BD040CE5409
:109D3000DF4F8881C25BD0408F7091F5C454DF4FF4
:109D40006881CC5BD040CE018F549F4F0E94031B93
:109D5000CF55DF4F2883C15AD040CE55DF4F3883CF
:109D6000C25AD040CD55DF4F4883C35AD040CC555E
:109D7000DF4F5883C45AD040CB55DF4F6883C55A54
:109D8000D040CA55DF4F7883C65AD040C955DF4FFF
:109D90008883C75AD040C855DF4F9883C85AD040EF
:109DA000C454DF4FE881F981CC5BD040EF2B11F434
:109DB0000C9426406CE87BE083E59DE00E94BAF2BB
:109DC0004AE050E0B60183E59DE00E940BF265E8B1
:109DD0007BE083E59DE00E94BAF2D101ED91FC9118
:109DE0006081718183E59DE00E9454F26FE77BE022
:109DF00083E59DE00E94BAF2C754DF4F6881798104
:109E0000C95BD04083E59DE00E9454F26DE77BE0A2
:109E100083E59DE00E94BAF2CE018F549F4F0E94CD
:109E2000D822C754DF4F88819981C95BD040009701
:109E300011F40C947240FC012081243211F00C9436
:109E4000724069E67BE083E59DE00E94BAF283E51B
:109E50009DE00E9404F18CEFA82EBB24BA9452CA54
:109E60002F923F924F925F926F927F928F929F922A
:109E7000AF92CF92DF92EF92FF920F931F93CF9307
:109E8000DF93CDB7DEB76D970FB6F894DEBF0FBE88
:109E9000CDBF009709F4A9C0FC0130853F70353073
:109EA00009F0A3C0D22E1A014B0166807780809101
:109EB0007E0E8F5F80937E0E6114710409F490C052
:109EC000F30180858F70843009F086C061857285CA
:109ED0008091840E9091850E0E94B0C02C01009755
:109EE00009F47AC0FC0180858F70853009F074C058
:109EF000B201CE0101960E94CD3A81149104B1F0D5
:109F0000CE0101960E946D2D882381F0AD2CC12CCD
:109F10007101F401008111812281338144815581D5
:109F200066817781CE0101960E94613F60E0C201A7
:109F30000E9428C10097E9F1FC0120852F70223092
:109F4000C1F581859285A385B4850797A105B105E3
:109F500081F561E0C2010E9428C12D2DA101B4014B
:109F60000E94304F8114910499F5882389F18091E2
:109F70007E0E815080937E0ECE0101960E946F3935
:109F800081E06D960FB6F894DEBF0FBECDBFDF91B6
:109F9000CF911F910F91FF90EF90DF90CF90AF90F6
:109FA0009F908F907F906F905F904F903F902F90F9
:109FB00008958114910461F4CE0101960E946D2DE3
:109FC000882331F0CE0101960E94F74F892B79F654
:109FD000CE0101960E946F39F301628073806CCFCD
:109FE00080917E0E815080937E0E80E0CACFDF92FA
:109FF000EF92FF920F931F93CF93DF9300D000D087
:10A000001F921F92CDB7DEB77C0119821A821B8284
:10A010001C821D821E821F8218868A818F708A830D
:10A02000D701ED91FC916081718183E59DE00E94F3
:10A0300054F268ED7BE083E59DE00E94BAF2C7012F
:10A040000E946D2D81111BC06FEC7BE083E59DE0CC
:10A050000E94BAF283E59DE00E9404F10FEF1FEF2A
:10A06000C80128960FB6F894DEBF0FBECDBFDF91B2
:10A07000CF911F910F91FF90EF90DF900895C7014E
:10A080000E94EB35D82EF70181859285009791F0DB
:10A09000DC01ED91FC910688F789E02D19958C0182
:10A0A00097FD08C081E00115110509F480E00E94C8
:10A0B0001C17D6CFF7018085873009F42EC0EFEF4B
:10A0C000ED0DE43150F5F0E08827E659FF4A8F4F57
:10A0D0000D9471227E5087508D508D5087507E5048
:10A0E0008D508D508D508D508D508D508D507E5097
:10A0F0008D508D508D508D507E507E5060EB7BE0AA
:10A1000083E59DE00E94BAF201E010E0A9CF80E073
:10A110000E941C1710E000E0A3CF40E052E0B7011E
:10A12000CE0101960E94F835D70118968C911897A8
:10A13000873089F160F4833009F457C0843061F0CE
:10A1400060EC7BE083E59DE00E94BAF2E3CF8830CB
:10A1500009F44BC08930A1F760E0CE0101960E945E
:10A16000E91D8C0165EB7BE083E59DE00E94BAF27E
:10A170004AE050E0B80183E59DE00E940BF283E5E0
:10A180009DE00E9404F191E080E0012B09F490E051
:10A19000092F182F65CF1296ED91FC9180858F7055
:10A1A00010E000E08530F1F66DEC7BE083E59DE0AA
:10A1B0000E94BAF220E050E040E070E060E0F70179
:10A1C000828193810E94304FF82E082F10E06AECB4
:10A1D0007BE083E59DE00E94BAF28F2D0E941C1760
:10A1E00083E59DE00E9404F13BCFCE0101960E94E1
:10A1F000511F8B01B7CFAF92CF92EF92FF920F9387
:10A200001F93CF93DF9300D000D01F921F92CDB742
:10A21000DEB719821A821B821C821D821E821F8257
:10A2200018861A811F70A12CCC24C394F12CE12C28
:10A2300002E02B813C8140E05E816F8178850E9445
:10A24000613F28960FB6F894DEBF0FBECDBFDF91F9
:10A25000CF911F910F91FF90EF90CF90AF90089505
:10A260002F923F924F925F926F927F928F929F9226
:10A27000AF92BF92CF92DF92EF92FF920F931F9314
:10A28000CF93DF93CDB7DEB7C255D1090FB6F8949F
:10A29000DEBF0FBECDBF4C013B0140E058E060E0A7
:10A2A00070E00E949D30672B682B692B09F45CC01D
:10A2B00019821A821B821C821D821E821F821886AE
:10A2C0008A818F708A8340E053E0B401CE01019609
:10A2D0000E94F835D40119968D919C91892B09F42F
:10A2E000FBC040E058E060E070E0C4010E944B30E9
:10A2F00065E27CE083E59DE00E94BAF2F40181858D
:10A300009285DC01ED91FC910488F589E02DA12C6A
:10A31000CC24C394F12CE12C09811A812B813C813E
:10A320004D815E816F8178851995D401ED91FC9105
:10A330008F3F9807C9F060817181892B09F036C180
:10A3400083E59DE00E9454F268EE7BE083E59DE0AA
:10A350000E94BAF260EE7BE083E59DE00E94BAF2D3
:10A3600083E59DE00E9404F165E0F4018081918124
:10A370000E9428C15C01009709F450C1DC011896C5
:10A38000BC916196BFAF6197B295BF706096BFAF49
:10A390006097FC0121843284438454840E9426D136
:10A3A0006096FFAD6097FF2309F438C1261A370A7B
:10A3B000480A590A19A21AA21BA21CA2F9A31AA19F
:10A3C0001F70106A1AA32DA23EA24FA258A624E025
:10A3D0006216710449F5D12CC12CE12C50E2F52E06
:10A3E0000F2F2BA13CA14DA15EA16FA178A5C401A7
:10A3F0000E94C130C201B10128EE33E040E050E0DC
:10A400000F941C22BA01A9012AE030E083E59DE007
:10A410000E94C3F165E37DE083E59DE00E94BAF20E
:10A4200083E59DE00E9404F157FEF8C082E0281603
:10A430003104410480E858060CF4F0C00F94DA0EA1
:10A440001B0163967FAF6EAF6397D12CC12CE12CBB
:10A4500040E2F42E09A11AA12BA13CA14DA15EA1BD
:10A460006FA178A5C4010E94C1306396AEADBFADA7
:10A470006397A83CB1050CF0A6C06CE17DE08CEAC6
:10A480009CE00E94BAF24AE050E0B1018CEA9CE004
:10A490000E940BF28CEA9CE00E9404F166246A940C
:10A4A000762CC301CE5ADF4F0FB6F894DEBF0FBE35
:10A4B000CDBFDF91CF911F910F91FF90EF90DF9073
:10A4C000CF90BF90AF909F908F907F906F905F9054
:10A4D0004F903F902F900895F4018085883009F4C3
:10A4E00045C0893019F1843009F03ECF80912409AC
:10A4F00090912509892B09F037CF40E058E060E0C2
:10A5000070E0C4010E944B3060E17CE083E59DE097
:10A510000E94BAF209811A812B813C814D815E81B2
:10A520006F817885C4010E94AD3CFFCE80912409E3
:10A5300090912509892B09F017CF40E058E060E0A1
:10A5400070E0C4010E944B306FEF7BE083E59DE03B
:10A550000E94BAF209811A812B813C814D815E8172
:10A560006F817885C4010E947D3EDFCE80912409F1
:10A5700090912509892B09F0F7CE40E058E060E082
:10A5800070E0C4010E944B306AEE7BE083E59DE001
:10A590000E94BAF209811A812B813C814D815E8132
:10A5A0006F817885C4010E94663DBFCE83E59DE042
:10A5B0000E9454F26EED7BE083E59DE00E94BAF2CA
:10A5C0006AED7BE0C9CEF50180858F7080871982A6
:10A5D0001A821B821C821D821E821F8218868A811B
:10A5E0008F708A836096FFAD6097F98361968FAD17
:10A5F00061978F70AA24A394873009F0A12CCC24F2
:10A60000C394F12CE12C09811A812B813C814D816D
:10A610005E816F817885C4010E94613F21E06216EE
:10A62000710459F4D40118968C91843079F08930F2
:10A6300009F470C1C4010E94F236F401818592854B
:10A64000009709F0A0C4712C612C2BCF80912409B4
:10A6500090912509892BB9F4F40142805380D201ED
:10A6600018968C918F70853041F4C2010E94BAC156
:10A67000082F10E00230110554F464E87CE083E513
:10A680009DE00E94BAF2C4010E94F2360ACF709295
:10A6900025096092240970E060E0C4010E945F2EE9
:10A6A0001C0161E070E0C4010E945F2E5C01053076
:10A6B00011050CF440C064E0C2010E9428C1FC01F5
:10A6C0000185128526E040E855E260E070E087E011
:10A6D0009AE00E94C6F32092F70A87E09AE09093EE
:10A6E000F60A8093F50A1092020C1092040C109254
:10A6F000030C60E77CE083E59DE00E94BAF2D401A0
:10A70000ED91FC916081718183E59DE00E9454F29E
:10A7100083E59DE00E9404F10130110509F4C2C0F7
:10A720006CF4012B09F4B3C064E57CE083E59DE0A3
:10A730000E94BAF225C002E010E0C4CF0230110539
:10A7400079F00330110581F7B092F90AA092F80A66
:10A7500081E090E09093FB0A8093FA0A84E00BC0BA
:10A76000B092F90AA092F80A81E090E09093FB0A77
:10A770008093FA0A83E00E9481D32F968FAF2F97A0
:10A780002F96BFAD2F97B11197C00091FC0A109181
:10A79000FD0A6FE47CE083E59DE00E94BAF2D401FB
:10A7A000ED91FC916081718183E59DE00E9454F2FE
:10A7B00068E47CE083E59DE00E94BAF2C801012EC6
:10A7C000000CAA0BBB0B89839A83AB83BC8380E10B
:10A7D00090E09E838D83BE016F5F7F4F83E59DE098
:10A7E0000E94E33A0E9404F1B801C4010E94D437E8
:10A7F000E0911D09F0911E0962817381CE010196DD
:10A800000E94CD3A80911D0990911E09892BB1F1CA
:10A81000CE0101960E946D2D882381F189858430B7
:10A8200069F570E060E0CE0101960E945F2E281667
:10A83000390621F561E070E0CE0101960E945F2E9D
:10A84000A816B906D9F4B801CE0101960E94D437F2
:10A85000E0911D09F0911E098281938190931E0958
:10A8600080931D09892B51F4E091840EF091850E9F
:10A870008681978190931E0980931D09CE010196D0
:10A880000E946F391092250910922409FCCEB092D3
:10A89000F90AA092F80A81E090E09093FB0A809375
:10A8A000FA0A69CFB092F90AA092F80A1093FB0A4B
:10A8B0000093FA0A82E05FCF6BE37CE083E59DE0E2
:10A8C0000E94BAF2D401ED91FC916081718183E51F
:10A8D0009DE00E9454F263E37CE083E59DE00E94EA
:10A8E000BAF22F96EFAD2F978E2F90E0B0E0A0E058
:10A8F00089839A83AB83BC8380E190E09E838D83C0
:10A90000BE016F5F7F4F83E59DE00E94E33A0E94A6
:10A9100004F1B8CF8091240990912509892B09F081
:10A92000B2CE70922509609224090E94B3F82C01DE
:10A93000009741F0DC0118968C911897807F866013
:10A9400018968C93F20180858F70808730E020E02C
:10A9500043E050E060E2CE0101960F94910DD401E6
:10A96000ED91FC91608171814FE150E0CE01019643
:10A970000F94EE2661EA75E0CE0101960F94C82689
:10A9800026E040E855E260E070E087E09AE00E944F
:10A99000C6F370E060E0C4010E945F2E8093F70A66
:10A9A00087E09AE09093F60A8093F50A1092020CE1
:10A9B0001092040C1092030C6CE07DE083E59DE0A6
:10A9C0000E94BAF2D401ED91FC916081718183E51E
:10A9D0009DE00E9454F283E59DE00E9404F162E351
:10A9E00070E080E090E00E94F3D084E398E09093E0
:10A9F000F90A8093F80A8AE090E09093FB0A80932A
:10AA0000FA0A83E00E9481D3182F811154C26FEF9C
:10AA10007CE083E59DE00E94BAF20CEF1AE090E141
:10AA2000292E9BE0392E20E1A22EB12CF801819134
:10AA300091918F01092E000CAA0BBB0B89A39AA33D
:10AA4000ABA3BCA3BEA2ADA2BE016F5D7F4F83E5E9
:10AA50009DE00E94E33A6DEF7CE00E94BAF220167E
:10AA6000310621F783E59DE00E9404F16091000B1F
:10AA70007091010B90E080E00F94B72020E030E06F
:10AA800048EC52E40F9410239B01AC0167EA76E096
:10AA9000C2010E94A6CAC090040BD090050BF12CF5
:10AAA000E12CA701960167EA75E0C2010E94DAC5B0
:10AAB0006091060B7091070B90E080E00F94B72037
:10AAC00020E030E048EC52E40F9410239B01AC01ED
:10AAD0006BEA75E0C2010E94A6CA6091080B7091F2
:10AAE000090B90E080E00F94B72020E030E040E2D6
:10AAF00051E40F9410239B01AC0169EA75E0C20197
:10AB00000E94A6CA2091FC0A3091FD0A50E040E064
:10AB10006DEA75E0C2010E94DAC5CD28CE28CF28A3
:10AB200009F47AC0D4011296ED91FC9190859F7042
:10AB3000953009F071C061E0CF010E9428C10097F3
:10AB400009F46AC0FC0120852F70243009F064C02C
:10AB500061857285CE0181960E94E338CE0181968F
:10AB60000E946D2D882309F453C022961CAE1DAEA1
:10AB70001EAE1FAE229726961CAE1DAE1EAE1FAE99
:10AB800026978FAD8F7080618FAF8FEF23968FAF39
:10AB9000239724965FAD249725963FAD259726965B
:10ABA0002FAD26979EAD7FAD21966FAD2197229652
:10ABB0004FAD2297092F27969FAF279728967FAFF3
:10ABC000289729966FAF29972A964FAF2A97482F33
:10ABD0002B968FAF2B972C965FAF2C972D963FAF70
:10ABE0002D972E962FAF2E97A12CCC24C394F12C09
:10ABF000E12C172F262F2A963FAD2A972D966FAD61
:10AC00002D972E967FAD2E97CE0181960E94613FA3
:10AC1000CE0181960E946F398091FC0A83FF76C134
:10AC200062ED7CE083E59DE00E94BAF2D401ED91F3
:10AC3000FC916081718183E59DE00E9454F283E57F
:10AC40009DE00E9404F162E370E080E090E00E94E9
:10AC5000F3D08EE398E09093F90A8093F80A81E0AC
:10AC600090E09093FB0A8093FA0A83E00E9481D3DC
:10AC700081110BC02091FC0A3091FD0A50E040E0A8
:10AC800060EB75E0C2010E94DAC5109225091092AE
:10AC90002409C4010E94F74F181619061CF4C401B8
:10ACA0000E94FB5081E090E0909325098093240955
:10ACB00062EC7CE083E59DE00E94BAF2D401ED9164
:10ACC000FC916081718183E59DE00E9454F283E5EF
:10ACD0009DE00E9404F162E370E080E090E00E9459
:10ACE000F3D083E190E09093F90A8093F80A84E02E
:10ACF00090E09093FB0A8093FA0A83E00E9481D34C
:10AD0000182F811115C165EB7CE083E59DE00E9461
:10AD1000BAF20CEF1AE084E0E82E8BE0F82EF8018E
:10AD2000619171918F014AE050E083E59DE00E94BE
:10AD30000BF263EB7CE083E59DE00E94BAF2E01643
:10AD4000F10669F783E59DE00E9404F10091FC0A99
:10AD50001091FD0A01151105D1F0B801012E000C6A
:10AD6000880B990B0F94B7202DEE3EE94CE35EE380
:10AD70000F94162122E538EB42E152E40F94A3220E
:10AD80009B01AC0164EB75E0C2010E94A6CA609110
:10AD9000FE0A7091FF0A072E000C880B990B0F9486
:10ADA000B7202DEE3EE94CE35EE30F94162122E539
:10ADB00038EB42E152E40F94A3226B017C01AC0119
:10ADC0009B0165EA75E0C2010E94A6CA6091020B70
:10ADD0007091030B161617060CF0A1C0072E000C7D
:10ADE000880B990B0F94B72020E030E040E251E44B
:10ADF0000F9410239B01AC0168EB75E0C2010E9427
:10AE0000A6CA20E030E040E252E4C701B6010F9448
:10AE1000B8231816B4F4012BA1F00E94CEC08823E9
:10AE200069F08091690E811109C0D401ED91FC9106
:10AE3000608171818CEB95E00E940FD2C4010E9469
:10AE4000FB5080E091E00F9482188C01892BD9F09F
:10AE50001CA21BA21EA21DA28FEF9FEF98A78FA37B
:10AE600085EA92E09AA389A31AA619A61CA70BA7A4
:10AE700080E091E098AB8FA71EA61DA6B201CE017F
:10AE800081960E94A3F60E94CEC0882349F080914B
:10AE9000690E811105C0B801CE0101960E940FD242
:10AEA000C8010F941E194114510409F4EBCCC201DE
:10AEB0000E947ACAE7CC60EF7CE083E59DE00E94C7
:10AEC000BAF2D401ED91FC916081718183E59DE03E
:10AED0000E9454F268EE7CE083E59DE00E94BAF2A5
:10AEE000812F90E0B0E0A0E089A39AA3ABA3BCA31C
:10AEF00080E190E09EA38DA3BE016F5D7F4F83E54F
:10AF00009DE00E94E33A0E9404F186CE20E030E00A
:10AF1000A90160EB75E0C2010E94DAC5C9CE20E04C
:10AF200030E0A90168EB75E0C2010E94DAC569CF83
:10AF300063EA7CE083E59DE00E94BAF2D401ED91E2
:10AF4000FC916081718183E59DE00E9454F26BE980
:10AF50007CE083E59DE00E94BAF2812F90E0B0E0B2
:10AF6000A0E089A39AA3ABA3BCA380E190E09EA339
:10AF70008DA3BE016F5D7F4F83E59DE00E94E33AA4
:10AF80000E9404F15ECFDC01ED91FC910284F38517
:10AF9000E02D1995892B09F456CBF4018185928512
:10AFA000DC01ED91FC910480F581E02DB301199550
:10AFB0003C0177CA2F923F924F925F926F927F929D
:10AFC0008F929F92AF92BF92CF92DF92EF92FF92B9
:10AFD0000F931F93CF93DF93CDB7DEB7C657D10939
:10AFE0000FB6F894DEBF0FBECDBFDC0114962D91D5
:10AFF0003C91232B11F40C94EE613B014C01FC01BC
:10B0000082819B01225031092230310508F017C698
:10B01000803409F4F7C208F04AC0843008F085C2D1
:10B020008091D5088F5F8093D508A3016FEFC4018D
:10B030000E944C1BD40112960C9112970695017038
:10B0400013961C9113978AEC810F803108F043C04E
:10B0500069EC75E08D919C910E94B0C07C010097D5
:10B06000D1F1FC0180858F708530A9F58091920D1A
:10B07000181324C08091930D803401F58091940DB4
:10B080009091950D5C01990FCC08DD0860E0C70137
:10B090000E9428C1FC0181859285A385B485A816EC
:10B0A000B906CA06DB060CF065C0512C3EC08234DE
:10B0B00009F4A8C208F439C28058AFCF1093920D9A
:10B0C00080E48093930D812F0E94BECF9093950DC5
:10B0D0008093940DD7CF212F30E0F901EE5DF74D2D
:10B0E0008491F901E452F84D1491F901EA56F84DB2
:10B0F000F490FF2009F43BC081110E9416CEEF2D81
:10B10000F0E0EE0FFF1FEF52F54DA591B491EC91D9
:10B110001E2331E020E009F430E0832F922F5524E4
:10B1200053940817190609F0C0CFF3E06F167104A5
:10B1300009F488C0D4011496ED91FC91E181EF707F
:10B14000E150EC3008F07EC0F0E08827E555F74A82
:10B150008F4F0D947122CC58485A02593859485A89
:10B160005159485A8559B259CB590D5A2F5A90E026
:10B1700080E0D5CF61E0C7010E9428C155245394D7
:10B18000FC0181859285A385B4858A159B05AC0554
:10B19000BD050CF0CACF89CF0E9426D19B01AC011E
:10B1A00044275527D4011496ED91FC916281738157
:10B1B00090E080E0AA24AA94BA2CC12CD12C18EEDD
:10B1C000E12E13E0F12E00E010E00F94720C8823C2
:10B1D000C9F1F401008111816FE175E0C8010E949D
:10B1E000B0C0892B41F464E275E0C8010E94B0C090
:10B1F000892B09F40EC142E050E063E0C4010E94D3
:10B200004C1B20C00E9426D19B01AC01442755272E
:10B21000D4011496ED91FC916281738190E080E0FD
:10B22000AA24AA94BA2CC12CD12C1CE2E12EFF2412
:10B23000F39400E010E00F94720C42E050E064E000
:10B24000811184C0D4011496ED91FC91808183FB1F
:10B25000992790F9951509F4D2C1982F907E09F499
:10B2600039C1982F907E90528F71892B808358C15D
:10B270000E9426D19B01AC0144275527D401149686
:10B28000ED91FC916281738190E080E0AA24AA9400
:10B29000BA2CC12CD12C16E9E12EF12C00E010E0E3
:10B2A000CACF0E9426D19B01AC0144275527D40167
:10B2B0001496ED91FC916281738190E080E0AA2464
:10B2C000AA94BA2CC12CD12C18EEE12E13E0F12E49
:10B2D00000E010E00F94720C882309F4B3CFF4015E
:10B2E000008111816AE275E0C8010E94B0C0892B1B
:10B2F00041F460E375E0C8010E94B0C0892B09F4F5
:10B3000088C042E050E068E079CF0E9426D19B01DE
:10B31000AC0144275527D4011496ED91FC9162812C
:10B32000738190E080E0AA24AA94BA2CC12CD12C7D
:10B330001CE2E12EFF24F39400E010E00F94720C65
:10B3400042E050E069E0882309F47CCFC4010E9408
:10B350004C1B0E9426D1D4011496ED91FC9173836D
:10B36000628370CF0E9426D19B01AC0144275527F0
:10B37000D4011496ED91FC916281738190E080E09C
:10B38000AA24AA94BA2CC12CD12C16E9E12EF12CB6
:10B3900000E010E0D3CF0E9426D19B01AC014427EE
:10B3A0005527D4011496ED91FC916281738190E050
:10B3B00080E0AA24AA94BA2CC12CD12C18EEE12E3C
:10B3C00013E0F12E00E010E00F94720C882309F4D2
:10B3D00039CFF4010081118167E375E0C8010E9453
:10B3E000B0C0892B39F46DE375E0C8010E94B0C08C
:10B3F000892B21F042E050E06BE000CF69E175E07D
:10B40000C8010E94B0C042E050E066E0892B09F418
:10B41000F5CE42E050E06DE0F1CE0E9426D19B01D6
:10B42000AC0144275527D4011496ED91FC9162811B
:10B43000738190E080E0AA24AA94BA2CC12CD12C6C
:10B440001CE2E12EFF24F39400E010E00F94720C54
:10B45000882309F4F7CE42E050E06CE077CF0E94F9
:10B4600026D19B01AC0144275527D4011496ED91B8
:10B47000FC916281738190E080E0AA24AA94BA2CA6
:10B48000C12CD12C16E9E12EF12C00E010E0DECF2A
:10B490000E9426D19B01AC0144275527D401149664
:10B4A000ED91FC916281738190E080E0AA24AA94DE
:10B4B000BA2CC12CD12C18E5E12E12E0F12E00E0BF
:10B4C00010E00F94720C882309F4BCCE42E050E0E7
:10B4D00060E094CE0E9426D1D4011496ED91FC91A7
:10B4E000159773836283E181EF70552009F445C09D
:10B4F000E230F1F050F4EE23E9F1D4011496ED912D
:10B50000FC91808150FA83F9B1CEE53089F0A30136
:10B510006AE0E73091F7C4010E944C1B8111EDCF26
:10B520008091D50881508093D50890E080E058C77D
:10B53000F4010081118163E175E0C8010E94B0C08F
:10B54000892BA9F46AE275E0C8010E94B0C0892B7A
:10B5500071F460E375E0C8010E94B0C0892B39F432
:10B560006BEF74E0C8010E94B0C0892B19F0A301F1
:10B5700066E0D1CFA30161E0CECFE150ED3008F01D
:10B58000BCCFF0E08827E853F54A8F4F0D94712225
:10B59000D55A7D5AD85AD85A7D5ADB5A7D5AFC5A08
:10B5A000FC5AFC5AFC5AFC5AD85AA30162E0B3CFA9
:10B5B000A30165E0B0CF0D911C9163E175E0C80176
:10B5C0000E94B0C0892BA9F46AE275E0C8010E940C
:10B5D000B0C0892B71F460E375E0C8010E94B0C06F
:10B5E000892B39F46BEF74E0C8010E94B0C0892B3D
:10B5F00019F0A30167E08FCFA30160E08CCF8F71BA
:10B60000806434CEB3E06B16710409F48ECF69EC1C
:10B6100075E0F401808191810E94B0C08C01D40159
:10B6200013968C919091920D8913E5C09091930D92
:10B63000903409F0E0C08091940D9091950D3C01FB
:10B640000115110509F404C1F80120852F7025307A
:10B6500009F0FEC0C8010E94BAC1A7968FAFA79794
:10B66000843008F4D4C063E0C8010E9428C1DC0122
:10B6700019968D919C912AE0F22EF89E5001F99E28
:10B68000B00C112462E0C8010E9428C1FC01818530
:10B690009285F89E1001F99E300C11246101032C53
:10B6A000000CEE08FF08E796CCAEDDAEEEAEFFAEC6
:10B6B000E79761E0C8010E9428C12C0160E0C80141
:10B6C0000E9428C1DC011996CD90DD90ED90FC9090
:10B6D0001C97AB96CCAEDDAEEEAEFFAEAB97930152
:10B6E000072C000C440B550B2C193D094E095F0922
:10B6F000B5010B2C000C880B990BE796CCACDDAC9C
:10B70000EEACFFACE7976C197D098E099F090F9489
:10B71000EA21D20119962D913D914D915C911C9792
:10B72000AB96CCACDDACEEACFFACAB972C193D09C5
:10B730004E095F09AB962CAF3DAF4EAF5FAFAB97F5
:10B740000F941C22E796CCACDDACEEACFFACE797D7
:10B75000C20ED31EE41EF51EA7962FADA797253067
:10B7600009F465C081E090E0A5010B2C000C660B8C
:10B77000770B4C155D056E057F050CF461C0B701B4
:10B78000A6016101032C000CEE08FF084C155D05B5
:10B790006E057F050CF459C06A017B01A796BFAD09
:10B7A000A797B23009F065C06301770CEE08FF0877
:10B7B00060E0C8010E9428C1FC0181859285A385B3
:10B7C000B485C816D906EA06FB060CF423C661E068
:10B7D000C8010E9428C1FC0181859285A385B4859A
:10B7E0008C159D05AE05BF050CF09FCE81E090E065
:10B7F000A0E0B0E012C68093920D90E49093930D78
:10B800000E94BECF9093950D8093940D18CF8AE03F
:10B81000869D6001879DD00C11240D2C000CEE0834
:10B82000FF08312C212CA12C88E2B82E9BCF64E09C
:10B83000C8010E9428C1DC0119968D919C9194CF7A
:10B8400066246A94B3E07B2E9CCF712C612CA6CF2A
:10B850002AE0289F6001299FD00C11240D2C000C98
:10B86000EE08FF08312C212CA12CA8E2BA2E81E091
:10B8700090E0D4011496ED91FC9162817381A30153
:10B88000461B570B57FF03C051954195510984172B
:10B8900095070CF4C0C08081982F9295969597706B
:10B8A000963008F0BBC09F5F9295990F907E8F7184
:10B8B000892BB3C0F20161857285DB018C91811106
:10B8C0003DC60115110509F457C0D80118968C9191
:10B8D00018978F70843009F04FC019966D917C9144
:10B8E000CE0101960E94E338CE0101960E946D2D93
:10B8F0008823F1F12114310409F460C0411451048A
:10B9000031F0F20180858F70843009F44CC02596A7
:10B910001CAE1DAE1EAE1FAE259729961CAE1DAEE9
:10B920001EAE1FAE299723961FAD23971F70239637
:10B930001FAF239781E022968FAF2297A12CCC24B2
:10B94000C394F12CE12C01E024962FAD2497259689
:10B950003FAD259740E027965FAD279728966FADBE
:10B96000289729967FAD2997CE0101960E94613FC5
:10B97000CE0101960E946F39D4011496ED91FC918D
:10B9800033822282D2CD6114710429F0F3018085C3
:10B990008F70843019F069E876E0D0C561857285D2
:10B9A000FB0180818CCF61857285FB0180818823BA
:10B9B000F9F2CE0101960E94E1C7DACF6114710459
:10B9C00031F0D30118968C918F708430F1F0259668
:10B9D0001CAE1DAE1EAE1FAE259729961CAE1DAE29
:10B9E0001EAE1FAE299723961FAD23971F70239677
:10B9F0001FAF239782E022968FAF2297A12CCC24F1
:10BA0000C394F12CE12C02E09FCFF3016185728594
:10BA1000DB018C91CCCF80818F7180838081803AD3
:10BA200098F0C101330CAA0BBB0B8C159D05AE051C
:10BA3000BF0551F0C501BB0CAA0BBB0B8C159D05B6
:10BA4000AE05BF0509F071CD6615770509F46DCD1A
:10BA5000A2961CAE1DAE1EAE1FAEA297A0968FADD5
:10BA6000A0978F708066A0968FAFA097A2968CAD9E
:10BA70009DADAEADBFADA29768968CAF9DAFAEAF9A
:10BA8000BFAF6897AAE0B0E0A70196010F943B22F0
:10BA90006C966CAF7DAF8EAF9FAF6C9764E678E02D
:10BAA00083E59DE00E94BAF24AE050E0F401638130
:10BAB00083E59DE00E9421F162E678E083E59DE068
:10BAC0000E94BAF2CE018C5A9F4F0E94D8226DEC90
:10BAD00075E0D4018D919C910E94B0C0B12CA12C35
:10BAE000D12CC12C6596EFAC65976696FFAC669736
:10BAF00067960FAD679768961FAD689769962FADEB
:10BB000069976A963FAD6A976B964FAD6B976C9647
:10BB10005FAD6C976FEF0F949610F4010081118167
:10BB200064E475E0C8010E94B0C07C0169E475E07E
:10BB3000C8010E94B0C08C010097F1F1DC01189699
:10BB40008C9118978F708430B9F519966D917C910E
:10BB500040E450E0CE0101960F940C276FE270E0B4
:10BB6000CE0101960F94D326892B51F4F80121853B
:10BB7000328543E050E060E4CE0101960F94910DD0
:10BB800000E020E032E040E150E0BE016F5B7F4F1B
:10BB9000CE018C5A9F4F0E94B7200E94CEC08823AE
:10BBA00059F08091690E811107C0BE016F5B7F4F14
:10BBB000CE0101960E94F4D1E114F104C9F1D7013C
:10BBC00018968C9118978F70843091F519966D9115
:10BBD0007C91CE0101960E94E338CE0101960E942D
:10BBE0006D2D882309F1A12CCC24C394F12CE12CD8
:10BBF00065960FAD659766961FAD669767962FADF4
:10BC0000679768963FAD689769964FAD69976A9652
:10BC10005FAD6A976B966FAD6B976C967FAD6C97C7
:10BC2000CE0101960E94613FCE0101960E946F39BC
:10BC3000D4011496ED91FC917382628276CC8830A7
:10BC400009F49BC2803109F488C3843009F06DCCBB
:10BC50000E9426D12B013C01C4010E942A16A12C6E
:10BC6000B12C650118E9E12E1AE3F12E00E010E095
:10BC7000A30192010F94720C882309F456CCF401AD
:10BC8000838127968FAF279796E128969FAF2897B5
:10BC9000282F30E0F901E452F84DE4912996EFAFF6
:10BCA0002997F901EA56F84DE4912A96EFAF2A97C1
:10BCB00040E85EE360E070E062964CAF5DAF6EAF6F
:10BCC0007FAF629762E00E94ABCE0E9426D1605D9A
:10BCD0007740810991092E966CAF7DAF8EAF9FAFF3
:10BCE0002E9787E364968FAF6497CE018F5B9F4F4B
:10BCF0000E947DD2882349F028968FAD28978C30FA
:10BD000009F46FC048F48B3011F1412C512C60ECD8
:10BD1000662E6FE7762E47C085518230B0F72496A5
:10BD20001FAD2497612F70E0762F662766277F77F7
:10BD300025968FAD2597682B90E080E00F94B52075
:10BD40002DEC3CEC4CEC5DE30F94162168C024967E
:10BD50006FAD249770E090E080E00F94B5206B0108
:10BD60007C0125961FAD259717FF0AC0AC019B01EA
:10BD700060E070E080E89FEB0F94A3226B017C01F0
:10BD80001F70612F70E090E080E00F94B7202DECE1
:10BD90003CEC4CEC5DE30F941621A70196010F9447
:10BDA000A4222B013C01CE018F5B9F4F0E947DD2CC
:10BDB000882309F4D7C128968FAD28978B3030F0AF
:10BDC0008D30B0F18551823008F4BAC1312C212C6C
:10BDD00030ECA7963FAFA7974FE7A8964FAFA8972D
:10BDE0004DC024961FAD2497612F70E090E080E055
:10BDF0000F94B5206B017C0125966FAD25976F7070
:10BE000070E090E080E00F94B7202DEC3CEC4CEC1F
:10BE10005DE30F941621A70196010F94A4222B0134
:10BE20003C0117FFC0CF77FA709477F87094BBCFBE
:10BE300023966FAD239770E090E080E00F94B720D9
:10BE40002DEC3CEC4CEC5DE30F9416216B017C0176
:10BE500022966FAD229770E090E080E00F94B720BB
:10BE60009B01AC01C701B6010F94A422362E272EE8
:10BE7000A7968FAFA797A8969FAFA8976EE878E090
:10BE800083E59DE00E94BAF24AE050E0D4011396A7
:10BE90006C9183E59DE00E9421F16EE778E083E5F7
:10BEA0009DE00E94BAF2B301A20183E59DE00E94E9
:10BEB0006CC667E778E083E59DE00E94BAF2432D07
:10BEC000522DA7966FADA797A8967FADA89783E54B
:10BED0009DE00E946CC665E778E083E59DE00E94E6
:10BEE000BAF283E59DE00E9404F1F4010081118122
:10BEF00061ED75E0C8010E94B0C0AD969FAF8EAFF6
:10BF0000AD9766ED75E0C8010E94B0C0AF969FAFD7
:10BF10008EAFAF97A3019201C301B2010F94182411
:10BF200081111FC019821A821B821C828A818F7024
:10BF30008067F82E8A83242D4D825E826F827886F8
:10BF4000B12CA12CD12CC12CE9800B811C813E810C
:10BF50004F8158856FEFAD968EAD9FADAD970F9425
:10BF60009610232D322DA7964FADA797A8965FADBB
:10BF7000A897632D722DA7968FADA797A8969FAD12
:10BF8000A8970F941824811127C019821A821B8246
:10BF90001C828A818F708067F82E8A83232D832DDF
:10BFA000922DA796AFADA797A896BFADA8978D8302
:10BFB0009E83AF83B887B12CA12CD12CC12CE980F2
:10BFC0000B811C813E814F8158856FEFAF968EADFE
:10BFD0009FADAF970F94961069E475E0D4018D91F1
:10BFE0009C910E94B0C07C01009709F4A1C0FC01A3
:10BFF00080858F70843009F09BC020E030E0A9017B
:10C00000C301B2010F94B020882309F491C020E04D
:10C0100030E0A901632D722DA7968FADA797A89642
:10C020009FADA8970F94B020882309F481C0A30185
:10C030009201C301B2010F94B020811179C0232D68
:10C04000322DA7964FADA797A8965FADA897632D01
:10C05000722DA7968FADA797A8969FADA8970F941E
:10C06000B020811165C01A821982FE0133968EE3D9
:10C07000DF011D928A95E9F7F7016185728540E439
:10C0800050E08E010F5F1F4FC8010F940C276FE225
:10C0900070E0C8010F94D326892B51F4D70119966B
:10C0A0002D913C9143E050E060E4C8010F94910D64
:10C0B0006AED75E0C8010F94C826B301A201CE0154
:10C0C0008C5A9F4F0F94810E0E94CEC0882351F04E
:10C0D0008091690E811106C0BE016C5A7F4FC80164
:10C0E0000E940FD2F80101900020E9F73197E01B80
:10C0F000F10BEC0FFD1F88E48083432D522DA79692
:10C100006FADA797A8967FADA897CE018C5A9F4F89
:10C110000F94810E0E94CEC0882351F08091690E49
:10C12000811106C0BE016C5A7F4FC8010E940FD218
:10C130000E9426D1AB01BC01C4010E940316F5C9BF
:10C1400023966EAD7FAD239776276727762790E0FD
:10C1500080E00F94B5202DEC3CEC4CEC5DE30F94AB
:10C16000162184CE312C212CF0ECA796FFAFA79797
:10C170002FE7A8962FAFA89781CE0E9426D12B013A
:10C180003C01C4010E942A16A12CB12C650118E9BA
:10C19000E12E1AE3F12E00E010E0A30192010F94CA
:10C1A000720C882309F4C1C9D4011496ED91FC9155
:10C1B0001597818113961C91811157C0163008F094
:10C1C0003FC08CE0EAE2F2E0DE01119601900D92B0
:10C1D0008A95E1F7E12FF0E0EE0FFF1FCC24C39426
:10C1E000D12CCC0EDD1EEC0DFD1D60E080810E9487
:10C1F000ABCE6AE776E183E01330C9F070F462E811
:10C2000076E181E0113099F06EE776E182E012305C
:10C2100071F066E876E180E00AC066E776E184E0E6
:10C22000143029F062E776E185E0153091F70E943D
:10C2300017C6D4011496ED91FC9181E0818375C9F4
:10C2400066EE78E083E59DE00E94BAF24AE050E0B5
:10C25000F401638183E59DE00E9421F169EB78E0C0
:10C2600083E59DE00E94BAF260C924E0129FF001CC
:10C270001124EA52F74FC080D180E280F38065EB51
:10C2800078E083E59DE00E94BAF24AE050E0D401F4
:10C2900013966C9183E59DE00E9421F161EA78E0BC
:10C2A00083E59DE00E94BAF22AE030E0B701A601E2
:10C2B00083E59DE00E94C3F169E475E0F4018081AB
:10C2C00091810E94B0C08C01009709F443C0DC0149
:10C2D00018968C9118978F708430E1F519966D91AE
:10C2E0007C9140E450E0CE0101960F940C276FE260
:10C2F00070E0CE0101960F94D326892B51F4F801FA
:10C300002185328543E050E060E4CE0101960F9430
:10C31000910DFF92EF92DF92CF9285E595E09F938A
:10C320008F938E010F5B1F4F1F930F930F94632703
:10C330000E94CEC00FB6F894DEBF0FBECDBF8823DB
:10C3400009F4F6CE8091690E8111F2CEB801CE01CA
:10C350000196ECCE62E978E083CF0E9426D12B01D2
:10C360003C01C4010E942A16A12CB12C650110E3E6
:10C37000E12E15E7F12E00E010E0A30192010F94E9
:10C38000720C882309F4D1C869E475E0D4018D9159
:10C390009C910E94B0C08C01009709F4C9CEFC01A9
:10C3A00080858F70843009F0C3CE0E9426D12AE0A8
:10C3B000AE014F5F5F4F0F945F1B0E94CEC088237A
:10C3C00009F4B6CE8091690E8111B2CEBE016F5FC5
:10C3D0007F4FD80119968D919C91A8CE8FEF9FEF3A
:10C3E000CA58DF4F0FB6F894DEBF0FBECDBFDF9146
:10C3F000CF911F910F91FF90EF90DF90CF90BF9062
:10C40000AF909F908F907F906F905F904F903F90F4
:10C410002F90089580E090E0DC01F40124813581C3
:10C42000F90142815381052E000C660B770B4817EA
:10C4300059076A077B0709F478C81C01D4016D907D
:10C440007C9064E475E0C3010E94B0C08C0169E493
:10C4500075E0C3010E94B0C07C010115110519F4FB
:10C46000892B09F489CA6EE075E0C3010E94B0C04F
:10C470002C0169E075E0C3010E94B0C03C016AE68E
:10C4800078E083E59DE00E94BAF24AE050E0F401D2
:10C49000638183E59DE00E9421F168E678E083E511
:10C4A0009DE00E94BAF24AE050E0B10183E59DE0D0
:10C4B0000E940BF283E59DE00E9404F1E114F10477
:10C4C00009F4FFC9D70118968C9118978F708430A2
:10C4D00009F0F7C919966D917C9140E450E0CE01C6
:10C4E00001960F940C270E94CEC0882309F4E9C955
:10C4F0008091690E8111E5C96FE270E0CE0101966D
:10C500000F94D326892B51F4F7012185328543E01E
:10C5100050E060E4CE0101960F94910D2114310496
:10C5200009F431CA4114510439F0D20118968C91A2
:10C530008F70843009F4BEC96EE776E0CE010196B3
:10C540000E94F4D1BEC9EF92FF920F931F93CF9335
:10C55000DF93EC018B011D821C821A821B82E88012
:10C56000F980E114F10409F45DC080911F099091F4
:10C570002009892B09F456C0672B09F48701F801BB
:10C5800080858F708630A9F46AED75E0C8010E943D
:10C59000B0C0009719F0FC0181858A8363E376E0DF
:10C5A000C8010E94B0C0009709F443C0FC01818516
:10C5B0008B836CED75E0C7010E94B0C0009779F5E0
:10C5C0006DE578E083E59DE00E94BAF24AE050E034
:10C5D0006B8183E59DE00E9421F16BE578E083E5C6
:10C5E0009DE00E94BAF24AE050E06A8183E59DE056
:10C5F0000E9421F183E59DE00E9404F120E030E0FB
:10C60000A9016CED75E0888199810E94DAC56CED15
:10C6100075E0888199810E94B0C0009719F0099651
:10C620009D838C83DF91CF911F910F91FF90EF90AD
:10C630000895F801808191810F944F1AB9CFAF927C
:10C64000BF92CF92DF92EF92FF920F931F93CF93FF
:10C65000DF9364E070E041E050E00091D108109178
:10C66000D2082091D3083091D408CA01052E000CBD
:10C67000AA0BBB0B80239123A223B323892B8A2BE4
:10C680008B2BD9F0C090D108D090D208E090D3087D
:10C69000F090D408CA0180959095092E000CAA0B41
:10C6A000BB0B8C219D21AE21BF218093D10890939B
:10C6B000D208A093D308B093D408440F551F6150FB
:10C6C000710959F68091CD089091CE08A091CF08BC
:10C6D000B091D008892B8A2B8B2B09F47DC00E9446
:10C6E00026D19B01AC016091CD087091CE0880915C
:10C6F000CF089091D008A12CB12C65011CE2E12E4D
:10C70000FF24F39400E010E00F94720C882309F4E6
:10C7100063C01092CD081092CE081092CF081092EC
:10C72000D0088091150990911609892B09F183E0B1
:10C73000E82EF12CD0E0C0E0E0911509F091160947
:10C74000EE0DFF1D008110E0DF0111972C9130E00C
:10C7500011974C9150E03397608170E0CE010E94B8
:10C76000571984E0E80EF11C2196C430D10521F759
:10C77000C1E0D0E080911C0290911D028C179D07B2
:10C7800048F580911C0290911D02E0917C0EF09181
:10C790007D0EE80FF91F4AE050E0608183E59DE0DF
:10C7A0000E9421F16FED75E083E59DE00E9454F257
:10C7B0002196C131D105F1F683E59DE0DF91CF915E
:10C7C0001F910F91FF90EF90DF90CF90BF90AF90AF
:10C7D0000C9404F1CE01D9CFDF91CF911F910F912D
:10C7E000FF90EF90DF90CF90BF90AF9008954F9261
:10C7F0005F926F927F92AF92BF92CF92DF92EF9251
:10C80000FF920F931F93CF93DF93CDB7DEB76D9752
:10C810000FB6F894DEBF0FBECDBF20911F09309137
:10C820002009FF24F394232B09F420C1811149C06E
:10C83000FF24F3946AEB71E183E59DE00E94BAF274
:10C8400083E59DE00E9404F180910C098F5F809345
:10C850000C09E091840EF091850E309709F48DC09B
:10C86000068117810115110509F491C0D8011896A8
:10C870008C918F70853009F5C8010E94BAC1882358
:10C88000E1F0F80160817181CE0101960E94E338E8
:10C89000CE0101960E946D2D882359F08A859B85D3
:10C8A000009739F0DC01ED91FC910084F185E02DD9
:10C8B0001995CE0101960E946F39F801028113810A
:10C8C000D1CF63EF71E183E59DE00E94BAF283E589
:10C8D0009DE00E9404F10E9426D12B013C01809131
:10C8E0007E0E882381F10E9426D19B01AC01A12CF0
:10C8F000B12C650110E1E12E17E2F12E00E010E00D
:10C90000C301B2010F94720C81111DC00E94E6F5A3
:10C910008091880E811128C00E941F638091820E31
:10C920009091830E059741F08091840E9091850E31
:10C93000892B11F00E9447AB0E9413AC82E090E07B
:10C940000E946CA4CCCF80917E0E882309F470CF16
:10C9500060ED71E18CEA9CE00E94BAF28CEA9CE006
:10C960000E9404F1F12C66CF8091860E9091870E83
:10C97000892B91F20E948FA1CFCF6AEA71E183E502
:10C980009DE00E94BAF283E59DE00E9404F11092BE
:10C990001E0910921D0962EA71E183E59DE00E9483
:10C9A000BAF283E59DE00E9404F164E670E080E065
:10C9B00090E00E94F3D01092260910921C096AE8B8
:10C9C00071E183E59DE00E94BAF20F94DA0EAB01AB
:10C9D000BC012AE030E083E59DE00E941FF18091D8
:10C9E0001F0990912009009711F00E947ACA1092B5
:10C9F000200910921F091092810E1092800E109241
:10CA0000850E1092840E1092680E1092670E10928E
:10CA10001A09109219091092660E1092650E109262
:10CA20001809109217091092870E1092860E109214
:10CA300023091092220965E871E183E59DE00E94D7
:10CA4000BAF20F94DA0EAB01BC012AE030E083E5C4
:10CA50009DE00E941FF183E59DE00E9404F1109289
:10CA60001B0980910C09815080930C098F2D6D96C4
:10CA70000FB6F894DEBF0FBECDBFDF91CF911F91EF
:10CA80000F91FF90EF90DF90CF90BF90AF907F908D
:10CA90006F905F904F900895FC016115710519F436
:10CAA00084819581089586819781681779072CF094
:10CAB00084819581860F971F0895828193810C94BC
:10CAC0005F2E4F925F926F927F928F929F92AF9262
:10CAD000BF92CF92DF92EF92FF920F931F93CF936B
:10CAE000DF93CDB7DEB7CD52D1400FB6F894DEBF9D
:10CAF0000FBECDBF2091820E3091830EF9013B967F
:10CB0000EB31F10508F0A0C68827E657FA498F4FA8
:10CB10000D947122DD72D072246C246C246C246C10
:10CB2000246C246C246C246C246CA565B56DBC6DE0
:10CB3000C86D166ECC71CB72246C246C246C246C82
:10CB4000246CFC7258737F7372738091BF0A809358
:10CB5000B20A8091010281110E94F2F960E08EE236
:10CB600090E00E94D3F980FF6FC685EC94E0CC5D25
:10CB7000DE4F99838883C452D140CA5DDE4F18824C
:10CB800019821A821B82C652D140C25EDE4F99833F
:10CB90008883CE51D140C05EDE4F188219821A823E
:10CBA0001B82C052D140C85EDE4F99838883C85132
:10CBB000D140C65EDE4F188219821A821B82CA518A
:10CBC000D140CE5EDE4F99838883C251D140CC5E86
:10CBD000DE4F188219821A821B82C451D14067EA43
:10CBE00073E182EA9CE00E94BAF282EA9CE00E9431
:10CBF00004F180917E0C90917F0C8E010F571F4F96
:10CC0000892B09F46FC00E94E8C1882309F46AC027
:10CC1000A0917E0CB0917F0C52961C921E9251975F
:10CC200054961C921E92539784E890E01D969C9314
:10CC30008E931C971E961C921E9782E755968C9396
:10CC40005597ED91FC9111970088F189E02D60E1F5
:10CC500070E0CD011995BE016F5F7F4F80917E0C12
:10CC600090917F0C0E94CAC189819A81AB81BC815D
:10CC7000CA5DDE4F88839983AA83BB83C652D140A5
:10CC800080917E0C90917F0CDC01ED91FC910488E9
:10CC9000F589E02D1995CA5DDE4F8881C652D140D5
:10CCA000882301F18F3FA9F4C95DDE4F8881C75207
:10CCB000D1408F3F71F4C85DDE4F8881C852D140AA
:10CCC0008F3F39F4C75DDE4F8881C952D1408F3F15
:10CCD00049F00E94CDC470FFA7C180910E09833036
:10CCE00008F0A2C16BE973E182EA9CE00E94BAF20B
:10CCF0000FB6F894A89580916000886180936000D9
:10CD0000109260000FBE8091BD0A9091BE0A0097FC
:10CD100011F00F941E1986E690E00F94821826E613
:10CD2000FC0111922A95E9F7FC01E55BFF4F1382A4
:10CD3000128248EE53E060E070E0448355836683DE
:10CD400077832DE934E03183208328E024873F96E0
:10CD500025EC34E031832083128213821482158201
:10CD60009093BE0A8093BD0A8091BF0A8093B20A55
:10CD70008091010281110E94F2F926E030E046E83C
:10CD80005CE064E089E090E00E945AFA85EC94E06F
:10CD90009A8389831B821C821D821E82CE01039688
:10CDA0000F94750660E08EE290E00E94D3F9F12CBA
:10CDB000E12C80FF9BC08091BD0A9091BE0ADC01EE
:10CDC00096961D921D921D921C929997FC0112A697
:10CDD00013A614A615A69E961D921D921D921C9236
:10CDE000D19712AE13AE14AE15AEFE9640EE5EE2D3
:10CDF00060E070E04083518362837383349640EA3D
:10CE00005FE060E070E04083518362837383189633
:10CE100026E0FD01322F11923A95E9F7AC01425F0D
:10CE20005F4F34E1FA0111923A95E9F7E6E8FCE048
:10CE300001900D922A95E1F7FC01E65BFF4F10820D
:10CE40000F94CC027C01019709F050C06091BD0A9B
:10CE50007091BE0A625F7F4FCE0101960E94FAF286
:10CE6000CE0103960F9475066091BD0A7091BE0ABB
:10CE7000665E7F4FCE0101960E94FAF2CE010396C4
:10CE80000F9485066091BD0A7091BE0A6A5E7F4F5D
:10CE9000CE0101960E94FAF2CE0103960F947D0610
:10CEA0006091BD0A7091BE0A6E5D7F4FCE01019602
:10CEB0000E94FAF28B819C81AD81BE818093B50A7C
:10CEC0009093B60AA093B70AB093B80AE091BD0A4E
:10CED000F091BE0A828993899093BA0A8093B90A25
:10CEE000848995899093BC0A8093BB0A88E199E272
:10CEF0000FB6F894A895809360000FBE90936000E1
:10CF0000A895EF2809F41FC362EF72E182EA9CE062
:10CF10000E94BAF235ECE32E34E0F32EFA82E98275
:10CF20001B821C821D821E82CE0103960F946D0609
:10CF30008B819C81AD81BE81CA5DDE4F88839983E0
:10CF4000AA83BB83C652D140FA82E982CE01019600
:10CF50000F94250E82EA9CE00E9404F1CE018C5DC4
:10CF60009E4F0E9429C38091B50A9091B60AA09164
:10CF7000B70AB091B80A8B839C83AD83BE83C05E31
:10CF8000DE4F88839983AA83BB83C052D140CE01F0
:10CF9000825E9E4F0E94FBC3FA82E9821B821C8242
:10CFA0001D821E8224E030E0AE014D5F5F4F60E0E5
:10CFB00081E090E00E949CF98B819C81AD81BE81D3
:10CFC000C65EDE4F88839983AA83BB83CA51D14052
:10CFD000CE01885E9E4F0E9464C4FA82E9821B8261
:10CFE0001C821D821E8224E030E0AE014D5F5F4F47
:10CFF00060E085E090E00E949CF98B819C81AD818E
:10D00000BE81CC5EDE4F88839983AA83BB83C451E3
:10D01000D140CE018E5E9E4F0E9492C381E00E945D
:10D0200089C510920E0910C265E873E182EA9CE09E
:10D030000E94BAF285EC94E09A838983CA5DDE4F40
:10D0400088819981AA81BB81C652D1408B839C8300
:10D05000AD83BE83CE0101960F94250E80917E0C88
:10D0600090917F0C892B09F459C20E94E8C1882352
:10D0700009F454C2A0917E0CB0917F0C52961C9280
:10D080001E92519754961C921E92539784E890E0FA
:10D090001D969C938E931C971E961C921E9782E75A
:10D0A00055968C935597ED91FC9111970088F189D5
:10D0B000E02D64E170E0CD011995BE016F5F7F4FF7
:10D0C00080917E0C90917F0C0E94CAC189819A81C7
:10D0D000AB81BC81C05EDE4F88839983AA83BB830A
:10D0E000C052D14080917E0C90917F0CDC01ED917B
:10D0F000FC910488F589E02D1995C05EDE4F88818A
:10D10000C052D140882309F409C28F3FB1F4CF5DEA
:10D11000DE4F8881C152D1408F3F79F4CE5DDE4F22
:10D120008881C252D1408F3F41F4CD5DDE4F88816E
:10D13000C352D1408F3F09F4F1C16FE773E182EA36
:10D140009CE00E94BAF285EC94E09A838983C05EE9
:10D15000DE4F88819981AA81BB81C052D1408B83E7
:10D160009C83AD83BE83CE0101960F94250E8091E2
:10D170007E0C90917F0C892B09F4A9C10E94E8C113
:10D18000882309F4A4C1A0917E0CB0917F0C529623
:10D190001C921E92519754961C921E92539784E8AB
:10D1A00090E01D969C938E931C971E961C921E9742
:10D1B00082E755968C935597ED91FC9111970088D5
:10D1C000F189E02D68E170E0CD011995BE016F5F36
:10D1D0007F4F80917E0C90917F0C0E94CAC1898103
:10D1E0009A81AB81BC81C65EDE4F88839983AA8316
:10D1F000BB83CA51D14080917E0C90917F0CDC01A1
:10D20000ED91FC910488F589E02D1995C65EDE4FFD
:10D210008881CA51D140882309F459C18F3FB1F4A4
:10D22000C55EDE4F8881CB51D1408F3F79F4C45E1B
:10D23000DE4F8881CC51D1408F3F41F4C35EDE4F39
:10D240008881CD51D1408F3F09F441C16AE773E134
:10D2500082EA9CE00E94BAF285EC94E09A8389838A
:10D26000C65EDE4F88819981AA81BB81CA51D140B7
:10D270008B839C83AD83BE83CE0101960F94250ED4
:10D2800080917E0C90917F0C892B09F4E0C00E9464
:10D29000E8C1882309F4DBC0A0917E0CB0917F0C1B
:10D2A00052961C921E92519754961C921E9253971E
:10D2B00084E890E01D969C938E931C971E961C927A
:10D2C0001E9782E755968C935597ED91FC91119797
:10D2D0000088F189E02D6CE170E0CD011995BE0167
:10D2E0006F5F7F4F80917E0C90917F0C0E94CAC12E
:10D2F00089819A81AB81BC81CC5EDE4F8883998322
:10D30000AA83BB83C451D14080917E0C90917F0C45
:10D31000DC01ED91FC910488F589E02D1995CC5E36
:10D32000DE4F8881C451D140882309F490C08F3FDB
:10D33000B1F4CB5EDE4F8881C551D1408F3F79F487
:10D34000CA5EDE4F8881C651D1408F3F41F4C95E2D
:10D35000DE4F8881C751D1408F3F09F478C063E721
:10D3600073E182EA9CE00E94BAF245ECE42E44E0CC
:10D37000F42EFA82E982CC5EDE4F88819981AA81FF
:10D38000BB81C451D1408B839C83AD83BE83CE01CE
:10D3900001960F94250EFA82E982CC5EDE4F8881D9
:10D3A0009981AA81BB81C451D1408B839C83AD8379
:10D3B000BE83F801F182E082C65EDE4F88819981EA
:10D3C000AA81BB81CA51D14082839383A483B58350
:10D3D000CE53DF4FF982E882C25CD040C05EDE4FA0
:10D3E00088819981AA81BB81C052D140CC53DF4F43
:10D3F00088839983AA83BB83C45CD040CE5FDE4F11
:10D40000F982E882C250D140CA5DDE4F888199819D
:10D41000AA81BB81C652D140CC5FDE4F88839983FD
:10D42000AA83BB83C450D1409E012F5F3F4FA80108
:10D43000BE016E537F4FCE018E5F9E4F0E94BACCCD
:10D4400082EA9CE00E9404F182E090E08FC085ECCB
:10D4500094E09A838983C65EDE4F488159816A8150
:10D460007B81CA51D1404B835C836D837E83D8011D
:10D470008D939C93C05EDE4F488159816A817B8188
:10D48000C052D140F8014283538364837583CE53E5
:10D49000DF4F99838883C25CD040CA5DDE4F8881AC
:10D4A0009981AA81BB81C652D140CC53DF4F88837A
:10D4B0009983AA83BB83C45CD040AE014F5F5F4FAA
:10D4C000B801CE018E539F4F0E94F9CCB9CF85ECA5
:10D4D00094E09A838983C05EDE4F488159816A81D6
:10D4E0007B81C052D1404B835C836D837E83D801A6
:10D4F0008D939C93CA5DDE4F88819981AA81BB81FF
:10D50000C652D140F80182839383A483B583BE01C0
:10D510006F5F7F4FC8010E944BCD92CF85EC94E0A6
:10D520009A838983CA5DDE4F88819981AA81BB81F4
:10D53000C652D1408B839C83AD83BE83CE010196BE
:10D540000E9496CD7DCF61E373E18CEA9CE00E945E
:10D55000BAF262E073E18CEA9CE00E94BAF2809138
:10D560000E098F5F80930E0986EF9FEF9093830ED5
:10D570008093820E89E0E6E3F2E0D80101900D92FB
:10D580008A95E1F787E1F8013996DF011D928A95C6
:10D59000E9F78AE89CE0009731F0A801485F5F4F07
:10D5A00062E00F94D40C85EC94E0CE53DF4F998366
:10D5B0008883C25CD040CC53DF4F188219821A8214
:10D5C0001B82C45CD04082EC90E08C0F9D1F0296C1
:10D5D0000F946D060E9426D1683B7B408105910522
:10D5E00038F464E670E080E090E00E94F3D0F2CF7F
:10D5F000CC53DF4F88819981AA81BB81C45CD04024
:10D600008093180C9093190CA0931A0CB0931B0CD8
:10D61000C8010E946ACC892BC9F0E090140CF090EC
:10D62000150CD701ED91FC91C088D18862E072E0C1
:10D63000CE0101960E94FAF249EE54E1BE016F5FFD
:10D640007F4FC701F6011995811169C261ED72E141
:10D650008CEA9CE00E94BAF28CEA9CE00E9404F101
:10D6600028E2A22E2CE0B22E7501D12CC12CD701BC
:10D670008D919C91892B49F1960143E050E060E047
:10D6800070E0CB010E94C4D9D701ED91FC91808557
:10D690009185009711F00F941E19D701ED91FC911F
:10D6A00086819781009711F00F941E19D701ED9193
:10D6B000FC91848195810F941E19F70180819181DD
:10D6C0000F941E19D7011D921C92BFEFCB1ADB0AD3
:10D6D000E2E0EE0EF11CF8E0CF16D10441F686E050
:10D6E000E6E5F2E09E012F5F3F4F4901D90101902D
:10D6F0000D928A95E1F7FE0137968AE1DF011D92CE
:10D700008A95E9F786E89CE0009731F0AE014A5F20
:10D710005F4F66E00F94D40C61EE75E0C8010F9482
:10D72000C826D12CC12CF501819191915F01892BE3
:10D7300009F0FEC18AE090E00F9482187C01009706
:10D7400009F4F6C1DC0119961C921E9218971596E1
:10D750001C921E921497F80101900020E9F7CF0166
:10D760000197801B910B0F9482185C01D7011596CD
:10D770009C938E931497892B11F40C940D74F401DF
:10D7800001900020E9F7CF010197881999090F94BA
:10D790008218D70119969C938E931897009711F4CD
:10D7A0000C940A74B4010F94E72680E590E0F70129
:10D7B0009183808313821282B801C5010F94E726FA
:10D7C000F50101900020E9F73197AE16BF0620F46D
:10D7D000319781818E32C9F75F0122E0A20EB11C20
:10D7E000D5010D900020E9F7CD018A199B090B9610
:10D7F0000F9482184C01F70197838683009741F0BC
:10D80000B5010F94E72668EE75E0C4010F94C826B1
:10D81000F601EE0FFF1FE85DF34FF182E082960103
:10D8200042E050E060E070E0CB010E94C4D9019773
:10D8300009F487C164EF75E08CEA9CE00E9454F221
:10D840008CEA9CE00E9404F10FB6F894A8958091B0
:10D850006000886180936000109260000FBE80912C
:10D86000820E9091830E02970CF432C180910E09C2
:10D8700081112EC160E08EE290E00E94D3F980FF1A
:10D8800099C70091BD0A1091BE0A0115110509F44E
:10D890001FC10E9426D14B015C01F80182AD93ADFE
:10D8A000A4ADB5AD98012A5B3F4F7901892B8A2B36
:10D8B0008B2B09F466C7F90180819181A281B38124
:10D8C000A5019401281B390B4A0B5B0BCA01B90156
:10D8D00097FD52C028EE33E040E050E00F941C2248
:10D8E000C65DDE4F688379838A839B83CA52D140A9
:10D8F0002401350188EE480E83E0581E611C711C1E
:10D90000C65DDE4F88819981AA81BB81CA52D14010
:10D91000481A590A6A0A7B0AD7014D925D926D92A4
:10D920007C921397BA01A9014F5F5F4F6F4F7F4FF2
:10D93000F80182A993A9A4A9B5A96A017B01CC0C1D
:10D94000DD1CEE1CFF1C8C159D05AE05BF050CF003
:10D9500003C712AA13AA14AA15AAF80186A997A99F
:10D96000A0ADB1AD8C159D05AE05BF050CF0FDC693
:10D9700016AA17AA10AE11AE6801FAE4CF0ED11C98
:10D98000D6018C91833009F0F9C6F80182A993A9D8
:10D99000A4A9B5A9181619061A061B060CF4EEC69A
:10D9A00084E0D6018C93C8010F94CC0201967C01CF
:10D9B000F6018081833011F0811117C0F80186A92A
:10D9C00097A9A0ADB1AD181619061A061B066CF082
:10D9D000D6011C9284E13E96DF011D928A95E9F7FB
:10D9E000C8010F94CC0203967C01D801DA968D927F
:10D9F0009D92AD92BC92DD97B2E0EB16F10429F056
:10DA0000E4E0EE16F10409F050C06091BD0A709197
:10DA1000BE0A625F7F4FCE0101960E94FAF2CE01EC
:10DA200003960F9475066091BD0A7091BE0A665EFA
:10DA30007F4FCE0101960E94FAF2CE0103960F9419
:10DA400085066091BD0A7091BE0A6A5E7F4FCE0165
:10DA500001960E94FAF2CE0103960F947D06609122
:10DA6000BD0A7091BE0A6E5D7F4FCE0101960E9485
:10DA7000FAF28B819C81AD81BE818093B50A90932F
:10DA8000B60AA093B70AB093B80AE091BD0AF09124
:10DA9000BE0A828993899093BA0A8093B90A8489CD
:10DAA00095899093BC0A8093BB0AF3E0EF16F104CA
:10DAB00009F494C60CF073C631E0E316F10409F4DE
:10DAC0008AC66BE475E142E0E416F10409F489C604
:10DAD00088E199E20FB6F894A895809360000FBE94
:10DAE000909360002091820E3091830EC901C35D36
:10DAF000DE4F0FB6F894DEBF0FBECDBFDF91CF91E2
:10DB00001F910F91FF90EF90DF90CF90BF90AF905B
:10DB10009F908F907F906F905F904F90089569EBEA
:10DB200072E182EA9CE00E94BAF282EA9CE096CD21
:10DB3000FFEFCF1ADF0A28E0C216D10409F0F3CDB7
:10DB400079CE68EA72E182EA9CE00E94BAF2B801FA
:10DB500082EA9CE00E9454F261EA72E182EA9CE06F
:10DB60000E94BAF282EA9CE06DCE82E090E090934F
:10DB7000830E8093820E68CE80911309811105C0B7
:10DB80000E94371A81E08093130983E090E0EFCF81
:10DB900080917E0E8111AACF0E94CDC463FD36C054
:10DBA00080911B0981112FC00E9402B6883C91050B
:10DBB00019F484E090E0DBCF80911C09882359F0B0
:10DBC0006CE176E182EA9CE00E94BAF282EA9CE093
:10DBD0000E9404F1EECF85EC94E09A8389831B8246
:10DBE0001C821D821E82CE0103960F946D068B81CE
:10DBF0009C81AD81BE81892B8A2B8B2B09F435C288
:10DC00008FE090E0B4CF6CE076E1DCCF80911C092E
:10DC1000882349F084E090E09093830E8093820EF5
:10DC200062ED75E19BCF8FE090E0F6CFA8958091F3
:10DC3000190990911A09009721F00E94BAC1823007
:10DC400068F46FEB75E182EA9CE00E94BAF282EA26
:10DC50009CE00E9404F187E090E089CFC85EDE4F2F
:10DC60001882C851D140FE01EE5FFE4F1192119211
:10DC70008EE0DF011D928A95E9F70E94CEC08823CD
:10DC800019F085E090E073CFE0901909F0901A093F
:10DC9000E114F10441F0C7010E94BAC1082F10E05D
:10DCA000023011055CF463EB74E18CEA9CE00E94A5
:10DCB000BAF28CEA9CE00E9404F1A2CF70E060E02E
:10DCC000C7010E943D17009709F49CC09093660E0F
:10DCD0008093650E66EA74E182EA9CE00E94BAF2E3
:10DCE0006091650E7091660E82EA9CE00E9454F28B
:10DCF00082EA9CE00E9404F18091650E9091660E8C
:10DD00000E946ACC892B09F080C065E176E08CEA3C
:10DD10009CE00E9454F28CEA9CE00E9404F1E090A6
:10DD20001909F0901A0961E070E0C7010E943D17DF
:10DD30005C010230110509F47FC062E0C7010E9456
:10DD400028C1FC01C184D2840330110509F47DC0CF
:10DD500063E070E0C7010E943D177C0180917E0C5A
:10DD600090917F0C892B09F475C00E94E8C188232B
:10DD700009F470C0A0917E0CB0917F0C52961C9259
:10DD80001E92519754961C921E92539784E890E0ED
:10DD90001D969C938E931C971E961C921E9782E74D
:10DDA00055968C935597ED91FC9111970088F189C8
:10DDB000E02D60E470E0CD0119954FE050E0BE0128
:10DDC0006E5F7E4F80917E0C90917F0C0E943DC2D1
:10DDD0004C0180917E0C90917F0CDC01ED91FC91C7
:10DDE0000488F589E02D19958114910499F1E2E0F8
:10DDF000F1E0EC0FFD1FE80DF91D10828E010E5FA2
:10DE00001E4F3EC08BEC93E061CF62E974E182EA81
:10DE10009CE00E94BAF26091650E7091660E82EAF3
:10DE20009CE00E9454F26BE874E182EA9CE00E945C
:10DE3000BAF282EA9CE071CF8BE5C82E87E0D82E3B
:10DE40009E01285E3E4F790189CFAE01485E5E4F4C
:10DE50007A0184CF053011058CF264E070E0809186
:10DE6000190990911A090E943D178C016BE674E123
:10DE700082EA9CE00E94BAF282EA9CE00E9404F1ED
:10DE8000B092EE0AA092ED0AD092F00AC092EF0A88
:10DE90008DE799E39093E60A8093E50A40E150E02C
:10DEA0006EE574E1CE018E539F4F0F94F21A30E06D
:10DEB00020E041E050E060E2CE018F579F4F0F9489
:10DEC000910D40E250E065ED7FE1CE018F579F4F0D
:10DED0000F94D41A6EE374E182EA9CE00E94BAF2D5
:10DEE000B50182EA9CE00E9454F26CE374E182EA9C
:10DEF0009CE00E94BAF24AE050E0B60182EA9CE05F
:10DF00000E940BF265E374E182EA9CE00E94BAF29F
:10DF1000B70182EA9CE00E9454F260E374E182EA75
:10DF20009CE00E94BAF2F7018081811104C010E0E8
:10DF300000E0F12CE12CA090650EB090660E0E94DE
:10DF4000CEC08111B5C18091D00A9091D10ADC0177
:10DF5000ED91FC910688F789E02D1995882309F445
:10DF600087C081E090E09093DB0A8093DA0A87E033
:10DF7000E6E7F2E0DE01119601900D928A95E1F755
:10DF8000FE01319685E090E02191A091D20AB091F6
:10DF9000D30AA80FB91F2C9301968C309105A1F7D5
:10DFA00086E3E114F10429F086EB0115110509F06F
:10DFB00086EFC090D20AD090D30AF6018487809170
:10DFC000D70A85878091D60A86878090D40A909058
:10DFD000D50AB401C5010F94051B41968816990610
:10DFE00008F07DC08091D00A9091D10ADC01ED91BA
:10DFF000FC910488F589E02D199569EF73E18CEAAD
:10E000009CE00E94BAF26091F30A7091F40A4AE02F
:10E0100050E08CEA9CE00E940BF261EE73E18CEA26
:10E020009CE00E94BAF28CEA9CE00E9404F10E94FB
:10E0300026D160930F097093100980931109909372
:10E04000120980910D098F5F80930D0983330CF4C1
:10E05000A0C164EB73E18CEA9CE00E94BAF28CEA06
:10E060009CE00E9404F110920D0986EF9FEF7FCD96
:10E070006091ED0A7091EE0A8091D00A9091D10AD8
:10E08000DC01ED91FC914091EF0A5091F00A61158D
:10E09000710571F00088F189E02D1995019709F457
:10E0A00060CF8EEF9FEF9093F40A8093F30AA5CF91
:10E0B0000684F785E02D25EC34E03A8329834090EF
:10E0C000E90A5090EA0A6090EB0A7090EC0A4B82E1
:10E0D0005C826D827E82BE016F5F7F4FDECF4FE03C
:10E0E00050E0B601C5010E9406C16C01A090D40A9F
:10E0F000B090D50AB501CE018F579F4F0F94051BE5
:10E100008C0D9D1D0296A816B90608F46BCF609180
:10E11000D20A7091D30AA601CE018F579F4F0E9459
:10E1200006C16C01A090D40AB090D50AB501CE0109
:10E130008E539F4F0F94051B8C0D9D1D0296A816A4
:10E14000B90608F44FCF6091D20A7091D30AA601A4
:10E15000CE018E539F4F0E9406C16C01E114F10461
:10E16000B9F1A090D40AB090D50AB501C7010F94B7
:10E17000051B96012E5F3F4F820F931FA816B9060D
:10E1800008F430CF6091D20A7091D30AA601C7017A
:10E190000E9406C16C0101151105D1F0E090D40A6E
:10E1A000F090D50AB701C8010F94051B96012E5FA8
:10E1B0003F4F820F931FE816F90608F413CF6091C2
:10E1C000D20A7091D30AA601C8010E9406C16C014F
:10E1D000A601455051096091D20A7091D30A80E19D
:10E1E0000E9432D10E9426D16093DC0A7093DD0A2E
:10E1F0008093DE0A9093DF0A6093E00A7093E10A4D
:10E200008093E20A9093E30A8091D00A9091D10A18
:10E21000DC01ED91FC910084F185E02D1995892BAD
:10E2200021F50E9426D10091E00A1091E10A209187
:10E23000E20A3091E30A6B017C01C01AD10AE20ABA
:10E24000F30A2091D80A3091D90AA8EEB3E00F94CE
:10E250004E22C616D706E806F906B0F28CEF9FEFFD
:10E260009093F40A8093F30ABDCECE018E5E9E4F4A
:10E270000E94CFD5643071058105910509F0B2CEB9
:10E28000E091D20AF091D30A838190E08111E8CF26
:10E290000E9426D16093E00A7093E10A8093E20A1B
:10E2A0009093E30A1092E40A1092F40A1092F30A8F
:10E2B00010920D0962E274E182EA9CE00E94BAF2D7
:10E2C0006091650E7091660E82EA9CE00E9454F2A5
:10E2D00082EA9CE00E9404F181E080931B0930E017
:10E2E00020E043E050E061E4CE0101960F94910DEF
:10E2F0006FE276E0CE0101960F94C826CE0101961A
:10E300000E942AD230E020E042E050E061E4CE01F9
:10E3100001960F94910D63E376E0CE0101960F9480
:10E32000C826BE016F5F7F4F83E59DE00E9408F124
:10E33000CE0101960E942AD230E020E041E050E078
:10E3400061E4CE0101960F94910D63E376E0CE0176
:10E3500001960F94C826BE016F5F7F4F83E59DE055
:10E360000E9408F1CE0101960E942AD285E090E039
:10E370009093830E8093820E0E9426D160930F09A2
:10E3800070931009809311099093120965E074E16C
:10E39000E5CB8CE090E0EBCB0E9426D19B01AC0159
:10E3A00060910F09709110098091110990911209E3
:10E3B000A12CB12C650110E4E12E1FE1F12E00E04B
:10E3C00010E00F94720C882309F43ECA30E020E07C
:10E3D00043E050E061E4CE018F579F4F0F94910DC1
:10E3E0006FE276E0CE018F579F4F0F94C8260091C1
:10E3F000D40A1091D50AB801CE018F579F4F0F94C0
:10E40000051B09960817190790F10E94CEC08823B2
:10E4100071F18091DA0A9091DB0A019609F4B8C093
:10E420009093DB0A8093DA0AE091D20AF091D30A42
:10E430008091DB0A8583E091D20AF091D30A809122
:10E44000DA0A86836091D20A7091D30A47E050E0DD
:10E45000CE018F579F4F0E9406C1AC014550510914
:10E460006091D20A7091D30A82EA0E9432D1FE01F1
:10E47000EE53FF4F119211928EE3DF011D928A95A8
:10E48000E9F71A821982FE0133968EE7DF011D92A9
:10E490008A95E9F730E020E041E050E060E4CE0109
:10E4A0008E539F4F0F94910D4FE350E065ED7FE148
:10E4B000CE018E539F4F0F94D41A4FE750E06FEC6C
:10E4C0007FE1CE0101960F94F21ABE016F5F7F4F7C
:10E4D000CE018E539F4F0E94F4D130E020E041E006
:10E4E00050E060E4CE018E539F4F0F94910D4FE3A7
:10E4F00050E066E175E1CE018E539F4F0F94D41A20
:10E500004FE750E06CE075E1CE0101960F94F21AEE
:10E510004FE750E069EF74E1CE0101960F94D41AF1
:10E52000BE016F5F7F4FCE018E539F4F0E94F4D18B
:10E5300030E020E041E050E060E4CE018E539F4F98
:10E540000F94910D4FE350E06CEE7FE1CE018E53BE
:10E550009F4F0F94D41A4FE750E069EE74E1CE015B
:10E5600001960F94F21ABE016F5F7F4FCE018E535A
:10E570009F4F0E94F4D186E090E09093830E8093A9
:10E58000820E68EA75E182EA9CE00E94BAF25CC9F8
:10E5900081E090E045CF0E94CEC0811155C909CBE2
:10E5A0000E9426D160930F0970931009809311097E
:10E5B0009093120985EF9FEFDACA0E9426D19B0142
:10E5C000AC0160910F09709110098091110990912F
:10E5D0001209A12CB12C650118E8E12E13E1F12EEE
:10E5E00000E010E00F94720C882309F42DC91092FA
:10E5F000830E1092820E28C90E94CEC0882309F48F
:10E600004AC0E091D20AF091D30A80EE8083E09173
:10E61000D20AF091D30A11828091D00A9091D10A46
:10E620006091D20A7091D30ADC01ED91FC910280D5
:10E63000F381E02D42E050E019958FEF9FEF90932A
:10E64000F40A8093F30A8091D00A9091D10ADC01F8
:10E65000ED91FC910680F781E02D19958091D00A0B
:10E660009091D10ADC01ED91FC910488F589E02DAF
:10E6700019950E9426D16093DC0A7093DD0A80937D
:10E68000DE0A9093DF0A6093E00A7093E10A8093B8
:10E69000E20A9093E30A0E9426D160930F097093D7
:10E6A000100980931109909312098DE090E05FCAE0
:10E6B0000E9426D19B01AC0160910F097091100955
:10E6C0008091110990911209A12CB12C650110E1E2
:10E6D000E12E17E2F12E00E010E00F94720C811190
:10E6E00068CAB2C80E9426D160930F0970931009BE
:10E6F00080931109909312098EE090E038CA8091BE
:10E700007E0E811105C00E94B8B4892B09F051CA50
:10E710000E9426D19B01AC0160910F0970911009F4
:10E720008091110990911209A12CB12C650110E37F
:10E73000E12E15E7F12E00E010E00F94720C882313
:10E7400009F482C865E875E18CEA9CE00E94BAF29F
:10E75000F0E0E0E0199578C8841B950BA60BB70B89
:10E7600082AB93ABA4ABB5ABF8C8841B950BA60BDF
:10E77000B70B86AB97ABA0AFB1AFFEC8F12CE12CC5
:10E7800017C9D501C40188519C4FAF4FBF4FF90144
:10E7900080839183A283B383F12CE12C26C96CE1A1
:10E7A00075E154E0E516F104E1F085E0E816F104C6
:10E7B00009F08EC96CE775E18CEA9CE00E94BAF220
:10E7C0008CEA9CE00E9404F186EF9FEF9093830E09
:10E7D0008093820E7DC968E675E1EECF68E375E14E
:10E7E000EBCF82EA9CE00E94BAF285EC94E09A8337
:10E7F00089831B821C821D821E82CE0103960F9488
:10E800006D06CE0101960F94250E82EA9CE00E94CF
:10E8100004F15EC9C5010F941E19D70116968D919A
:10E820009C91009711F00F941E19F7018085918536
:10E83000009711F00F941E19C7010F941E190C9424
:10E840001A6CAF92BF92DF92EF92FF920F931F93D9
:10E85000CF93DF9300D000D0CDB7DEB78C017B0122
:10E86000D42EFB0184819581892BF9F0A080B180A1
:10E870006FE370E0C5010F94D3260097B1F09C01BF
:10E880002A193B0937FD11C050E040E0B701CE0125
:10E8900001960E94CEEEBE016F5F7F4FC7010E94BE
:10E8A00004EECE0101960E94ACEEF70184819581C1
:10E8B000892BD9F1E080F18065E376E0C7010F9400
:10E8C000DE26892B01F5F801128A118A80E090E199
:10E8D0009587848784E890E0948B838B81E086879A
:10E8E000D58A81E090E026960FB6F894DEBF0FBE81
:10E8F000CDBFDF91CF911F910F91FF90EF90DF90EF
:10E90000BF90AF90089562E476E0C7010F94DE26D1
:10E91000892B59F4F801128A118A148A138A84E81F
:10E9200090E0958784871686DBCF90E080E0DBCF90
:10E9300090E080E00895DC01ED91FC910284F38584
:10E94000E02D1994DF92EF92FF920F931F93CF93D4
:10E95000DF93EC010C891D890115110559F01D8A01
:10E960001C8AC801DF91CF911F910F91FF90EF900A
:10E97000DF900895EC85FD858E859F85DF01A80FCA
:10E98000B91F2C91243209F055C011962C912B37C8
:10E9900009F050C00296E80FF91FF12CE12CDF01BD
:10E9A000D190DD2009F446C08DE7D816E9F08FEF4D
:10E9B000E81AF80AF4CF198A188A2C853D852115A2
:10E9C000310579F08E859F85280F391FF901208147
:10E9D000222321F001969F878E873EC01D861C86CC
:10E9E000C0CF0FEF1FEFBDCFE114F10419F11C925E
:10E9F0008E859F8502966C857D85680F791FE881DD
:10EA0000F9810684F785E02DCE011995998B888BC5
:10EA10001B8A1A8AEC85FD858E859F85E80FF91F74
:10EA2000EE0DFF1DD2828E859F850396E80EF91E9E
:10EA3000FF86EE86288939892115310509F4BDCF75
:10EA40008A899B89280F391FF9012081222309F423
:10EA5000B2CF01969B8B8A8B022F220F110B81CF95
:10EA6000DC011C96ED91FC911D971E968D919C9159
:10EA7000E80FF91F8081082E000C990B0895DC0126
:10EA800015968D919C91009739F0DC01ED91FC91E8
:10EA90000680F781E02D199408950097D1F0DC01EC
:10EAA0001696ED91FC913097A1F080858F7084309F
:10EAB00021F481859285009771F40680F781E02D1D
:10EAC000309739F080858F70843019F48185928574
:10EAD000089590E080E0089583E090E00895DC01DF
:10EAE0001296ED91FC9113973097B9F016968D918F
:10EAF0009C918430910541F08530910541F0039758
:10EB000049F482E090E0089581E090E0089581E189
:10EB100090E00895808590E0089590E080E0089569
:10EB200085E090E0089590E080E008958EE090E028
:10EB30000895DC011296ED91FC9113973097B9F08E
:10EB400016968D919C918430910541F08530910508
:10EB500041F0039749F482E090E0089581E090E06D
:10EB6000089581E190E00895808590E0089590E017
:10EB700080E0089584E190E00895DC01ED91FC913E
:10EB80000484F585E02D60E0199581E090E008951A
:10EB90008FE090E09093830E8093820E88EC90E05B
:10EBA00008956CEA7CE1811102C06EEA7CE182EAA0
:10EBB0009CE00C94BAF267ED78E182EA9CE00E9456
:10EBC000BAF2F0E0E0E0199584EF91E008954F92F9
:10EBD0005F926F927F92AF92BF92DF92EF92FF921D
:10EBE0000F931F93CF93DF9300D000D0CDB7DEB744
:10EBF0007C01D62E80912609882309F4BEC0D70156
:10EC000014969C9180911E02891708F4B6C08091D9
:10EC1000950990919609BAE06B13F0C08B5B964F03
:10EC2000FC011082D70118960D911C910115110558
:10EC300009F49FC0F801618572856115710591F431
:10EC400045805680678070848091A60A9091A70ABB
:10EC5000A091A80AB091A90A481659066A067B062F
:10EC600009F487C0D8011B964D915C911C97411502
:10EC7000510509F47EC0F701248153968C91539776
:10EC800090E0322F377002C0959587953A95E2F75C
:10EC900080FF6FC0A22EB12CC501887F9370892B95
:10ECA00039F451968D919C91887F9370A82AB92A46
:10ECB000D8018D919C91DC01ED91FC91611571055C
:10ECC00009F486C00688F789E02D1995019709F0A7
:10ECD00050C06CE3F801808191810E94BCF1A501D4
:10ECE00070E060E02AE0D8018D919C910E94B8F01C
:10ECF000F8012281808191816CE577E2222311F075
:10ED00006AE577E20E94BAF2D8011D966D917C9176
:10ED10001E978D919C910E9454F260E2F8018081CF
:10ED200091810E94BCF1D8011F966D917C91509702
:10ED30008D919C910E9454F2F801228180819181F1
:10ED40006FE477E2222311F069E477E20E94BAF2DD
:10ED500065E479E0D8018D919C910E9454F2F8010C
:10ED600080819181DC01ED91FC91008CF18DE02D91
:10ED700019951092960910929509D70115968D91C3
:10ED80009C911697009771F014963C9120911F0268
:10ED9000231740F0DC01ED91FC910190F081E02D12
:10EDA0006D2D199581E090E026960FB6F894DEBFA0
:10EDB0000FBECDBFDF91CF911F910F91FF90EF90CC
:10EDC000DF90BF90AF907F906F905F904F900895CD
:10EDD0000488F589E02D25EC34E03A832983D801B5
:10EDE00015964D905D906D907C9018974B825C824B
:10EDF0006D827E82BE016F5F7F4F67CF8F3491053A
:10EE00000CF0BBCFBDE06B1709F4B7CF9C012F5FAF
:10EE10003F4F30939609209395098B5B964FFC01E9
:10EE20006083ABCFCF93DF93EC016BE874E283E5B3
:10EE30009DE00E94BAF283E59DE00E9404F1E88122
:10EE4000F9810484F585E02D60E0CE01199581E01B
:10EE500090E0DF91CF910895CF93DF93EC0164E1CF
:10EE600071E283E59DE00E94BAF2EA81FB810190A4
:10EE7000F081E02D6081718183E59DE00E9454F274
:10EE800083E59DE00E9404F1E881F9810484F58521
:10EE9000E02D60E0CE01199581E090E0DF91CF9107
:10EEA00008950D941E190D941E190D941E190D949C
:10EEB0001E190D941E190D941E190D941E190D94F2
:10EEC0001E19CF93C1E068EE73E080E090E00E94ED
:10EED000F3D04AE050E06C2F82EA9CE00E9421F1DE
:10EEE000CF5FC43181F784EF91E0CF910895FC01A9
:10EEF000828193810E94EB3521E030E0823011F471
:10EF000030E020E0C90108950F931F93CF93DF9362
:10EF10008C01D0E0C0E001151105B1F0BE01685CC4
:10EF20007E4DC8010F94BB1A892B51F4FE01E45C9D
:10EF3000FE4D849190E0DF91CF911F910F91089544
:10EF40002596C233D10539F781E090E0F4CFCF9216
:10EF5000EF92FF920F931F93CF93DF9300D000D0D7
:10EF60001F921F92CDB7DEB77C0109831A832B83D2
:10EF70003C834D835E836F8378876BEF70E283E51C
:10EF80009DE00E94BAF2CE0101960E94D8228981AA
:10EF900081112AC00A810F70013071F128F010E050
:10EFA0000230E9F5CC20E9F060E0CE0101960E9444
:10EFB000E91DF70102811381892B69F0C8010E94C4
:10EFC000FD2D672B682B692B61F480E00F94730D86
:10EFD000AB01BC0103C040E050E0BA01C8010E948F
:10EFE000BC2D81E090E02EC08031D0F58E30D8F578
:10EFF0008130C9F18230D9F16EEE70E283E59DE097
:10F000000E94BAF24AE050E0698183E59DE00E94E7
:10F0100021F183E59DE00E9404F101E010E06EED36
:10F0200070E283E59DE00E94BAF24AE050E0B80148
:10F0300083E59DE00E940BF283E59DE00E9404F1D0
:10F0400090E080E028960FB6F894DEBF0FBECDBFEB
:10F05000DF91CF911F910F91FF90EF90CF90089586
:10F060008351833048F6F70102811381A7CF40E036
:10F0700050E0BA01F70182819381B1CFFF920F93E3
:10F080001F93CF93DF93CDB7DEB764970FB6F89495
:10F09000DEBF0FBECDBF8C01F62E8FE290E09A83CB
:10F0A0008983FE01339688E0DF011D928A95E9F796
:10F0B000F8016681FF2011F081E06827D8011496DD
:10F0C0008C910E947DCEF80187819085A185B285C3
:10F0D000883E9340A105B10508F491C06CEA76E240
:10F0E00083E59DE00E94BAF2D80114966D917C915F
:10F0F0004AE050E083E59DE00E940BF267EA76E289
:10F1000083E59DE00E94BAF26F2D70E04AE050E086
:10F1100083E59DE00E940BF283E59DE00E9404F1EF
:10F120006EEC76E2CE0101960F94B01AF80182815E
:10F1300093810E94EB35FF2009F46DC06FE976E200
:10F14000843151F068E976E2853131F06CE876E29D
:10F150008F3011F464E976E2CE010B960F94C41A55
:10F1600067E776E283E59DE00E94BAF2D801129645
:10F17000ED91FC9113970190F081E02D60817181F8
:10F18000ED91FC910288F389E02D9E012F5F3F4FA6
:10F19000AE01455F5F4FC80119954AE050E0BC01E0
:10F1A00083E59DE00E940BF265E776E283E59DE052
:10F1B0000E94BAF2D8011296ED91FC910190F08173
:10F1C000E02D6081718183E59DE00E9454F2BE01D3
:10F1D0006F5F7F4F83E59DE00E9454F262E776E225
:10F1E00083E59DE00E94BAF2BE01655F7F4F83E533
:10F1F0009DE00E9454F283E59DE00E9404F1649634
:10F200000FB6F894DEBF0FBECDBFDF91CF911F9137
:10F210000F91FF90089568E876E2823009F49CCF60
:10F2200063E876E299CFAF92BF92CF92EF92FF92CE
:10F230000F931F93CF93DF9300D000D01F921F92A4
:10F24000CDB7DEB75C0109831A832B833C834D83E2
:10F250005E836F83788765ED76E283E59DE00E94AB
:10F26000BAF2CE0101960E94D822E114F10439F0DD
:10F270006EEC76E2C7010F94BB1A009731F1F501ED
:10F280000281138101151105F1F0898181115DC0A1
:10F290008A818F70813009F460C048F1823029F191
:10F2A000082F10E061EB76E283E59DE00E94BAF260
:10F2B0004AE050E0B80183E59DE00E940BF283E54F
:10F2C0009DE00E9404F190E080E028960FB6F8944B
:10F2D000DEBF0FBECDBFDF91CF911F910F91FF9089
:10F2E000EF90CF90BF90AF900895CC20C1F060E038
:10F2F000CE0101960E94E91D892B09F447C0C8017F
:10F300000E94FD2D672B682B692BE1F480E00F94A0
:10F31000730DAB01BC01C8010E94BC2D13C0C80114
:10F320000E94EB358E3019F050F4813059F460E0D2
:10F33000CE0101960E94E91D892B21F0E0CF835177
:10F340008330A8F381E090E0C0CF8031D0F48E30DC
:10F35000B0F68130A1F28230C9F061EC76E283E54B
:10F360009DE00E94BAF24AE050E0698183E59DE0A9
:10F370000E9421F183E59DE00E9404F101E010E08C
:10F3800091CF8351833008F4BACFE7CF40E050E00B
:10F39000BA01C8010E94BC2D60E0C5010E943E7800
:10F3A000D1CF2F923F924F925F926F927F928F9226
:10F3B0009F92AF92BF92CF92DF92EF92FF920F9304
:10F3C0001F93CF93DF93CDB7DEB760970FB6F89456
:10F3D000DEBF0FBECDBF6130710509F495C0DC0101
:10F3E00012966D917C916115710509F48DC04C01E7
:10F3F00019821A821B821C821D821E821F8218861D
:10F400008A818F708A8340E052E0CE0101960E948B
:10F41000F83560E0CE0101960E94E91D1C01F4015F
:10F42000828193810E94FD2D2B013C01D40117960E
:10F430002D913D914D915C911A97D1010F944622E7
:10F440002FEF30E040E050E00F94FA2129873A870F
:10F450004B875C870E9426D19B01AC0189859A85E8
:10F46000AB85BC850097A105B10509F468C0A12C46
:10F47000B12C65017C018D01C301B2010F94720CA6
:10F4800089874114510461047104F1F1D401179684
:10F490008D919D910D90BC91A02D8D879E87AF87FA
:10F4A000B88B0E9426D19B01AC018D859E85AF85CE
:10F4B000B8890097A105B10561F0A12CB12C6501B7
:10F4C0007C018D01C301B2010F94720C882309F4F1
:10F4D00051C0D40112966D907C9080E00F94730D12
:10F4E000AB01BC01C3010E94BC2D232869F0F401CB
:10F4F00084810F945C0DD40116969C91891304C0ED
:10F5000061E0C4010E943E7890E080E060960FB612
:10F51000F894DEBF0FBECDBFDF91CF911F910F9149
:10F52000FF90EF90DF90CF90BF90AF909F908F9023
:10F530007F906F905F904F903F902F90089591E053
:10F5400099879FCFB985BB23F1F060E0C4010E9489
:10F550003E78F401828193810E94F74F892BA1F6B6
:10F5600040E050E0BA01D40112968D919C910E9426
:10F57000BC2DCACFF40184810F945C0DD401169682
:10F580009C918913DFCF232809F4BECFF401848135
:10F590000F945C0DD40116969C918913B5CFB98553
:10F5A000B111B2CFADCF60E08DE00C947DCE61E0C3
:10F5B0008DE00C947DCECF93DF93EC0166E676E28E
:10F5C00083E59DE00E94BAF26C817D814AE050E0C3
:10F5D00083E59DE00E940BF260E676E283E59DE024
:10F5E0000E94BAF283E59DE00E9404F160E08C8104
:10F5F0000E94ABCEE881F9810484F585E02D60E0BE
:10F60000CE01199581E090E0DF91CF910895CF93DD
:10F61000DF93EC016DE376E283E59DE00E94BAF2B0
:10F620006C817D814AE050E083E59DE00E940BF211
:10F630006BE376E283E59DE00E94BAF2EA81FB810A
:10F640000190F081E02D6081718183E59DE00E9451
:10F6500054F265E376E283E59DE00E94BAF283E529
:10F660009DE00E9404F1E881F981048CF58DE02D84
:10F67000CE0119958130910529F0029759F060E08B
:10F680008C811AC063E070E0CE010E944C6560E09E
:10F690000E94ABCE60E08C810E94ABCE61E070E056
:10F6A000CE010E944C6560E00E94ABCE62E070E04B
:10F6B000CE010E944C6560E00E94ABCEE881F981EA
:10F6C0000484F585E02D60E0CE01199581E090E09D
:10F6D000DF91CF910895EF92FF921F93CF93DF9325
:10F6E000192F7B01C82FD92FD7FF03C0D195C19502
:10F6F000D10961E08C2F0E94ABCE82E0E816F104C4
:10F7000099F460E08C2F0E947DCE67EC7FE183E569
:10F710009DE00E94BAF283E59DE0DF91CF911F91B9
:10F72000FF90EF900C9404F1612FEF2851F4609555
:10F73000661F6627661F8C2F0E947DCE63EC7FE1DB
:10F74000E6CF661F6627661F8C2F0E947DCE6EEB6C
:10F750007FE1DDCFCF93DF93EC0164E576E283E5D3
:10F760009DE00E94BAF26C817D814AE050E083E521
:10F770009DE00E940BF26EE476E283E59DE00E943C
:10F78000BAF283E59DE00E9404F161E08C810E9461
:10F79000ABCE6E818C810E947DCE8A819B81009749
:10F7A00029F040E050E0BA010E94BC2DE881F981C7
:10F7B0000484F585E02D62E0CE0119958A819B8154
:10F7C0000E94F74F181619065CF40A80DB81C02DE1
:10F7D00080E00F94730DAB01BC01CE010E94BC2DE3
:10F7E00081E090E0DF91CF910895CF93DF93EC011A
:10F7F0006BE276E283E59DE00E94BAF26C817D8146
:10F800004AE050E083E59DE00E940BF269E276E277
:10F8100083E59DE00E94BAF2EA81FB810190F081CC
:10F82000E02D6081718183E59DE00E9454F263E2E6
:10F8300076E283E59DE00E94BAF283E59DE00E94B6
:10F8400004F18A819B81892B09F451C08C819D81AF
:10F85000892B09F04CC0E881F981048CF58DE02DED
:10F86000CE0119958130910529F0029759F061E098
:10F870008C811AC063E070E0CE010E944C6561E0AB
:10F880000E94ABCE61E08C810E94ABCE61E070E063
:10F89000CE010E944C6561E00E94ABCE62E070E058
:10F8A000CE010E944C6561E00E94ABCE8091A10028
:10F8B000887F8093A10080919100887F8093910040
:10F8C0008091A10082608093A1008091910082606C
:10F8D00080939100E881F9810484F585E02D62E050
:10F8E000CE01199581E090E0DF91CF91089590E0ED
:10F8F00080E0FACFCF93DF93EC0165E071E283E51E
:10F900009DE00E94BAF2EA81FB810190F081E02D36
:10F910006081718183E59DE00E9454F283E59DE062
:10F920000E9404F1E881F9810484F585E02D62E00C
:10F93000CE01199581E090E0DF91CF910895DC012F
:10F94000ED91FC910484F585E02D62E0199581E04C
:10F9500090E00895AF92BF92CF92DF92EF92FF9224
:10F960000F931F93CF93DF93CDB7DEB768970FB692
:10F97000F894DEBF0FBECDBFFC01098B1A8B2B8B19
:10F980003C8B4D8B5E8B6F8B788F82819381009740
:10F9900009F4A3C024813581232B09F49EC0CC2017
:10F9A00009F49BC06F0170E060E00E945F2E192F88
:10F9B000D601ED91FC91048CF58DE02DC6011995D1
:10F9C0005C018230910509F47CC0039709F447C0BB
:10F9D00095E0F1E0AF16B10409F091E019861A86BE
:10F9E0001B861C861D861E861F86188A9295907F10
:10F9F0008A858F70892B8A87EE24EA94FE2C0989E8
:10FA00001A892B893C894D895E896F89788DCE0151
:10FA100009960E946123F1E0AF16B10409F453C0C6
:10FA200082E0A816B10409F049C06F8570E0D601E4
:10FA300014968C910E94E7CE61E070E0C6010E94AE
:10FA40004C656E8570E00E94E7CE62E070E0C60112
:10FA50000E944C656D8570E00E94E7CE2FC0612F3B
:10FA6000661F6627661FCE0141960E94E91D5C0154
:10FA7000BC01D60114968C910E94E7CE69E476E22F
:10FA800083E59DE00E94BAF2F601648175814AE047
:10FA900050E083E59DE00E940BF267E476E283E5A7
:10FAA0009DE00E94BAF24AE050E0B50183E59DE096
:10FAB0000E940BF283E59DE00E9404F181E090E05A
:10FAC0000EC094E08BCF63E070E0C6010E944C65ED
:10FAD000688970E00E94E7CEA8CF90E080E0689649
:10FAE0000FB6F894DEBF0FBECDBFDF91CF911F914F
:10FAF0000F91FF90EF90DF90CF90BF90AF9008955F
:10FB0000CF92DF92FF920F931F93CF93DF9300D09A
:10FB100000D01F921F92CDB7DEB76C01F02E012FDF
:10FB20001A830F7010E0FF2029F00115110511F460
:10FB300001E010E040E050E460E070E0F601828116
:10FB400093810E9474300130110591F1023011054A
:10FB500041F0012B99F56CE474E283E59DE00E948D
:10FB6000BAF28A81807FA1F1F60102811381C80176
:10FB70000E94FD2D672B682B692B89F401E010E0B2
:10FB8000C80128960FB6F894DEBF0FBECDBFDF9137
:10FB9000CF911F910F91FF90DF90CF90089580E05B
:10FBA0000F94730DAB01BC01C8010E94BC2DE6CFC0
:10FBB000F1E0FF1681F082E0F81669F060E474E28B
:10FBC00083E59DE00E94BAF283E59DE00E9404F186
:10FBD00010E000E0D5CFF601C280D380C6010E94BC
:10FBE000FD2D672B682B692B49F280E00F94730D74
:10FBF000AB01BC01C6010E94BC2DC2CFCF92DF92E7
:10FC0000EF92FF920F931F93CF93DC011296ED9129
:10FC1000FC9160E0828193810E9428C18C01009751
:10FC200029F0FC0180858F708530D1F061E975E2A3
:10FC30008CEA9CE00E94BAF28CEA9CE00E9404F1FB
:10FC4000C12CD12C90E8E92E9FEBF92EC701B6010B
:10FC5000CF911F910F91FF90EF90DF90CF9008957B
:10FC6000C8010E94BAC1813040F18630A8F18930C4
:10FC700020F565E0C8010E9428C1FC0190859F70B5
:10FC80009330F9F4C184D284E384F484C1E060E069
:10FC9000C8010E9428C1FC0190859F70933009F52E
:10FCA000618572858385948520E030E0A9010F94F9
:10FCB000B02087FF1FC0C111C9CFC12CD12C760144
:10FCC000C5CF923049F461857285838594850F9400
:10FCD000B7206B017C01DACFC0E0C12CD12C7601BA
:10FCE000D6CF923039F461857285838594850F94DF
:10FCF000B720DACFC111AACFC12CD12C8FE7E82EC3
:10FD000083E4F82EA3CFAF92BF92CF92DF92EF920F
:10FD1000FF920F931F93CF93DF9300D000D01F92D9
:10FD20001F92CDB7DEB7DC011296ED91FC913097B2
:10FD300009F466C022813381232B09F461C08C0150
:10FD4000662309F46EC00E94FE7DE62EB72E6C017C
:10FD5000D8011296ED91FC910190F081E02D608127
:10FD600071818CEA9CE00E9454F267EB75E28CEAA8
:10FD70009CE00E94BAF28CEA9CE00E9404F120E030
:10FD800030E0A9016E2D7B2DC6010F94B82387FDAD
:10FD900037C06BEA75E28CEA9CE00E94BAF24E2D05
:10FDA0005B2DB6018CEA9CE00E946CC68CEA9CE05C
:10FDB0000E9404F1D8011296ED91FC9161E08281DC
:10FDC00093810E9428C119821A821B821C822A8177
:10FDD0002F702067F22E2E2D4E2D5B2DB6014D83F8
:10FDE0005E836F837887B12CA12CD12CC12CE98044
:10FDF0000B811C813E814F8158856FEF0F949610C7
:10FE000028960FB6F894DEBF0FBECDBFDF91CF911D
:10FE10001F910F91FF90EF90DF90CF90BF90AF9028
:10FE200008950190F081E02D6081718182EA9CE06B
:10FE30000E9454F264EC75E282EA9CE00E94BAF2FD
:10FE400082EA9CE028960FB6F894DEBF0FBECDBFC5
:10FE5000DF91CF911F910F91FF90EF90DF90CF90A6
:10FE6000BF90AF900C9404F16F927F928F929F920B
:10FE7000AF92BF92CF92DF92EF92FF920F931F93B8
:10FE8000CF93DF93CDB7DEB7A8970FB6F894DEBF58
:10FE90000FBECDBF09A31AA32BA33CA34DA35EA302
:10FEA0006FA378A7DC011496ED91FC91309719F4BB
:10FEB00090E080E0C3C020813181232BC9F34C0145
:10FEC000DC01ED91FC910284F385E02D19950297F8
:10FED00079F78AA1982F9F70E92EF12C19A111238F
:10FEE00021F0E114F10409F424C1923009F4CDC0E9
:10FEF000B8F4992309F4C9C09130B9F067ED75E2FF
:10FF000083E59DE00E94BAF24AE050E0B70183E544
:10FF10009DE00E940BF283E59DE00E9404F1C8CFB2
:10FF2000933009F43EC0993049F7D4011296ED910F
:10FF3000FC9161E0828193810E9428C13C01198E6D
:10FF40001A8E1B8E1C8E1D8E1E8E1F8E18A28A8DE1
:10FF50008F708A8F198F61E0CE0149960E94031B32
:10FF60001150153108F056C1E12FF0E08827E45414
:10FF7000F0488F4F0D9471229D809D800A810A81E7
:10FF80000A810A810A810A810A81E180FB800A8153
:10FF90000A819D809D800A810A810A819D809D80C1
:10FFA0009D80807F09F484CFCE0181960E940A1F34
:10FFB000D4011496ED91FC916683778380879187B5
:10FFC0006DE176E283E59DE00E94BAF2D4011296DB
:10FFD000ED91FC910190F081E02D6081718183E5CC
:10FFE0009DE00E9454F26FE076E283E59DE00E947E
:10FFF000BAF2D4011496ED91FC9146815781608547
:020000021000EC
:10000000718583E59DE00E946CC683E59DE00E94BA
:1000100004F1F401E480F5800E9426D1D7015296C4
:100020006D937D938D939C935597D4011496ED9188
:10003000FC918689811117C081E090E0A8960FB6E7
:10004000F894DEBF0FBECDBFDF91CF911F910F910E
:10005000FF90EF90DF90CF90BF90AF909F908F90E8
:100060007F906F900895168A60E0C4010E94837E9D
:10007000D4011496ED91FC9180E090E0A0E0B0EC0A
:1000800086879787A08BB18BD7CF807F09F410CF5D
:10009000CE0181960E940A1FD4011496ED91FC9125
:1000A000628773878487958769E076E283E59DE0C0
:1000B0000E94BAF2D4011296ED91FC910190F08168
:1000C000E02D6081718183E59DE00E9454F26EEF26
:1000D00075E283E59DE00E94BAF2D4011496ED9199
:1000E000FC91428553856485758583E59DE00E947A
:1000F0006CC683E59DE00E9404F1D4011296ED9157
:10010000FC9162E0828193810E9428C1009709F4EA
:1001100093CFB12CA12CD12CC12CE9A0FAA00BA11A
:100120001CA12DA13EA14FA158A56FEF0F949610D1
:1001300083CFEE24E394F12CF8CEB12CA12CD12C5A
:10014000C12CE98CFA8C0B8D1C8D2D8D3E8D4F8D25
:1001500058A16FEFC3010F94961019861A861B865B
:100160001C861D861E861F86188A8A858F708A8740
:1001700040E050E061E070E0F401828193810E94F0
:100180009D30672B682B692BD1F46AE0CE0109966C
:100190000E942A1BB12CA12CD12CC12C79018A01DF
:1001A0009B01AC016FEFC3010F94961060E074E007
:1001B000D40112968D919C910E9480363DCF6BE0C8
:1001C000E5CF40E050E460E070E0F401828193818B
:1001D0000E947430B12CA12CD12CC12CE98CFA8C4A
:1001E0000B8D1C8D2D8D3E8D4F8D58A16FEFC30152
:1001F0000F9496103DCFB12CA12CD12CC12CE98CA1
:10020000FA8C0B8D1C8D2D8D3E8D4F8D58A16FEF6F
:10021000C3018CCF6CEE75E283E59DE00E94BAF2DB
:100220004AE050E069A183E59DE00E9421F183E569
:100230009DE00E9404F162CE2F923F924F925F9216
:100240006F927F928F929F92AF92BF92CF92DF92E6
:10025000EF92FF920F931F93CF93DF93CDB7DEB74B
:10026000A9970FB6F894DEBF0FBECDBF6130710500
:1002700009F439C3DC011496ED91FC913097D9F45F
:1002800081E090E0A9960FB6F894DEBF0FBECDBF17
:10029000DF91CF911F910F91FF90EF90DF90CF9062
:1002A000BF90AF909F908F907F906F905F904F9096
:1002B0003F902F90089520813181232B09F31C0159
:1002C000DC01ED91FC910284F385E02D19950297F4
:1002D000B9F6F101028113810115110589F2C801F6
:1002E0000E94EB35823061F240E050E061E070E066
:1002F000C8010E949D30672B682B692B09F6D1013C
:100300001496ED91FC9100811181F80182AD882352
:1003100009F495C20E9426D169A37AA38BA39CA35A
:10032000F80182A193A1A4A1B5A149A15AA16BA1F1
:100330007CA1481B590B6A0B7B0B86A597A5A0A92E
:10034000B1A9481759076A077B0708F478C2048CDB
:10035000F58DE02D80819181A281B3818D8F9E8F5B
:10036000AF8FB8A3D8019096ED91FC912D8D3E8D65
:100370004F8D58A160817181828193810F94A32256
:100380004B015C01F80122A533A544A555A56D8D4F
:100390007E8D8F8D98A10F94A3226B017C01D801D3
:1003A00050962D913D914D915C915397C501B401AB
:1003B0000F941621F80126A137A140A551A50F944D
:1003C000A4222B013C01D80196964D925D926D922C
:1003D0007C929997DB96BC91BDA3B11116C0F80130
:1003E0002485358546855785C701B6010F941621AA
:1003F0009B01AC01C301B2010F94A322D8019696D0
:100400006D937D938D939C939997F80146A057A087
:1004100060A471A4F6A9F98FD801D796BC91BA8FC0
:10042000F801F0ADFB8FD801D996BC91BC8F298D16
:100430003A8D4F2F5B2FC301B2010F94B8231816CA
:100440000CF035C2898D9A8DAB8DBC8DF80186A3D9
:1004500097A3A0A7B1A7FDA1FF2309F440C2D8012B
:100460001C962D913D914D915C911F97C501B40152
:100470000F9416214B015C01F801248935894689C6
:100480005789C701B6010F9416219B01AC01D80111
:1004900096966D917D918D919C9199970F94A32241
:1004A000A50194010F94A4226B017C019B01AC0176
:1004B000698D7A8D8B8D9C8D0F94B02087FD1CC02B
:1004C000F801F2A9F98FD801D396BC91BA8FF8013F
:1004D000F4A9FB8FD801D596BC91BC8F298D3A8D9C
:1004E0004F2F5B2FB601C7010F94B02087FD04C0CA
:1004F000C98EDA8EEB8EFC8ED8015E96ED91FC9162
:10050000898D9A8DAB8DBC8D80839183A283B383BB
:100510008D8D9E8DAF8DB8A1F80182A793A7A4A75A
:10052000B5A789A19AA1ABA1BCA182A393A3A4A3BF
:10053000B5A3D1011496ED91FC9186898823A1F091
:10054000C1010E94FE7D6B017C0120E030E0A90129
:100550000F94B82387FD08C0D1011496ED91FC914A
:10056000C282D382E482F5826BE875E283E59DE086
:100570000E94BAF2D1011296ED91FC910190F081A6
:10058000E02D6081718183E59DE00E9454F265E871
:1005900075E283E59DE00E94BAF2D1011496ED91D7
:1005A000FC91428553856485758583E59DE00E94B5
:1005B0006CC660E875E283E59DE00E94BAF2D10165
:1005C0001496ED91FC91468157816085718583E594
:1005D0009DE00E946CC66EE476E083E59DE00E949B
:1005E00054F2D1011496ED91FC91428153816481C2
:1005F000758183E59DE00E946CC66CE775E283E53A
:100600009DE00E94BAF2D1011496ED91FC91019007
:10061000F081E02D408151816281738183E59DE00D
:100620000E946CC668E775E283E59DE00E94BAF21D
:10063000D1011496ED91FC910190F081E02D44815F
:1006400055816681778183E59DE00E946CC664E7F1
:1006500075E283E59DE00E94BAF2D1011496ED9116
:10066000FC910190F081E02D408551856285738574
:1006700083E59DE00E946CC6D1011496ED91FC913A
:100680008689882331F06DE675E283E59DE00E945E
:10069000BAF283E59DE00E9404F1F1010481158125
:1006A000D8011296CD90DD90ED90FC9015971E9696
:1006B0004D905D906D907C905197A3019201C70180
:1006C000B6010F94A3224B015C0120E030E0A901A8
:1006D0000F94B823181624F0B7FAB094B7F8B09472
:1006E00020E030E040E85FE3C501B4010F94B82397
:1006F000181674F040E050E460E070E0F10182818F
:1007000093810E949D30672B682B692B09F497C059
:10071000D80156968C918111B3CDF10102811381DC
:1007200061E0D80112968D919C910E9428C14C01E4
:1007300020E030E0A901C301B2010F94B020811183
:1007400009C020E030E0A901C701B6010F94B82329
:1007500018165CF040E050E460E070E0C8010E94D0
:100760009D30672B682B692B21F119821A821B821D
:100770001C821D821E821F8218868A818F708A8346
:1007800061E0CE0101960E942A1B29873A874B8798
:100790005C876D877E878F87988BB12CA12CD12C9D
:1007A000C12C79018A019B01AC016FEFC4010F9448
:1007B000961040E050E460E070E0F10182819381A6
:1007C0000E944B30D1011496ED91FC9142815381EE
:1007D00064817581198A1A8A1B8A1C8A8A898F709A
:1007E00080678A8B4D8B5E8B6F8B788F62E0CE013A
:1007F00041960E94031B29833A834B835C836D835C
:100800007E838F839887B12CA12CD12CC12CE988B1
:10081000FA880B891C892D893E894F89588D6FEF85
:10082000C4010F949610D1011496ED91FC91828130
:100830009381A481B58186879787A08BB18BD101E5
:100840001496ED91FC91868981111ACD8789908D3E
:10085000009709F415CD28EE33E0829F7001839F45
:10086000F00C929FF00C11240E9426D19B01AC0148
:10087000F10184809580E114F10489F010E000E03A
:10088000D40152966D917D918D919C915597A12C9B
:10089000B12C65010F94720C882309F4F1CC81E02E
:1008A000F401868B61E0C1010E94837EE9CCD8010E
:1008B000D2968D919D910D90BC91A02D8EA39FA35A
:1008C000A8A7B9A79C01AD01C301B2010F94B02044
:1008D00087FFC1CD8EA19FA1A8A5B9A5B7CD812CB9
:1008E000912C5401C9CD90E080E0CCCCCF93DF9324
:1008F000EC016FE575E283E59DE00E94BAF2EA81C2
:10090000FB810190F081E02D6081718183E59DE0A4
:100910000E9408F1EC81FD81309721F08081918166
:100920000F941E198C819D810F941E1970E060E058
:100930008A819B810E94792D1D821C8281E090E03A
:10094000DF91CF910895CF93DF93EC0164E576E0DA
:1009500083E59DE00E9408F140E050E0BA018A8101
:100960009B810E94BC2DE881F9810484F585E02DEE
:1009700060E0CE0119956D858C810E947DCE6D85DC
:100980008D810E947DCE81E090E0DF91CF9108952E
:10099000CF93DF93EC0163E676E083E59DE00E9470
:1009A00054F2EA81FB810190F081E02D6081718138
:1009B00083E59DE00E9408F18C819D81009711F0F4
:1009C0000F941E1970E060E08A819B810E94792D4E
:1009D0001D821C8281E090E0DF91CF9108952F92DB
:1009E0003F924F925F926F927F928F929F92AF92BF
:1009F000BF92CF92DF92EF92FF920F931F93CF930C
:100A0000DF93CDB7DEB765970FB6F894DEBF0FBEA4
:100A1000CDBF1C01DC0114968D919C911597892BFB
:100A200099F41296ED91FC91FA83E98389E190E0C3
:100A30000F948218BC0189819A810E94792DD1017D
:100A400015969C938E931497F101048115810115DD
:100A5000110569F46CE475E28CEA9CE00E94BAF23C
:100A60008CEA9CE00E9404F190E080E0FCC4D80194
:100A70001D921C920280F381E02DFD8BEC8B309750
:100A800091F0828193819A838983009761F0DC01E0
:100A900018968C9118978F70853029F4CD010E949B
:100AA000BAC1811190C062E175E28CEA9CE00E94BB
:100AB000BAF261E070E0F10184819581892B11F433
:100AC00070E060E04AE050E08CEA9CE00E940BF2AB
:100AD00060E175E28CEA9CE00E94BAF261E070E0AD
:100AE000D10112968D919C91892B11F470E060E0F8
:100AF0004AE050E08CEA9CE00E940BF26EE075E266
:100B00008CEA9CE00E94BAF2D1011296ED91FC9120
:100B100061E070E082819381892B11F470E060E0E4
:100B20004AE050E08CEA9CE00E940BF26CE075E237
:100B30008CEA9CE00E94BAF2D1011296ED91FC91F0
:100B40000280F381E02D80858F7061E070E0853058
:100B500011F470E060E04AE050E08CEA9CE00E9412
:100B60000BF26AE075E28CEA9CE00E94BAF2D101D5
:100B70001296ED91FC91828193810E94BAC161E04D
:100B800070E0823010F070E060E04AE050E08CEA03
:100B90009CE00E940BF28CEA9CE00E9404F166E269
:100BA00075E28CEA9CE00E94BAF28CEA9CE00E941A
:100BB00004F1D101ED91FC910484F585E02D61E013
:100BC000C101199551CF60E089819A810E9428C1A5
:100BD0009B8B8A8B009729F0FC0180858F70853074
:100BE00039F060EF74E28CEA9CE00E94BAF2D3CF55
:100BF0008A899B890E94BAC18150883008F0AEC1B1
:100C0000E82FF0E08827E85FF9478F4F0D947122B5
:100C10007A874D872087AA86888688866F86108681
:100C200067E08A899B890E9428C1FC0190859F709A
:100C3000933009F045C081859285A385B485898369
:100C40009A83AB83BC8391E09D8366E08A899B890C
:100C50000E9428C1FC0190859F70933009F049C023
:100C600081859285A385B4858E839F83A887B98764
:100C700091E09D8364E08A899B890E9428C1FC01E0
:100C800080858F70833009F056C0618572858385B9
:100C900094850F9489234B0163E08A899B890E9484
:100CA00028C1FC0180858F70833009F068C0818580
:100CB0009285A385B4858E879F87A88BB98B6CC0DE
:100CC000923069F461857285838594850F94B7208D
:100CD00069837A838B839C83A1E0AD83B6CF80E068
:100CE00090E0AFE7B3E489839A83AB83BC831D8232
:100CF000ACCF9230D9F461857285838594850F9449
:100D0000B7206E837F8388879987A1E0AD83B2CFB8
:100D100080E090E0AFE7B3E489839A83AB83BC8340
:100D20001E821F82188619861D82A4CF1E821F82F2
:100D3000188619869FCF40EC842E47E2942E49E016
:100D4000A42EB12C823009F0A7CF81849284A38491
:100D5000B484A2CF50EC852E57E2952E59E0A52EF3
:100D6000B12C80E090E0AFE7B3E489839A83AB8352
:100D7000BC831E821F82188619861D828DCF823009
:100D800009F07BC061857285838594850F94B720B7
:100D90006E877F87888B998B62E08A899B890E9406
:100DA00028C1FC0180858F70833009F06BC04184BD
:100DB00052846384748461E08A899B890E9428C17B
:100DC000FC0180858F70833009F087C08185928512
:100DD000A385B4858A879B87AC87BD8760E08A89B5
:100DE0009B890E9428C1FC0190859F70933009F077
:100DF000AAC0C184D284E384F48420E030E0A90155
:100E0000C701B6010F94B02087FFD6C0F7FAF0945F
:100E1000F7F8F094A1E0B0E0BB8BAA8BAC89BD8958
:100E20001496ED91FC9180858F70823009F4C7C0D3
:100E3000833009F40AC280E090E0A0EAB1E409C27C
:100E400030EC832E37E2932E39E0A32EB12C80E0D4
:100E500090E0A0EAB0E48E879F87A88BB98B80E0F2
:100E600090E0AFE7B3E489839A83AB83BC831E82AF
:100E70001F82188619861D828FCF80E090E0A0EA3D
:100E8000B0E419CF823029F5618572858385948518
:100E90000F94B7202B013C018ECF20EC822E27E24D
:100EA000922E29E0A22EB12C80E090E0A0EAB0E4DE
:100EB0008E879F87A88BB98B80E090E0AFE7B3E483
:100EC00089839A83AB83BC831E821F82188619860E
:100ED0001D82412C512C32016ECF823079F5618513
:100EE0007285838594850F94B7206A877B878C876A
:100EF0009D8774CF90EC892E97E2992E99E0A92EC8
:100F0000B12C80E090E0A0EAB0E48E879F87A88BA8
:100F1000B98B80E090E0AFE7B3E489839A83AB8339
:100F2000BC831E821F82188619861D82412C512C7B
:100F300032014A865B866C867D8650CF1A861B8678
:100F40001C861D864BCF923089F56185728583851D
:100F500094850F94B7206B017C014FCF80EC882ED5
:100F600087E2982E89E0A82EB12C80E090E0A0EADC
:100F7000B0E48E879F87A88BB98B80E090E0AFE7C5
:100F8000B3E489839A83AB83BC831E821F82188655
:100F900019861D821B8A1A8A412C512C32014A86DD
:100FA0005B866C867D867301620138CF1B8A1A8A44
:100FB000C12CD12C760132CF1B8A1A8A2FCF6185A2
:100FC0007285838594850F94B720F80162877387B3
:100FD00084879587D80116961D921D921D921C92AA
:100FE0001997F80112821382148215820E9426D169
:100FF000D80152966D937D938D939C935597D10113
:101000001496ED91FC91B1E0B68B908E878A61E0E9
:10101000C1010E94837EF10104811581D8018D9167
:101020009C9167ED74E2892B09F0DDCD8CE390E0B3
:101030000F9482189D8B8C8BC8010296EC89FD89D8
:10104000978F868F0496958F848F065F1F4F11A30D
:1010500000A312AE12AA13AA14AA15AA80E090E067
:10106000AFE7B3E486AB97ABA0AFB1AF84E690E057
:10107000A0E0B0E086A797A7A0ABB1AB8A899B8917
:10108000918F808F20E030E0A901C701B6010F9455
:10109000B02087FD8AC020E030E0A9016A857B8509
:1010A0008C859D850F94B02087FD7FC020E030E0C7
:1010B000A901C301B2010F94B02087FD76C081E081
:1010C00090E0AC89BD895B969C938E935A97E1E042
:1010D000DB96EC93DB97CD92DD92ED92FC92139729
:1010E0008A859B85AC85BD85EC89FD898483958344
:1010F000A683B7834086518662867386C486D5866A
:10110000E686F7862DEC3CEC4CEC5DE36A857B854E
:101110008C859D850F9416214B015C01AC89BD899E
:1011200050968D929D92AD92BC9253972DEC3CECD3
:101130004CEC5DE3C301B2010F9410232B013C0181
:10114000EC89FD89448A558A668A778A8A899B89CF
:10115000019759F5A701960160E070E0CB010F946B
:10116000A322AC89BD891C966D937D938D939C932E
:101170001F97A501940160E070E0CB010F94A322BA
:10118000EC89FD89608B718B828B938BA30192011B
:1011900060E070E0CB010F94A322AC89BD89549626
:1011A0006D937D938D939C9357970E9426D1EC89E4
:1011B000FD8986A497A4A0A8B1A8681979098A090D
:1011C0009B0962A373A384A395A3D1011496ED9107
:1011D000FC918C899D8991838083009709F4DFCCF1
:1011E000DC01DA968C91DA97811147C05E96ED9119
:1011F000FC915F97C080D180E280F380FD01C6A2A0
:10120000D7A2E0A6F1A65C96ED91FC918081918138
:10121000A281B381EC89FD8982A793A7A4A7B5A772
:1012200046A857A860AC71ACA3019201C701B601F2
:101230000F94B82318169CF4AC89BD8996964D92EC
:101240005D926D927C92999718C081859285A38555
:10125000B485F80182879387A487B587BBCEEC89D4
:10126000FD8942A853A864A875A8A3019201C701EB
:10127000B6010F94B02087FDDFCF81E0EC89FD89B6
:1012800082AFFD81FF2309F474C029813A814B812B
:101290005C816E817F81888599850F94B82387FF53
:1012A00068C08E819F81A885B985EC89FD8982AB54
:1012B00093ABA4ABB5AB89819A81AB81BC8186AB82
:1012C00097ABA0AFB1AF068D178DD801CD90DD9053
:1012D000ED90FC90A701960169817A818B819C81B8
:1012E0000F94B02087FF26C089819A81AB81BC8191
:1012F000F80180839183A283B383AC89BD899696DC
:101300004D905D906D907C909997D696CD90DD90A4
:10131000ED90FC90D997A7019601C301B2010F94FB
:10132000B8231816B4F4EC89FD89C6A2D7A2E0A6AA
:10133000F1A61FC0A70196016E817F8188859985DE
:101340000F94B8231816CCF68E819F81A885B98595
:10135000CFCFAC89BD89D296CD90DD90ED90FC9039
:10136000D597A7019601C301B2010F94B02087FD64
:10137000DACF20E030E04AE754E46E857F85888943
:1013800099890F9416210F94822316161706ECF5EF
:101390006B01770FEE08FF08C701B6010F94B72065
:1013A0002B013C01C501B4010F94B5209B01AC0198
:1013B000C301B2010F9410234B015C01AC019B01EE
:1013C000AC89BD8950966D917D918D919C9153977B
:1013D0000F941621EC89FD89608B718B828B938B26
:1013E000A501940164897589868997890F941023D2
:1013F000AC89BD8954966D937D938D939C9357973B
:10140000FD01C6A6D7A6E0AAF1AA68E375E282EAC2
:101410009CE00E94BAF2D1011296ED91FC910190EC
:10142000F081E02D6081718182EA9CE00E9454F29B
:1014300082EA9CE00E9404F1D1011496ED91FC91A6
:1014400080E090E0A0E0B0EC86879787A08BB18B1E
:10145000D101ED91FC910484F585E02D62E0C1019C
:10146000199581E090E065960FB6F894DEBF0FBE47
:10147000CDBFDF91CF911F910F91FF90EF90DF9043
:10148000CF90BF90AF909F908F907F906F905F9024
:101490004F903F902F9008952F923F924F925F92DE
:1014A0006F927F928F929F92AF92BF92CF92DF9274
:1014B000EF92FF920F931F93CF93DF93CDB7DEB7D9
:1014C000C057D1090FB6F894DEBF0FBECDBFFC01E7
:1014D00062960FAF629763961FAF639764962FAFC4
:1014E000649765963FAF659766964FAF6697679628
:1014F0005FAF679768966FAF689769967FAF699798
:1015000086EF800F823008F4A4C4E196FFAEEEAE01
:10151000E197A396FFAFEEAFA397812F8F70282F8F
:1015200030E0AB963FAF2EAFAB97002361F1232B9A
:1015300009F4C0C1873039F5013109F493C1023192
:1015400009F4B0C10031F9F46FEF70E0CE018F5AA9
:101550009F4F0E94901D2A962FAF2A972B963FAF40
:101560002B972C964FAF2C972D965FAF2D972E96DD
:101570006FAF2E972F967FAF2F9760968FAF6097A4
:1015800061969FAF6197A396AEADBFADA39714963A
:10159000ED91FC91309709F47DC286809780AD96DD
:1015A0001FAE1EAEAD97A5961FAE1EAEA5976F9649
:1015B0001FAE1EAE6F97712C612C512C412C8114E3
:1015C000910409F473C264EB75E0C4010E94B0C0D9
:1015D0001C0164EB78E0C4010E94B0C06B969FAF21
:1015E0008EAF6B9762E776E0C4010E94B0C0AF9601
:1015F0009FAF8EAFAF972114310409F42EC16B96C3
:10160000EEADFFAD6B97309709F427C1D101189665
:101610008C918F70823009F020C180858F7082306C
:1016200009F01BC167EA76E0C4010E94B0C0DC018A
:1016300019962D913D914D915C911C97A9962CAFD7
:101640003DAF4EAF5FAFA997E196EEADFFADE1972D
:10165000309709F4BBC0D401CD90DC90BF01C60126
:101660000F94DE26892B09F0B1C062968FAD629788
:10167000811127C163968FAD6397807FAB96EEADE6
:10168000FFADAB97379709F0B2C1882309F478C052
:10169000CE018F5A9F4F0E94511F6B96EEADFFAD4A
:1016A0006B970185128523853485672B682B692B01
:1016B00009F4BAC1023011052105310529F00F3FA7
:1016C0001F4F2F4F3F4F31F566E776E083E59DE0F2
:1016D0000E9454F283E59DE00E9404F121E030E095
:1016E00040E050E06B96AEADBFAD6B9719962D9371
:1016F0003D934D935C931C9761E0CE018F5A9F4FB1
:101700000E942A1B29A33AA34BA35CA36DA37EA32B
:101710008FA398A7CE018F5A9F4F0E94511FF101AE
:1017200061877287838794878091820E9091830E60
:10173000059731F1D401CD90DC90E12C93E0F92EA6
:1017400062960FAD629763961FAD639764962FAD57
:10175000649765963FAD659766964FAD66976796B9
:101760005FAD679768966FAD689769967FAD69972B
:10177000A396EEADFFADA397828193810E94C13005
:10178000AF96EEADFFADAF97309701F1B12CA12C24
:10179000D12CC12C6296EFAC62976396FFAC639735
:1017A00064960FAD649765961FAD659766962FADED
:1017B000669767963FAD679768964FAD689769964D
:1017C0005FAD69976FEFCF010F9496106B96EEADFA
:1017D000FFAD6B9781859285A385B4858230910595
:1017E000A105B105A1F18F3F9F4FAF4FBF4F79F1D9
:1017F000F10181859285A385B485A7964EAD5FAD35
:10180000A797849F9001859F300D949F300D1124E0
:10181000420E531EAD96EEADFFADAD97AF01FF0F7B
:10182000660B770B481759076A077B0784F4AD9658
:101830009FAF8EAFAD97A5963FAF2EAFA597A7965A
:101840002EAD3FADA7976F963FAF2EAF6F97A79680
:101850004EAD5FADA797640E751ED40112968D90A4
:101860009C90ADCE60E870E0CE018F5A9F4F0E94F1
:10187000901D22962FAF229723963FAF2397249651
:101880004FAF249725965FAF259726966FAF269783
:1018900027967FAF279728968FAF289729969FAFD7
:1018A000299771CE6AE070E0CE018F5A9F4F0E9457
:1018B000B61E69CE41E050E0AB965FAF4EAFAB973E
:1018C00062CE482F50E070E060E06B96AEADBFADE9
:1018D0006B9719964D935D936D937C931C97813014
:1018E00009F462C0823009F472C08091820E909136
:1018F000830E059761F16B96EEADFFAD6B97818519
:101900009285A385B4850197A105B10501F5F10183
:1019100081859285A385B4854497A105B105BCF462
:101920002EE130E040E050E0218732874387548742
:101930006EE170E0CE018F5A9F4F0E94901D29A743
:101940003AA74BA75CA76DA77EA78FA798AB8091FE
:10195000820E9091830E059709F412CFF401C08096
:10196000D180E12C23E0F22E62960FAD6297639650
:101970001FAD639764962FAD649765963FAD6597ED
:1019800066964FAD669767965FAD679768966FAD41
:10199000689769967FAD6997A396AEADBFADA397E3
:1019A00012968D919C91EACEF10161857285CE01EE
:1019B0008F5A9F4F0E94901D29AF3AAF4BAF5CAF3B
:1019C0006DAF7EAF8FAF21969FAF21978ECF70E026
:1019D00060E0CE018F5A9F4F0E94901D29AB3AAB19
:1019E0004BAB5CAB6DAB7EAB8FAB98AF7ECF882340
:1019F00009F4C6CE60E0CE018F5A9F4F0E94E91DC8
:101A0000092E000CAA0BBB0BF10181879287A387DB
:101A1000B4878091820E9091830E059709F4B0CE21
:101A2000E12C82E0F82EA0CF02301105210531050E
:101A300059F10F3F1F4F2F4F3F4F31F161E876E0D3
:101A400083E59DE00E9454F283E59DE00E9404F14D
:101A500022E030E040E050E06B96AEADBFAD6B975A
:101A600019962D933D934D935C931C9762E0CE01A4
:101A70008F5A9F4F0E942A1B298F3A8F4B8F5C8F62
:101A80006D8F7E8F8F8F98A3F1011186128613863A
:101A900014864ACEA5961FAE1EAEA5976F961FAEB2
:101AA0001EAE6F97712C612C512C412C6114710466
:101AB00009F4CFC1C201B3010F945D224B016EEC5A
:101AC00074E283E59DE00E94BAF24AE050E0B3017F
:101AD00083E59DE00E940BF263EC74E283E59DE0F8
:101AE0000E94BAF20FEF10E0C201B8010F945D221C
:101AF0004AE050E083E59DE00E940BF26CEB74E25B
:101B000083E59DE00E94BAF24AE050E0B40183E52B
:101B10009DE00E940BF26EEA74E283E59DE00E9474
:101B2000BAF2A5968EAD9FADA597B8010F945D2230
:101B30004AE050E083E59DE00E940BF267EA74E220
:101B400083E59DE00E94BAF24AE050E06F966EADE8
:101B50007FAD6F9783E59DE00E940BF263EA74E22C
:101B600083E59DE00E94BAF283E59DE00E9404F1C6
:101B700019821A821B821C821D821E821F82188675
:101B80008A818F708A83B401CE0101960E94901DD4
:101B900029873A874B875C876D877E878F87988BED
:101BA00061E08114910409F462E0CE0109960E947B
:101BB0002A1B79018A012B013C01298BFA8A4B8B64
:101BC0001C8B6D8B5E8A8F8B788E6BE178E0A39691
:101BD000EEADFFADA397848195810E94B0C0B12C7A
:101BE000A12CD12CC12C9201A3016FEF0F94961060
:101BF0008928E1F481E090E0C059DF4F0FB6F894F6
:101C0000DEBF0FBECDBFDF91CF911F910F91FF902F
